:100000000C944B300C9473300C9473300C9473300C
:100010000C9473300C9473300C9473300C947330D4
:100020000C9473300C9426720C9431720C947330CF
:100030000C9473300C942C5D0C9473300C947330CE
:100040000C944E740C9473300C9473300C94733085
:100050000C9429580C9473300C9473300C947330B6
:100060000C94A2B60C9473300C94CBB20C947330F5
:100070000C9480530C94B8530C9473300C947330DC
:100080000C9484720C9473300C9473304D875787A2
:1000900061877587868793876D88A487B18708886D
:1000A00043885A882599289930992D9933993699FA
:1000B00039993E99439948994D995099559958992C
:1000C0005D99EBB208B346B3ACB3C4B3FFB3AEB4FF
:1000D0004AB54AB54AB54AB54AB54AB54AB54AB528
:1000E0004AB54AB54AB54AB54AB54AB51EB520B56E
:1000F000DEC6EFC6F6C609C722C732C73FC75AC712
:100100005EC7E6CDEACDEECDF2CDF6CD4ECE0BCE2E
:100110000FCE13CE1DCE21CE9FCDBACDBECDC2CD3A
:10012000C6CDCACDCECDD2CDD6CDDACDDECDE2CDC7
:10013000B0CD2BCE4ACE05A84CCDB2D44EB9383670
:10014000A9020C50B9918688083CA6AAAA2ABE002A
:100150000000803F07634236B79BD8A71A3968561C
:1001600018AEBAAB558C1D3CB7CC5763BD6DEDFDD9
:10017000753EF6177231BF000000803F0800000096
:10018000BE922449123EABAAAA2ABECDCCCC4C3E8C
:1001900000000080BEABAAAAAA3E00000000BF007B
:1001A0000000803F0000000000084178D3BB438777
:1001B000D1133D190E3CC3BD4282AD2B3E68EC828B
:1001C00076BED98FE1A93E4C80EFFFBE01C4FF7F10
:1001D0003F0000000000332E362E376400536F6658
:1001E00074776172653A0031312E32303132004815
:1001F0006172647761726520504B5420332E3978D8
:100200000030392E323031310048617264776172CA
:100210006520504B5420332E396D004576616C7546
:100220006174696F6E20283836384D487A2920204D
:1002300000526164696F74726F6E69782057692E1D
:100240003233324454530042617564726174653ACA
:1002500020004B6162656C20616E7363686C696538
:100260007373656E2E202000504B542065696E20FC
:1002700067656B7265757A746573202020005A7704
:1002800069736368656E204D4B2D55534220756E22
:10029000642020004D4B2D55534220616E20504369
:1002A00020616E7363686C2E20004643203E204D13
:1002B0004B2D555342203E2042544D2D32323200B8
:1002C00042544D2D323232204B6F6E666967757223
:1002D000696572656E0042617564726174653A2089
:1002E0000052452D49443A200042617564726174A0
:1002F000653A20004665686C65723A204B65696E08
:100300006520446174656E00464300204E61766945
:100310002D4374726C20446973706C6179202020C5
:10032000004E430020466C696768742D4374726CFC
:1003300020446973706C617920002020002044699A
:1003400073706C6179202020202020202020202024
:10035000202000464300204E6176692D4374726C64
:1003600020446973706C6179202020004E43002086
:10037000466C696768742D4374726C2044697370AD
:100380006C6179200020200020446973706C6179D1
:100390002020202020202020202020202000464334
:1003A00000204E6176692D4374726C20446973702D
:1003B0006C6179202020002E002E00302E38386EFF
:1003C00000454550726F6D5265762000454550726C
:1003D0006F6D52657620002E003F004F5344202061
:1003E000202020202020202020202020004F5344A7
:1003F0002020202020202020202020202020004FEE
:100400005344202020202020202020202020202095
:10041000004D4B20446973706C61792020202020AE
:100420002020004D4B20446973706C61792020209E
:1004300020202020004D4B20446973706C6179208E
:1004400020202020202000547261636B696E672099
:10045000202020202020202000547261636B696ED0
:100460006720202020202020202000547261636B10
:10047000696E6720202020202020202000506172FB
:10048000616D657465722020202020201D000050C1
:100490006172616D6574657220202020201D00004E
:1004A00000506172616D6574657273202020201D9B
:1004B000000000446562756720446174612020205B
:1004C000202020200044656275672044617461200B
:1004D000202020202020004465627567204461743C
:1004E00061202020202020200047505320496E66A4
:1004F0006F2020202020202020200047505320491A
:100500006E666F202020202020202020004750539E
:1005100020496E666F2020202020202020200046C9
:100520006F6C6C6F77204D652020202020202020CC
:1005300000466F6C6C6F77204D65202020202020B6
:10054000202000466F6C6C6F77204D6520202020A6
:1005500020202020004A6F79737469636B2020206B
:10056000202020202020004A6F79737469636B205B
:100570002020202020202020004A6F797374696396
:100580006B20202020202020202000504B5420547D
:100590006F6F6C732020202020201D0000504B54D2
:1005A00020546F6F6C7320202020201D000000500D
:1005B0004B5420546F6F6C7320202020201D0000AE
:1005C000004D4B20446973706C61792020202020FD
:1005D0002020004D4B20446973706C6179202020ED
:1005E00020202020004D4B20446973706C617920DD
:1005F00020202020202000506172616D657465729A
:10060000202020202020201D00506172616D657423
:100610006572202020202020201D00506172616D15
:1006200065746572202020202020201D0044656212
:100630007567204461746120202020202020004420
:10064000656275672044617461202020202020208D
:100650000044656275672044617461202020202079
:10066000202000504B5420546F6F6C7320202020AA
:100670002020201D00504B5420546F6F6C7320209D
:1006800020202020201D00504B5420546F6F6C738D
:10069000202020202020201D005375636865204DF8
:1006A000696B726F6B6F70746572007365617263F2
:1006B00068204D696B726F6B6F7074200073656199
:1006C000726368204D696B726F6B6F7074200042AB
:1006D0004C2D4374726C2E20546573746572202007
:1006E00000424C2D4374726C2E20546573746572F5
:1006F000202000424C2D4374726C2E20546573747C
:100700006572202000504320425420203E204B6F31
:1007100070746572202000504320425420203E20F7
:100720004B6F70746572202000504320425420208B
:100730003E204B6F7074657220200050432055534B
:1007400042203E204B6F7074657220200050432081
:10075000555342203E204B6F70746572202000502C
:100760004320555342203E204B6F70746572202009
:1007700000504B5420536574757020202020202099
:10078000201D00504B54205365747570202020208C
:100790002020201D00504B5420536574757020207C
:1007A00020202020201D00504B5420566572736974
:1007B0006F6E20202020202000504B542056657260
:1007C00073696F6E20202020202000504B5420564B
:1007D00065727369652020202020202000202020C1
:1007E0002020202020202020202020202020202009
:1007F00020200028432920474E552047504C204CAC
:100800006963656E7365202000202020204E4F20F4
:1008100057415252414E5459202020202020002080
:1008200020202020202020202020202020202020C8
:100830002020202000323030382054686F6D6173E2
:10084000204B616973657220202000323030392DD1
:1008500032303130205065746572204D61636B20F9
:1008600000323031302053656261737469616E20EB
:10087000426F65686D200032303132204368722E3D
:10088000204272616E64746E657220260020202002
:100890002020486172616C6420426F6E67617274DF
:1008A0007A20003230313220676562616420202076
:1008B00020202020202020200032303132204D61A5
:1008C0007274696E2052756E6B656C202020003248
:1008D000303133204F6C697665722047656D6573E2
:1008E00069202020002000120013001200130020B5
:1008F0000020202020202020202020202020202018
:1009000020202020202000332E362E376400504B2C
:100910005420546F6F6C2020562E20202020202041
:1009200020202000456E646500206E696368742095
:100930006DF6676C6963682100204D6974206469F5
:1009400065736572204861726477617265002D5528
:10095000666C6173683A773A46494C452E6865780B
:100960003A6120002D50636F6D3F202D623131358B
:10097000323030202020202020002D706D31323880
:100980003470202D636176723130392020202000B0
:10099000537461727420617672647564652E657833
:1009A00065202020200020504B5420557064617435
:1009B0006520202020202020202020002020202012
:1009C000206E6F7420706F737369626C65202020D5
:1009D00020200020202020206E6F7420706F737301
:1009E00069626C652020202000302E38386E00505F
:1009F0004B542D546F6F6C2046432000130012009F
:100A0000302E38386E00504B542D546F6F6C20468A
:100A10004320001D00200015000101010101011506
:100A20000017012D014301150059016F01850115C2
:100A3000009B01AD01BF011500D101DB01E50115EE
:100A400000EF01F901030215000D021D022D021530
:100A5000003D024E026302150078028E02A20215CA
:100A600000B702CD02DA021500ED020303170315E9
:100A7000002B034103410315005703680379031555
:100A8000008B038B038B0315009B039B039B0315B8
:100A900000A603A603A6031500B203B203B2031512
:100AA00000BF03BF03BF031500CC03CC03CC031569
:100AB00000DA03DA03DA031500E703E703E70315B7
:100AC00000F503F503F5031500020418042E0415C0
:100AD0000044045A047004150086049C04B20415F2
:100AE00000C804DE04DE041500F4040A0520051520
:100AF00000360546055605150066056C0572051598
:100B00000078057D05820515008705900599051576
:100B100000A205A905B0051500B705CA05D8051539
:100B200000EA05EA05EA051500FB0506060E0615AE
:100B300000190619061906150025062506250615AD
:100B4000002F062F063906150043064C06550615DC
:100B5000005E0667067006150079068A069D061572
:100B600000B106B106B1061500BE06C906D40615C9
:100B700000DF06E506EB061500F106F706FD061593
:100B800000030703070307150007071A072B0715BC
:100B90000040074A07540715005E0774078A0715C7
:100BA00000A007B607CC071500E207F8070E0815E6
:100BB0000024083A085008150066087B088F0815BD
:100BC000009D08AA08B7081500C408DA08E6081549
:100BD00000FC080F092209150035094609500915BE
:100BE00000620978098B091500A009B609C8091522
:100BF00000DC09F209FC0915000E0A210A2D0A156C
:100C0000003B0A4E0A5A0A15006E0A820A960A1515
:100C100000A90AB90A50091500C80ADA0AEC0A152F
:100C200000FE0A140B2A0B1500400B500B630B152A
:100C300000780B880B980B1500AA0BAA0BAA0B15B2
:100C400000C00BD60BEC0B1500020C180C2E0C156B
:100C500000440C5A0C700C1500860C860C860C1582
:100C6000009C0CAC0CAC0C1500BA0CD00CE60C15AE
:100C700000FC0C120D210D1500320D480D5E0D15F6
:100C800000730D730D730D1500890D9F0DB50D15B6
:100C900000CB0DE10DF70D15000D0E230E390E15CD
:100CA000004F0E650E6D0E1500790E7F0E790E1534
:100CB00000850E850E850E15008E0E8E0E960E1575
:100CC000009E0EA60EAE0E1500D101B60EC00E157A
:100CD00000CA0EDB0EE90E1500FB0E050F0E0F15F8
:100CE00000170F230F2F0F15003B0F470F530F1542
:100CF000005F0F6B0F770F1500830F8F0F9B0F1582
:100D000000A70FBD0FD30F1500E90FFA0F0B101539
:100D1000001C10271032101500391049105A1015F8
:100D2000006A107810861015009410A210A21015F9
:100D300000B010B010B0101500BF10BF10BF1015DC
:100D400000CD10DD10DD101500ED10ED10ED1015CB
:100D500000F710F710F7101500061106110611150F
:100D60000015111511151115002411241124111548
:100D7000003311331133111500431155116711154B
:100D80000079118F119E111500AF11BA11C4111500
:100D900000D611DB11D6111500E011E511EA11158D
:100DA00000EF110512051215001B12311242121527
:100DB00000AF11BA11C41115005412661278121541
:100DC000008A12A012A0121500B612C412D2121577
:100DD00000E112F112F1121500B612C412D212156E
:100DE00000011317132B1315004013531360131531
:100DF0000076137613851315009413961396131526
:100E00000098139A139C1315009E139E139E13159E
:100E100000A013A013A0131500A213A213A2131570
:100E200000A513A513A5131500A813AB13AB131539
:100E300000AE13C413D5131500EB13FB13071415E1
:100E400000161420142A141500331449145F1415C5
:100E50000075147C14831415008F149A14A31415B0
:100E600000AD14B714C1141500CD14E314F3141518
:100E700000091519152415150032154215501515C0
:100E800000601571157E1515008A15A015B615158B
:100E900000CC15DF15EC151500F8150E16241615E7
:100EA0000036164C166216150078168E16A4161506
:100EB00000BA16D016E6161500FC161217281715DC
:100EC000003E175417541715006A1780178017151E
:100ED000009617AC17AC171500C217D017D017150E
:100EE00000DE17EC17EC171500FA1708180818158C
:100EF0000016182418241815003218401840181528
:100F0000004E185C185C1815006A187818781815C7
:100F10000086188618861815008E188E188E1815DB
:100F2000009618A518A5181500B418C718C71815E5
:100F300000DA18E518E5181500F018FB18FB18156D
:100F40000006191119111915001C1927192719154F
:100F50000032193219321915003C193C193C191587
:100F60000046194619461915004B194B194B19150E
:100F700000501950195019150055196119611915AA
:100F8000006D1979197919150085198519851915B3
:100F900000321932193219150091199B199B191534
:100FA00000A519A519A5191500AF19B919B9191571
:100FB00000C319CD19CD191500D719E119E119157B
:100FC00000EB19F519FF191500091A1F1A1F1A1538
:100FD00000351A461A461A1500571A661A661A1567
:100FE00000751A861A861A1500971AA81AA81A15D3
:100FF00000B91ACA1ACA1A1500DB1AED1AED1A1529
:1010000000FF1A0F1B0F1B15001F1B2F1B2F1B157B
:10101000003F1B4F1B4F1B1500611B611B611B1504
:1010200000701B701B701B1500831B831B831B151B
:1010300000931BA41BA41B1500B51BB51BB51B15EA
:1010400000C61BD71BD71B1500E81BF91BF91B1586
:10105000000A1C1B1C1B1C15002C1C421C421C15CE
:10106000002C1C421C421C1500571C651C651C15DD
:1010700000731C891C891C15009F1CB01CB01C151A
:1010800000C11CD71CD71C1500ED1C031D031D152A
:1010900000191D191D191D1500221D291D291D15B9
:1010A00000301D381D381D15003F1D461D461D15FD
:1010B000004E1D611D611D1500741D871D871D15C6
:1010C000009A1DAD1DAD1D1500C01DD31DD31D15EE
:1010D00000E61DF91DF91D15000C1E1F1E1F1E1513
:1010E00000321E451E451E1500581E581E581E155E
:1010F000006B1E761E761E1500811E811E811E1538
:1011000000941EA71EA71E1500BA1ECD1ECD1E15CB
:1011100000E01EF31EF31E1500061F131F131F15FC
:1011200000201F2D1F2D1F15003A1F4B1F4B1F1591
:1011300000591F6C1F6C1F15007F1F861F861F150F
:10114000008D1F941F941F4B616EE46C652020205E
:101150002020202020004368616E6E656C202020D6
:1011600020202020004B616E61616C202020202017
:10117000202020004B6F6E66696775726174696F1D
:101180006E20006D61696E2020202020202020200C
:101190002000436F6E66696775726174696520200F
:1011A00000537469636B2020202020202020200021
:1011B000737469636B20202020202020202000539E
:1011C0007469636B202020202020202020004C6F99
:1011D0006F70696E6720202020202020004C6F6FE8
:1011E00070696E6720202020202020004C6F6F70D7
:1011F000696E67202020202020200048F6686520A6
:1012000020202020202020202000416C746974754B
:10121000646520202020202000486F6F67746520BF
:1012200020202020202020004B616D65726120204D
:101230002020202020200043616D65726120202045
:1012400020202020200043616D6572612020202035
:1012500020202020004E6176694374726C2020208B
:10126000202020004E6176694374726C202020207B
:101270002020004E6176694374726C20202020206B
:10128000200041757367E46E6765202020202020D0
:10129000004F75747075747320202020202020006A
:1012A00055697467616E67656E20202020200056A6
:1012B0006572736368696564656E6573200044696F
:1012C000766572732020202020202020004469763B
:1012D000657273656E202020202020004779726F90
:1012E00020202020202020202020004779726F20FD
:1012F000202020202020202020004779726F2020ED
:1013000020202020202020200042656E75747A6500
:10131000722020202020200055736572202020207C
:10132000202020202020004765627275696B65725D
:10133000202020202000416368736B6F70706C75F3
:101340006E67202000436F75706C204178657320B4
:10135000202020004B6F7070656C696E67204173B0
:101360007320004D697865722D5365747570202067
:101370002000436F6E666967204D69782020202029
:1013800000436F6E6669672E204D69786572200094
:1013900045617379205365747570202020200043C7
:1013A0006F6E666967204561737920202000436F66
:1013B0006E6669672E20656173792020004761732E
:1013C0002020202020202020202020005468726F20
:1013D00074746C6520202020202000476173202039
:1013E0002020202020202020200047696572202016
:1013F0002020202020202020004769657220202006
:1014000020202020202020004769657220202020F5
:10141000202020202020004E69636B2020202020E7
:101420002020202020004E69636B202020202020D7
:1014300020202020004E69636B20202020202020C7
:1014400020202000526F6C6C2020202020202020A3
:10145000202000526F6C6C20202020202020202093
:101460002000526F6C6C2020202020202020202083
:1014700000506F746920312020202020202020007F
:10148000506F74692031202020202020202000501F
:101490006F74692031202020202020202000506FF0
:1014A00074692032202020202020202000506F74DA
:1014B000692032202020202020202000506F7469D5
:1014C0002032202020202020202000506F7469200E
:1014D00033202020202020202000506F74692033EA
:1014E000202020202020202000506F7469203320ED
:1014F0002020202020202000506F746920342020DC
:1015000020202020202000506F74692034202020CB
:10151000202020202000506F7469203420202020BB
:101520002020202000506F746920352020202020AA
:1015300020202000506F746920352020202020209A
:10154000202000506F74692035202020202020208A
:101550002000506F74692036202020202020202079
:1015600000506F7469203620202020202020200089
:10157000506F746920362020202020202020005029
:101580006F74692037202020202020202000506FF9
:1015900074692037202020202020202000506F74E4
:1015A000692037202020202020202000506F7469DF
:1015B0002038202020202020202000506F74692017
:1015C00038202020202020202000506F74692038EF
:1015D0002020202020202020004D6F746F72205387
:1015E0006963682E536368004D6F742E536166659E
:1015F00074792053772E004D6F742E7361662E73AD
:101600006368616B2E004D6F746F72205377692E83
:101610004D6F6465004D6F746F72205377692E4D66
:101620006F6465004D6F746F72205377692E4D6F34
:101630006465004572772E205369672E2050722E04
:101640002000456E682E205369672E436865636BE2
:1016500000556974672E5369672E436865636B0094
:10166000456D7066E46E6765722054797020005293
:1016700065636569766572205479706520004F6EE8
:101680007476616E672E2054797065200048F66884
:10169000656E726567656C65722020004374726CBC
:1016A00020416C74697475646520004374726C2009
:1016B000486F6F677465202020004750532020201A
:1016C00020202020202020200047505320202020B0
:1016D00020202020202020004750532020202020A0
:1016E000202020202020004B6F6D7061737320201C
:1016F000202020202000436F6D7061737320202014
:1017000020202020004B6F6D70617320202020204E
:10171000202020004B6F6D704665737420417573F7
:10172000722E00436F6D704F7269656E742E46693C
:1017300078004B6F6D706173207661737420202088
:10174000004572772E205369672E2050722E20009C
:1017500053656E732E52637653696756616C00450C
:101760007874526563205369676E61616C004163F0
:10177000687328652E296B6F70706C2E0041786934
:101780007320436F7570696E672020004173206B72
:101790006F7070656C696E672020004472656872B6
:1017A0006174656E626567722E00526F7452617467
:1017B00065206C696D69742E00526F745261746596
:1017C000206C696D69742E0048656164696E6720DC
:1017D000486F6C642020004E69636B2F526F6C6CF5
:1017E0002020202020004B6F657273207661737477
:1017F00020202020004E69636B2F526F6C6C2050AC
:10180000202020004E69636B2F526F6C6C2050209B
:101810002020004E69636B2F526F6C6C205020208B
:1018200020004E69636B2F526F6C6C204420202087
:10183000004E69636B2F526F6C6C20442020200097
:101840004E69636B2F526F6C6C2044202020004740
:101850006965722050202020202020202000476928
:10186000657220502020202020202020004769651C
:1018700072205020202020202020200045787465F0
:10188000726E65204B6F6E74722E004578746572AF
:101890006E204374726C2020200045787465726E4F
:1018A00020436F6E74726F6C004C6F6F70696E675F
:1018B000206F62656E2020004C6F6F70696E67202C
:1018C000757020202020004C6F6F70696E67206F4C
:1018D0006D686F6F67004C6F6F70696E6720756E13
:1018E00074656E20004C6F6F70696E6720646F774F
:1018F0006E2020004C6F6F70696E672062656E65A8
:10190000642E004C6F6F70696E67206C696E6B732C
:1019100020004C6F6F70696E67206C6566742020C4
:10192000004C6F6F70696E67206C696E6B7320007E
:101930004C6F6F70696E6720726563687473004CDA
:101940006F6F70696E6720726967687420004C6FF2
:101950006F70696E672072656368747300476173A6
:10196000204C696D69742020202020005468726F1B
:1019700074746C65204C696D697400476173204C08
:10198000696D6965742020202000416E7370726556
:101990006368736368772E2000526573702E20543D
:1019A00068726573682E20004472656D70656C778F
:1019B000616172646520004879737465726573654E
:1019C0002020202020004879737465726573697344
:1019D000202020200048797374657265736520208B
:1019E00020202000556D6B656872702E204E696353
:1019F0006B20005475726E6F766572204E69636B52
:101A000020004E69636B206765696E766572742E7F
:101A100000556D6B656872702E20526F6C6C2000E3
:101A20005475726E6F76657220526F6C6C20005226
:101A30006F6C6C206765696E766572742E0048F66F
:101A400068656E726567656C756E672000416C74C1
:101A50006974756465204374726C2000486F6F6709
:101A6000746520436F6E74726F6C004A3A48426529
:101A7000672C4E3A566172696F00593A4C696D484D
:101A80002C4E3A566172696F00593A4C696D482C78
:101A90004E3A566172696F00536368616C74657287
:101AA00020662E20482E007573652053772E206601
:101AB0002E5365747000536368616B2E20486F6FFE
:101AC0006774652000616B7573742E2056617269AE
:101AD0006F20200061636F757374696320566172B3
:101AE000696F00416B6F6573742E20566172696F68
:101AF0002000536F6C6C68F6686520202020202041
:101B000000536574706F696E7420202020202000BF
:101B1000476577656E73746520686F6F6774004DF5
:101B2000696E2E20476173202020202020006D69DF
:101B30006E2E207468726F74746C6520004D696E2F
:101B4000696D61616C2067617320200048F66865EB
:101B50002050202020202020202000416C74697417
:101B600075646520502020202000486F6F677465E1
:101B70002050202020202020004C7566746472754F
:101B8000636B2044202020004261726F6D65747287
:101B9000696320442020004261726F6D6574722E6B
:101BA0002044202020005A2D414343202020202083
:101BB0002020202000414343205A202020202020A4
:101BC00020202000414343205A2020202020202094
:101BD0002020004D61782E2048F6686520202020C6
:101BE00020004D61782E20416C7469747564652005
:101BF000004D61782E20686F6F677465202020008B
:101C00005665727374E4726B756E672F52200067AD
:101C100061696E2F72617465202020202000566556
:101C20007273742E2F7261746520202000536368D4
:101C300077656265676173202B2F2D00686F6F7663
:101C400065722076617269612E2000686F6F76651B
:101C5000722076617269612E2000475053205A200D
:101C6000202020202020202000475053205A2020D0
:101C70002020202020202000475053205A202020C0
:101C800020202020202000537469636B204E65754E
:101C900074722E205000737469636B206E657574C6
:101CA000722E205000737469636B206E65757472B8
:101CB0002E2050004E69636B20532E20416E7374AA
:101CC0002E20006E69636B207365727620637472D8
:101CD0006C006E69636B2073657276206374726C3E
:101CE000004E69636B204B6F6D70656E732E200024
:101CF0006E69636B20636F6D70656E732E20006E6E
:101D000069636B20636F6D70656E732E20004E6982
:101D1000636B20556D6B656872656E20006E69633C
:101D20006B20696E762E206469722E006E69636B7B
:101D300020696E762E726963682E004E69636B208F
:101D4000536572766F206D696E006E69636B2073E8
:101D50006572766F206D696E006E69636B207365C6
:101D600072766F206D696E004E69636B20536572E9
:101D7000766F206D6178006E69636B207365727693
:101D80006F206D6178006E69636B20736572766F8A
:101D9000206D6178004E69636B2053657276204632
:101DA000696C74004E69636B2053657276204669D6
:101DB0006C74004E69636B20536572762046696CC3
:101DC0007400526F6C6C20532E20416E73742E2061
:101DD00000726F6C6C2073657276206374726C0095
:101DE000726F6C6C2073657276206374726C005233
:101DF0006F6C6C204B6F6D70656E732E2000726F70
:101E00006C6C20636F6D70656E732E2000726F6C4A
:101E10006C20636F6D70656E732E2000526F6C6C5A
:101E200020556D6B656872656E2000726F6C6C205A
:101E3000696E762E206469722E00726F6C6C206F52
:101E40006D6B6572656E202000526F6C6C2053655F
:101E500072766F206D696E00726F6C6C20736572A4
:101E6000766F206D696E00726F6C6C207365727690
:101E70006F206D696E00526F6C6C20536572766FC7
:101E8000206D617800726F6C6C20736572766F20C4
:101E90006D617800726F6C6C20736572766F206D67
:101EA000617800526F6C6C20536572762046696CC5
:101EB0007400526F6C6C20536572762046696C74A6
:101EC00000526F6C6C20536572762046696C74000A
:101ED000416E73742E204765736368772E200073FC
:101EE0006572766F2072656672657368200053654F
:101EF00072766F207265667265736820004D616E40
:101F000075656C6C65204765736368006D616E75FF
:101F1000656C6C2053706565642000536E656C6859
:101F20002E68616E646265642E0043616D205269A3
:101F3000636874756E6720200043616D204F72697D
:101F4000656E74202020200043616D6572612072EF
:101F5000696368742E2000536572766F20332020E9
:101F6000202020202000536572766F20332020200F
:101F70002020202000536572766F203320202020FF
:101F800020202000536572766F20342020202020EE
:101F9000202000536572766F2034202020202020DE
:101FA0002000536572766F203420202020202020CE
:101FB00000536572766F20352020202020202000DD
:101FC000536572766F20352020202020202000537A
:101FD0006572766F20352020202020202000475079
:101FE00053202020202020202020202000656E610A
:101FF000626C65204750532020202000656E61628E
:102000006C65204750532020202000475053204D1E
:102010006F6475732053742E2000475053206D6FEA
:10202000646520636F6E747200475053206D6F6457
:102030006520636F6E74720047505320566572734B
:1020400074E4726B2E2000475053204761696E2064
:10205000202020202000475053207665727374653D
:10206000726B2E20004750532053742E2053636808
:10207000772E200047505320737469636B20746877
:102080007265004750532073742E206472656D7022
:102090002E004D696E2E205361742E2020202020AA
:1020A000004D696E2E205361742E202020202000C8
:1020B0004D696E2E205361742E2020202020004771
:1020C00050532D5020202020202020202000475039
:1020D000532D502020202020202020200047505326
:1020E0002D50202020202020202020004750532D3C
:1020F00049202020202020202020004750532D4917
:10210000202020202020202020004750532D49202F
:102110002020202020202020004750532D44202024
:1021200020202020202020004750532D4420202014
:10213000202020202020004750532D442020202004
:1021400020202020200050204C696D697420202020
:1021500020202020004C696D697420205020202010
:10216000202020004C696D696574202050202020BB
:1021700020200049204C696D6974202020202020F7
:1021800020004C696D6974202049202020202020E7
:10219000004C696D696574202049202020202000B2
:1021A00044204C696D697420202020202020004CA0
:1021B000696D6974202044202020202020004C6973
:1021C0006D69657420204420202020200047505352
:1021D00020416363202020202020200047505320EE
:1021E00041636320202020202020004750532041BD
:1021F000636320202020202020004750532057696F
:102200006E646B6F72722E20004750532057696EB8
:102210006420436F72722E004750532057696E64DA
:1022200020436F72722E004272656D737769726B14
:10223000756E67202000537065656420636F6D7054
:10224000656E732E0052656D7765726B696E6720DF
:1022500020202000475053206D61782E2052616469
:102260002E2000475053206D61782E72616469758D
:102270007300475053206D61782E726164697573E5
:10228000004750532057696E6B656C204C692E00D7
:1022900047505320616E676C2E6C696D69740047FE
:1022A000505320686F656B206C696D2E200050487C
:1022B000204C6F67696E2074696D6520005048205E
:1022C0006C6F67696E2074696D6520005048206CE2
:1022D0006F67696E2074696A64200044796E616D6D
:1022E0006963205048202020200044796E616D6988
:1022F00063205048202020200044796E616D69736E
:102300006368652050482000475053206D2E2052AE
:1023100061642064504800475053206D2E20526164
:10232000642064504800475053206D2E2052616451
:10233000206450480043482048F66865202020204B
:1023400020202000434820416C7469747564652026
:10235000202000434820486F6F67746520202020AC
:1023600020004C454431204269746D61736B6520D7
:10237000004F757431204269746D61736B202000C9
:10238000556974673120426974706174722E00203F
:102390002020202054696D696E67202020004F7531
:1023A00074312054696D696E67202020005569746E
:1023B00067312054696D696E67202000202020203D
:1023C00020736F666F727420616E0041637469766A
:1023D0002020202020202020200044697265637482
:1023E0002061616E202020200020202020206E2EE1
:1023F0006D2E4D6F746F72004163742E2077692EBD
:10240000204D6F746F7200416B742E206D6F746F6E
:102410007220756974004C454432204269746D61C4
:10242000736B6520004F757432204269746D61735F
:102430006B202000556974673220426974706174A2
:10244000722E00202020202054696D696E672020A4
:1024500020004F7574322054696D696E672020200A
:102460000055697467322054696D696E67202000D9
:102470002020202020736F666F727420616E0041EF
:1024800063746976202020202020202020004469C9
:10249000726563742061616E20202020002020205E
:1024A00020206E2E6D2E4D6F746F72004163742E5E
:1024B0002077692E204D6F746F7200416B742E204F
:1024C0006D6F746F7220756974004F75743120568A
:1024D0006D696E2E5761726E004F75743120756E86
:1024E000646572766F6C74005569746731206F6E25
:1024F00064657273702E004F75743220566D696E6C
:102500002E5761726E004F75743220756E6465725D
:10251000766F6C74005569746732206F6E646572F3
:1025200073702E004D696E2E20476173202020208D
:102530002020006D696E2E207468726F74746C6553
:1025400020006D696E696D61616C20676173202088
:10255000004D61782E20476173202020202020002C
:102560006D61782E207468726F74746C6520006DD4
:102570006178696D61616C206761732020004B6F29
:102580006D706173737769726B756E6700636F6DE1
:102590007061737320656666656374004B6F6D7060
:1025A00061732065666665637420004361726566C9
:1025B0007265652053742E20200043617265667237
:1025C0006565204374726C200043617265667265B4
:1025D00065204374726C2000546561636861626CAD
:1025E00065204361726500546561636861626C6572
:1025F000204361726500546561636861626C6520A7
:102600004361726500556E7465727370616E6E75AC
:102610006E672000756E646572766F6C74616765B5
:102620002020004F6E6465727370616E6E696E6714
:102630002000566F6C74205265666572656E7A2054
:1026400000566F6C74205265666572656E7A200064
:102650005265662E207370616E6E696E6720004E43
:102660006F7420476173205A656974202000456D9E
:102670006572672E5468722E54696D65004E6F6FD7
:1026800064206761732074696A6420004E6F74204F
:102690004761732020202020202000456D6572674F
:1026A0002E5468726F74746C65004E6F6F6420678F
:1026B0006173202020202020004661696C732E2049
:1026C00043482054696D65004661696C732E204350
:1026D000482054696D65004661696C732E2043483B
:1026E0002054696A64004661696C732E20436861F6
:1026F0006E6E656C004661696C732E204368616E76
:102700006E656C004661696C732E204368616E6E65
:10271000656C006B2E53756D6D6572206F2053656F
:102720006E006E20626565702061637420545820CD
:10273000006E20626565702061637420545820002B
:10274000566172696F206661696C20416C74005635
:102750006172696F206661696C20416C740056611A
:1027600072696F206661696C20416C7400436F6D03
:1027700070617373204572726F722000436F6D70C9
:10278000617373204572726F7220004B6F6D7061C0
:1027900073204572726F722020006B2E5374617229
:1027A00074206F2E53442D4B006E2073742E2077AF
:1027B00074686F20534420006E2073742E20777449
:1027C000686F20534420006B2E5374617274206F25
:1027D0002E47505320006E2073742E207774686F3C
:1027E00020475053006E2073742E207774686F203A
:1027F000475053004779726F20502020202020201E
:102800002020004779726F20502020202020202097
:1028100020004779726F2050202020202020202087
:10282000004779726F20492020202020202020009E
:102830004779726F20492020202020202020004747
:1028400079726F2049202020202020202000477905
:10285000726F204420202020202020200047797201
:102860006F20442020202020202020004779726FF4
:10287000204420202020202020200047696572204D
:10288000502020202020202020004C6163657420EF
:1028900050202020202020200047696572205020F1
:1028A0002020202020202000476965722049202018
:1028B000202020202020004C6163657420492020C6
:1028C00020202020200047696572204920202020F8
:1028D000202020200044796E616D69736368652053
:1028E00053742E0064796E616D6963207374616244
:1028F000692E0044796E616D69732E207374616274
:102900002E0044726568726174656E6265672E2080
:1029100000526F7452617465206C696D69742E0089
:10292000546F6572656E74616C206C696D2E004128
:1029300043432F4779726F2046616B2E200041433D
:10294000432F4779726F20466163742000414343EF
:102950002F4779726F204661637420004143432FF3
:102960004779726F204B6F6D702E00436F6D702032
:102970004143432F4779726F2000436F6D702041B0
:1029800043432F4779726F200048617570747265F8
:10299000676C6572204920004D61696E20492020D6
:1029A00020202020202000486F6F666472656765D4
:1029B0006C2E20492000447269666B6F6D70656EE5
:1029C0007361742E00647269667420436F6D706564
:1029D0006E732E00447269667420636F6D70656E4D
:1029E000732E004779726F20737461622E2020204D
:1029F00020004779726F2073746162696C69747921
:102A0000004779726F2073746162696C69742E007B
:102A10004D6F746F7220736D6F6F74682020004D5E
:102A20006F746F7220736D6F6F74682020004D6F2C
:102A3000746F7220736D6F6F746820200050617224
:102A4000616D6574657220312020200050617261D3
:102A50006D65746572203120202000506172616DB7
:102A600065746572203120202000506172616D65AF
:102A7000746572203220202000506172616D65748F
:102A80006572203220202000506172616D6574658E
:102A900072203220202000506172616D6574657271
:102AA000203320202000506172616D6574657220B2
:102AB0003320202000506172616D6574657220338F
:102AC00020202000506172616D6574657220342091
:102AD000202000506172616D657465722034202081
:102AE0002000506172616D65746572203420202071
:102AF00000506172616D6574657220352020200080
:102B0000506172616D65746572203520202000501F
:102B10006172616D657465722035202020005061FE
:102B200072616D65746572203620202000506172DC
:102B3000616D6574657220362020200050617261DD
:102B40006D65746572203620202000506172616DC1
:102B500065746572203720202000506172616D65B8
:102B6000746572203720202000506172616D657499
:102B70006572203720202000506172616D65746598
:102B800072203820202000506172616D657465727A
:102B9000203820202000506172616D6574657220BC
:102BA00038202020004163687328652E296B6F70E0
:102BB000706C2E0028446529436F75706C20417835
:102BC0006573004173206B6F7070656C696E672070
:102BD00020004769657220706F732E204B6F7070F4
:102BE00000526574726F6163206C616365742000CC
:102BF0004769657220706F732E206B6F702E004EC8
:102C000069636B2F526F6C6C204B6F707000526554
:102C100074726F20726F756C2F74616E004E6963F1
:102C20006B2F526F6C6C206B6F702E004769657252
:102C3000204B6F7272656B74757200436F727265B0
:102C40006374206C6163657420004769657220635A
:102C50006F72726563746965004F7269656E74693D
:102C60006572756E672020004F7269656E746965C4
:102C700072756E672020004F7269656E74617469A9
:102C80006F6E2020200048F668656E726567656C7F
:102C9000756E672000416C746974756465204374B7
:102CA000726C2000486F6F67746520436F6E74729A
:102CB0002E2000536F6C6C68F66865202020202061
:102CC0002000536574706F696E74202020202020CE
:102CD00000476577656E73742E686F6F6774650063
:102CE000537469636B204E657574722E20500073A7
:102CF0007469636B206E657574722E205000537476
:102D000069636B206E657574722E205000475053B6
:102D1000202020202020202020202000656E6162BD
:102D20006C65204750532020202000456E61626C66
:102D300065204750532020202000475053204D6FDE
:102D40006475732053742E2000475053206D6F64B8
:102D50006520636F6E747200475053206D6F646519
:102D600020636F6E74720044796E616D69632050E8
:102D700048202020200044796E616D69632050480E
:102D8000202020200044796E616D69632050482026
:102D90002020200043482048F6686520202020207D
:102DA00020200043482048696768202020202020F8
:102DB0002000434820686F6F677465202020202022
:102DC0000043617265667265652053742E20200091
:102DD0004361726566726565204374726C200043BE
:102DE00061726566726565204374726C200054657B
:102DF00061636861626C652043617265005465615E
:102E0000636861626C65204361726500546561634B
:102E10006861626C652043617265004D6F746F720A
:102E200020536963682E536368004D6F742E53619D
:102E3000666574792053772E004D6F742E7361662A
:102E40002E736368616B2E004F7269656E746965DD
:102E500072756E672020004F7269656E74617469C7
:102E60006F6E202020004F7269656E746174696511
:102E700020202020000000010C03010101000001BE
:102E80000C040404040000010C010303030000010E
:102E90000C020202020003011905050505000301E9
:102EA00019060606060003011907070707000301B4
:102EB0001908080808000301190909090900030194
:102EC000190A0A0A0A000301190B0B0B0B00030174
:102ED000190C0C0C0C0000000C6300000000020038
:102EE000086E000000000200046D000000000600F3
:102EF0000627010101010200010D0000000102008E
:102F0000200D010101010200080D01010101020073
:102F1000100D000000010200046D0000000102001D
:102F2000400D010101010200800D000000010200BE
:102F3000040D00000002000014170A080602000039
:102F4000141810100A020100FF19060604020100FD
:102F5000FF60000000030200016B0000000302009C
:102F6000026B000000030200046B0000000302007B
:102F7000086B000000030100FF3B32323203000007
:102F8000F73C5A5A5A030000F73D32323203000030
:102F9000F7414E4E4E030000F7424E4E4E040200E3
:102FA000010D000000040200016D00000004020099
:102FB000020D010101040200026D01010104010082
:102FC000FF10FFFFFF040000F70E1E1E1E0401008D
:102FD000FF110F0F0F040100FF0F1E1E1E04010042
:102FE000FF13000000040100FF679696960400009E
:102FF000F7120F0F0F040000F7140808080401006F
:10300000FF15404040040000A0160000000501002C
:10301000FF2D808080050000F72E3232320502003D
:10302000016C000000050000F72F0F0F0F050000D6
:10303000F730E6E6E605000019690000000501002A
:10304000FF31808080050000F7325555550502009C
:10305000026C000000050000F733464646050000FC
:10306000F734DCDCDC050000196A00000005000212
:103070000835040404050000F7363C3C3C05050017
:10308000F737000000050100FF387D7D7D05010058
:10309000FF397D7D7D050100FF3A7D7D7D060200C3
:1030A000200D010101060100FF50FEFEFE06010099
:1030B000FF51646464060000F75A0808080600001F
:1030C000F759060606060100FF525A5A5A06010031
:1030D000FF535A5A5A060100FF545A5A5A06010021
:1030E000FF554B4B4B060100FF5655555506010049
:1030F000FF574B4B4B060100FF5800000006010034
:10310000FF5B5A5A5A060100FF5C2A2A2A06010070
:10311000FF5DF5F5F5060100FF5E8C8C8C06000066
:10312000F75F050505060200206D0000000602009D
:10313000026E000000060000F765000000070400B2
:10314000FF4A5F5F5F070100FF4B14141407020082
:10315000206B000000070200106B01010107040052
:10316000FF4CF3F3F3070100FF4D141414070200A2
:10317000406B000000070200806B010101070400A2
:10318000FF4EAAAAAA070400FF4FAAAAAA08000095
:10319000F71A080808080000F71BE6E6E608010031
:1031A000FF1D404040080100FF62000000080200CF
:1031B000406D000000080000F724212121080200D2
:1031C000086D000000080000F7265A5A5A0800004F
:1031D000F7252D2D2D080000F766000000080000DF
:1031E0000C68000000080200106D000000080200DA
:1031F000046E000000080200806D0000000802005C
:10320000016E000000080200106E000000090100BD
:10321000FF1E5A6464090100FF1F787878090100D5
:10322000FF200A0A0A090100FF215A64640901000B
:10323000FF22787878090100FF45464646090200DA
:10324000800D000000090000F71C1B1B1B0900007B
:10325000F743202020090100FF281010100900006A
:10326000F7440000000900001023060606090000CC
:10327000F7640000000A0100FF290000000A0100B5
:10328000FF2A0000000A0100FF2B0000000A0100D5
:10329000FF2C0000000A0100FF460000000A0100A8
:1032A000FF470000000A0100FF480000000A01007B
:1032B000FF490000000B0200400D0000000B010060
:1032C000FF3E5A5A5A0B0100FF3F3737370B0100B8
:1032D000FF404646460C050017610000000D020045
:1032E000010D0000000D0100FF10FFFFFF0D0000A9
:1032F000A0160000000D0200200D0101010D0100CB
:10330000FF50FEFEFE0D0200206D0000000D0000CB
:10331000F7650000000D0100FF620000000D0200D3
:10332000406D0000000D00000C630000000D050062
:10333000176100000050504D202020202020202028
:103340002020202020005370656B7472756D202042
:10335000202020202020005370656B7472756D2032
:1033600048695265732020005370656B7472756DE7
:10337000204C6F5265732020004A6574692020201C
:10338000202020202020202020004143542044538E
:103390004C20202020202020202000484F54542062
:1033A0002020202020202020202020004675747519
:1033B0006261205342555320202020200055736520
:1033C00072202020202020202020202020001300F8
:1033D000120013005553520053425500486F5400D9
:1033E000414354004A65740053704C0053704800C8
:1033F0005370650050504D00575045005300202039
:103400004E0020204A00205000200025001200130A
:10341000001200200012003000310020192020206E
:1034200020301149202020456E64652020204F4B1C
:10343000005750450053005374642E0028312D531B
:1034400031322F57292028643A20202029001D00DE
:10345000200020001D002A002A00506F00506F201D
:1034600029005374642E0028302D3234372D503803
:103470002928643A506F2029005374642E002820B4
:1034800020202D202020292028643A2020202900D7
:103490004B6F706965727420756E6420416B74693E
:1034A0007669657274005769726B6C696368204B4A
:1034B0006F70696572656E3F004D6F746F72205456
:1034C00065737465722020202020004D6F746F7228
:1034D000205465737465722020202020004D6F7485
:1034E0006F72205465737465722020202020005371
:1034F0006572766F205465737465722020202020D9
:1035000000536572766F20546573746572202020B5
:10351000202000536572766F2054657374657220A5
:103520002020202000504320425420203E204B6F7A
:1035300070746572202000504320425420203E20A9
:103540004B6F70746572202000504320425420203D
:103550003E204B6F707465722020005043205553FD
:1035600042203E204B6F7074657220200050432033
:10357000555342203E204B6F7074657220200050DE
:103580004320555342203E204B6F707465722020BB
:1035900000504B542053657475702020202020204B
:1035A000201D00504B54205365747570202020203E
:1035B0002020201D00504B5420536574757020202E
:1035C00020202020201D00504B5420566572736926
:1035D0006F6E20202020202000504B542056657212
:1035E00073696F6E20202020202000504B542056FD
:1035F000657273696F6E20202020202000566F6C4A
:103600007400456E6465001D00200020001D005000
:103610004320555342203E204B6F7074657200501A
:103620004320425420203E204B6F7074657200137B
:1036300000120020504B542D546F6F6C73202020CB
:10364000202020202020202000120057692E323315
:1036500032204E414B00576932333220496E697433
:103660004572726F72202000576932333220496EE2
:103670006974206F6B2E2E2E2E0057693233322044
:10368000496E69744572726F722020002E002E0000
:103690002E002E002E002E002E002E002E002E00BA
:1036A0002E002E002E002E002E002E002E002E00AA
:1036B0002E00496E69742057693233322077616970
:1036C000742E2E2E2E0056657273696F6E3A004569
:1036D00072726F72207365742052414D2020202039
:1036E00020004572726F7220736574204E562D5201
:1036F000414D0057692E3233322077726F6E67204A
:1037000042617564726174650057692E32333220EC
:10371000666F756E64200057692E323332205379FC
:103720007461786572726F72202020006E6F20576E
:10373000692E32333220666F756E64007365617274
:1037400063682057692E323332204D6F64756C00E8
:1037500031313532303000203537363030002033CB
:1037600038343030002031393230300020203936C2
:1037700030300020203234303000207769746820E7
:103780002020202020202042617564005556F73209
:10379000EE1AAB0DDC066F03B801DC006E003700DB
:1037A0001B000E0007000300020001005365727643
:1037B0006F736368726974746520202020007365DC
:1037C00072766F20737465707320202020000000D3
:1037D000736572766F2073746570732020202020CB
:1037E0000000536572766F20312020202020202099
:1037F00020201D00736572766F203120202020204C
:10380000202020201D00736572766F20312020203B
:103810002020202020201D00536572766F2032204A
:1038200020202020202020201D00736572766F202C
:10383000322020202020202020201D007365727659
:103840006F20322020202020202020201D005365C2
:1038500072766F74657374202020202020201D0054
:10386000736572766F746573742020202020202089
:103870001D00736572766F7465737420202020209C
:1038800020201D00546573742050756C736CE46EB9
:10389000676520202000746573742070756C732038
:1038A0007769647468000000746573742070756CC7
:1038B000732077696474682000005465737420660F
:1038C0006F72746C617566656E641D0074657374E7
:1038D00020636F6E742E2020202020201D00746530
:1038E000737420636F6E742E2020202020201D0012
:1038F000536572766F202020202020202020202059
:103900002000736572766F20202020202020202048
:1039100020000000736572766F2020202020202078
:10392000202020200000506572696F6465202020EF
:1039300020202020202020006672616D652020203C
:10394000202020202020200000006672616D65206C
:10395000202020202020202020200000537461728D
:10396000742054657374202020202020200073745C
:103970006172742074657374202020202020200040
:103980007374617274207465737420202020202069
:10399000200045696E7A656C73636872697474207F
:1039A0002020200073696E676C6520737465702039
:1039B00020202020200073696E676C652073746579
:1039C0007020202020202000416E7A61686C2054F5
:1039D000657374202020202020006E756D62657252
:1039E000206F662074657374202020006E756D62F0
:1039F0006572206F6620746573742020200050610A
:103A000075736520456E64706F736974696F6E00BD
:103A1000706175736520656E6420706F732020205F
:103A20002000706173756520656E6420706F73206F
:103A30002020200050617573652070726F20496EE0
:103A4000632E2020200070617573652070726F6393
:103A500020696E632E20200070617573652070727E
:103A60006F6320696E632E20200052657665727345
:103A700065202020202020202020200072657665EF
:103A800072736520202020202020202020007265D5
:103A900076657273652020202020202020202000C1
:103AA0004C696E6B732020202020202020202020B5
:103AB00020006C65667420202020202020202020FB
:103AC000202020006C6566742020202020202020EB
:103AD000202020202000526563687473202020205D
:103AE0002020202020202000726967687420202078
:103AF0002020202020202020200072696774682068
:103B00002020202020202020202020004D697474B7
:103B100065202020202020202020202020006D69EA
:103B200064646C652020202020202020202020009C
:103B30006D6964646C6520202020202020202020D6
:103B4000200013001200736572766F5F6D656E75ED
:103B5000001300120061646A75737420207365722B
:103B6000766F200013001200536572766F746573D0
:103B70007420636F6E742E001300120074657374EA
:103B80005F736572766F5F6D656E7520200053659B
:103B900072766F203200536572766F203100536564
:103BA00072766F3A00010000000A00000064000015
:103BB00000E803000010270000A086010040420F2B
:103BC000008096980000E1F50500CA9A3B456E64B6
:103BD000650020547261636B696E67204D696B727A
:103BE0006F6B6F7074657200547261636B696E679E
:103BF00020426C7565746F6F7468202020006C6FB4
:103C000073742057692E3233322064617461004727
:103C10005053206F6B2C207374617274206F6B2073
:103C200020002020202020202020202020202020B4
:103C30002020202000576861697420666F72204739
:103C40005053204669782000576861697420666F78
:103C5000722047505320466978200053204C6174ED
:103C6000697475646520204C6F6E6769747564654E
:103C7000004665686C6572206265696D20547265E6
:103C80006E6E656E00737769746368206F6E204294
:103C900054204D6F7573652121004572726F72203B
:103CA000617420636F6E6E656374696E6700475060
:103CB00053207472656E6E656E006C6F7374204273
:103CC0005420646174610048444F503A004669785A
:103CD0003A005361743A004D00480053204C61741F
:103CE000697475646520204C6F6E676974756465CE
:103CF000004641494C00204F4B2000203F3F200010
:103D000054696C743A0050616E203A006D00446949
:103D100073743A001E00426561723A0020204C49DB
:103D2000504F202021215761726E756E672121202E
:103D30002000194F18002073657269656C6C65204E
:103D4000506F74697320312D352000DC6265727309
:103D50006963687420202020202020200073756D66
:103D60006D61727920202020202020200000007327
:103D7000756D6D6172792020202020202020200088
:103D800000537469636B20312020202020202020E4
:103D9000201D00737469636B2031202020202020B7
:103DA0002020201D00737469636B203120202020A7
:103DB00020202020201D00537469636B20322020B6
:103DC000202020202020201D00737469636B203286
:103DD0002020202020202020201D00737469636B88
:103DE00020322020202020202020201D0053746914
:103DF000636B20332020202020202020201D0073F2
:103E00007469636B20332020202020202020201D77
:103E100000737469636B2033202020202020202031
:103E2000201D00537469636B203420202020202043
:103E30002020201D00737469636B20342020202013
:103E400020202020201D00737469636B2034202003
:103E5000202020202020201D00537469636B203512
:103E60002020202020202020201D00737469636BF7
:103E700020352020202020202020201D0073746960
:103E8000636B20352020202020202020201D005082
:103E90004B54204C69706F6D657373756E6720208D
:103EA00000504B54204C69706F206D6561737572C2
:103EB000652E00504B54204C69706F206D65617306
:103EC0007572652E004D696E696D616C2057657263
:103ED000742020000000006D696E696D616C2076B1
:103EE000616C756520000000006D696E696D616C24
:103EF0002076616C756520000000004D6178696D69
:103F0000616C20576572742020000000006D61789C
:103F1000696D616C2076616C756520000000006D34
:103F20006178696D616C2076616C756520000000B8
:103F3000005479706520202020202020202020009F
:103F4000000000747970652020202020202020208F
:103F5000200000000074797065202020202020209F
:103F6000202020000000005269636874756E67208D
:103F700020202020200000000064697265637469BD
:103F80006F6E2020202020000000006469726563AD
:103F900074696F6E2020202020000000004E65759F
:103FA0007472616C69736965726564000000006E0B
:103FB00065757472616C697A696E67202000000013
:103FC000006E65757472616C697A696E6720200095
:103FD000000000130012004A6F79737469636B204C
:103FE000202020202020202020200013001200204C
:103FF00020204A6F79737469636B20536574757000
:1040000020202020004F4B00504B54204C69706FF3
:104010006D657373756E672020200059004E005245
:104020006576004E6F726D005461737400506F744A
:10403000690053204D696E204D61782054797020BD
:104040002044697220204E002020204A6F7973742A
:1040500069636B20536574757020202020005665BD
:104060007262696E64756E67207A756D204D4B00C3
:10407000636F6E6E656374696F6E20746F204D4B55
:10408000200041616E736C756974696E67206F7092
:10409000204D4B00504B5420616C6C67656D656919
:1040A0006E2020201D00504B5420676C6F62616CA5
:1040B0002020202020201D00504B5420676C6F6270
:1040C000616C2020202020201D0057692E323332C1
:1040D000202020202020202020201D0057692E3263
:1040E0003332202020202020202020201D0057694E
:1040F0002E323332202020202020202020201D009E
:1041000042544D2D323232202020202020202020E9
:104110001D0042544D2D32323220202020202020FC
:1041200020201D0042544D2D3232322020202020EC
:10413000202020201D00536572766F204D656EFC97
:104140002020202020201D00736572766F206D6571
:104150006E752020202020201D00736572766F2050
:104160006D656E752020202020201D004F534420B7
:10417000416E7A6569676520202020201D004F531D
:10418000442073637265656E2020202020201D006E
:104190004F53442073637265656E202020202020D9
:1041A0001D004750532020202020202020202020A8
:1041B00020201D0047505320202020202020202098
:1041C000202020201D004750532020202020202088
:1041D0002020202020201D00466F6C6C6F77204D22
:1041E00065202020202020201D00466F6C6C6F77FA
:1041F000204D65202020202020201D00466F6C6C63
:104200006F77204D65202020202020201D004A6F40
:1042100079737469636B20202020202020201D00EA
:104220006A6F79737469636B20202020202020201E
:104230001D006A6F79737469636B20202020202031
:1042400020201D00504B542D416B6B7520202020E9
:10425000202020201D00504B542D416363752020E9
:104260002020202020201D00504B542D41636375D9
:1042700020202020202020201D00504B542055704D
:10428000646174652020202020202000504B5420A1
:104290005570646174652020202020202000504B40
:1042A0005420557064617465202020202020200057
:1042B000446562756720504B542020202020202028
:1042C0002000446562756720504B54202020202038
:1042D00020202000446562756720504B5420202028
:1042E000202020202000454550726F6D20526573BC
:1042F0006574202020202000454550726F6D2052AB
:1043000065736574202020202000454550726F6D34
:10431000205265736574202020202000496E666F4E
:1043200073206265696D2053746172742000696E38
:10433000666F206174207374617274757020200040
:10434000696E666F2062696A206F7073746172743F
:1043500020004F534420456D7066616E6773617530
:1043600073662E004F53442072656365697665203D
:104370004572726F72004F534420726563656976AF
:1043800065204572726F72005370726163686520B8
:10439000202020202020202020006C616E67756185
:1043A0006765202020202020202020007461616C7F
:1043B00020202020202020202020202020004C69A8
:1043C00063687420617573206E6163682E2E2E0001
:1043D0006C69676874206F66662061667465722018
:1043E00020006C6963687420756974206E612020F8
:1043F0002020200048656C6C69676B65697420201B
:104400002020202020006272696768746E657373D3
:10441000202020202020200068656C64657268657B
:10442000696420202020202020004B6F6E74726170
:10443000737420202020202020202000636F6E74C1
:104440007261737420202020202020202000636FC0
:104450006E747261737420202020202020202000A0
:104460004E6F726D616C2F496E76657273202020DD
:1044700020006E6F726D616C2F696E766572746567
:10448000642020004E6F726D616C2F696E766572CC
:104490007465642020004F7269656E746965727579
:1044A0006E672020202020006F7269656E74617431
:1044B000696F6E202020202020006F7269656E7465
:1044C00061746965202020202020200056617269D7
:1044D0006F20546F6E204572772E20202000566189
:1044E00072696F20536F756E64204578742E2000BA
:1044F000566172696F20536F756E64204578742E13
:10450000200048617264776172652042656570655C
:10451000722020004861726477617265204265658F
:104520007065722020004861726477617265204274
:1045300065657065722020004C6175747374E47257
:104540006B652020546F6E202000566F6C756D6572
:10455000202020202020202020202000566F6C7555
:104560006D652020202020202020202020004D6F5D
:1045700064756C2065696E6765626175743F2000C3
:104580006D6F64756C65206275696C7420696E3F2F
:1045900020004D6F64756C65206765696E7374618A
:1045A0006C2E3F0054582F5258204B616E616C2086
:1045B00020202020200054582F5258204368616E3C
:1045C0006E656C202020200054582F5258204368DC
:1045D000616E6E656C20202020004E6574572E2081
:1045E0004772757070652020202020004E6574573A
:1045F0002E2047726F7570202020202020004E65ED
:1046000074572E2047726F757020202020202000C4
:104610004E6574572E204D6F646520202020202089
:1046200020004E6574572E204D6F64652020202099
:10463000202020004E6574572E204D6F6465202089
:1046400020202020200054582054696D656F757417
:10465000202020202020200054582054696D656FB0
:104660007574202020202020200054582054696D8B
:10467000656F757420202020202020005458204D84
:104680005455202020202020202020202000545875
:10469000204D5455202020202020202020202000A4
:1046A0005458204D54552020202020202020202008
:1046B000200042617564726174652057693233323B
:1046C0002F425400426175647261746520576932EB
:1046D00033322F4254004261756472617465205711
:1046E000693233322F425400496E697469616C69D2
:1046F00073696572656E20202000696E6974696156
:104700006C697A652020202020202000496E697481
:1047100069616C697A6520202020202020004B6F81
:104720006E6669672E206D6974205043202020003A
:10473000636F6E6669672E20776974682020504326
:104740002000436F6E6669672E206D6574205043AC
:10475000202020004D6F64756C2065696E6765626E
:104760006175743F20006D6F64756C6520627569BA
:104770006C7420696E3F20006D6F64756C652067F6
:1047800065696E7374616C6C3F004E616D652020CD
:104790002020202020202020202020006E616D6518
:1047A00020202020202020202020202020004E61BA
:1047B000616D20202020202020202020202020008B
:1047C00050696E2020202020202020202020202022
:1047D000200070696E202020202020202020202012
:1047E0002020200050696E20202020202020202022
:1047F000202020202000496E697469616C6973690A
:104800006572656E20202000696E697469616C694B
:104810007A652020202020202000496E697469617B
:104820006C697A652020202020202000426C75656C
:10483000746F6F7468204D41432D41647200426C67
:104840007565746F6F7468204D41432D416472002B
:10485000426C7565746F6F7468204D41432D4164DF
:10486000720052452D494420202020202020202065
:104870002020200052452D494420202020202020A7
:1048800020202020200052452D4944202020202097
:1048900020202020202020004B6F6E6669672E208C
:1048A0006D697420504320202000636F6E66696735
:1048B0002E2077697468202050432000436F6E6675
:1048C00069672E206D657420504320202000504BD6
:1048D000542D416B6B7574797020202020202000AE
:1048E000504B542D41636375747970202020202033
:1048F0002000504B542D626174746572696A207493
:1049000079706500504B5420416B6B75204D657379
:1049100073756E672000504B5420416363754D657D
:104920006173757265202000504B5420626174746D
:104930002E206D6574696E67200077E4686C6520D1
:10494000475053204D6175732020200073656C65BE
:10495000637420475053206D6F7573652000736535
:104960006C65637420475053206D6F75736520002C
:10497000537563686520475053204D61757320203F
:10498000200073656172636820475053206D6F7516
:104990007365200073656172636820475053206D12
:1049A0006F7573652000475053204D617573205417
:1049B0007970202020202000475053206D6F7573A0
:1049C00065207479702020202000475053206D6F9F
:1049D0007573652074797020202020004750532083
:1049E0004D61757320616B7469763F2020004750DC
:1049F00053206D6F7573652061637469763F200085
:104A0000475053206D6F7573652061637469763FFD
:104A100020005A65696765204750532044657669D0
:104A20006365200073686F77204750532064657674
:104A300069636520200073686F77204750532064B6
:104A40006576696365202000475053204461746592
:104A50006E20202020202020200047505320646119
:104A60007461202020202020202020004750532047
:104A70006461746120202020202020202000466FC7
:104A80006C6C6F774D6520526566726573680000C7
:104A9000466F6C6C6F774D65205265667265736802
:104AA0000000466F6C6C6F774D65205265667265CD
:104AB00073680000466F6C6C6F774D6520537065AE
:104AC000656420200000466F6C6C6F774D65205345
:104AD0007065656420200000466F6C6C6F774D65D3
:104AE00020537065656420200000546F6C6572610E
:104AF0006E7A20526164697573200000546F6C6592
:104B000072616E6365205261646975730000546F51
:104B10006C6572616E636520526164697573000033
:104B20000000000000000000000000000000000085
:104B30000000000000000000000000000000000075
:104B40000000000000000000000000000000000065
:104B50000000000000000000000000000000000055
:104B60000000000000000000000000000000000045
:104B70000000000000000000000000000000000035
:104B80000000000000000000000000000000000025
:104B90000000000000000000000000000000000015
:104BA0000000000000000000000000000000000005
:104BB00000000000000000000000000000000000F5
:104BC00000004F5554312F3220466F726D617420B2
:104BD000202020004F5554312F3220666F726D61B6
:104BE0007420202020004F5554312F3220666F72E0
:104BF0006D617420202020004F5554312F322050F9
:104C00006F6C61726974E47420004F5554312F3217
:104C100020706F6C61726974792020004F55543197
:104C20002F3220706F6C61726974792020004E61A0
:104C3000766920446174656E20616E20535632009F
:104C40004E617669206461746120746F205356321E
:104C500020004E617669206461746120746F205376
:104C6000563220004D61782E2053696E6B7261744C
:104C700065206D2F73006D61782066616C6C7370B8
:104C8000656564206D2F73006D61782066616C6CC2
:104C90007370656564206D2F7300566172696F6D66
:104CA00065746572204265657020200056617269E6
:104CB0006F6D6574657220626565702020005661B5
:104CC00072696F6D65746572206265657020200081
:104CD000486F6D6520617573204D4B205369636883
:104CE0007400686F6D652066726F6D204D4B207685
:104CF00069657700686F6D652066726F6D204D4B3A
:104D00002076696577004D4B204C6F7742617420A7
:104D10005761726E756E67004D4B204C6F77426124
:104D200074207761726E696E67004D4B204C6F4244
:104D3000617420616C61726D202020004D4B206DEC
:104D40004168202020205761726E756E67004D4BC0
:104D5000206D4168207761726E696E6720202000A7
:104D60004D4B206D416820616C61726D20202020C8
:104D700020004D4B20566F6C742020202042616C27
:104D80006B656E004D4B20766F6C742062617267AC
:104D90007261706820004D4B20766F6C74206261E8
:104DA0007267726170682000130012001300120015
:104DB00013001200566F6C74004C69496F004C6907
:104DC000506F004C69506F004C69496F004572721A
:104DD0006F7220646973636F6E6E656374696E676A
:104DE00021004572726F7220636F6E6E6563746925
:104DF0006E67210062697474652077617274656EF4
:104E00002E2E2E00475053207472656E6E656E0014
:104E10006C6F73742042542064617461006D002EC5
:104E2000002E0020202D2D2D00416C743A200020F2
:104E30004C617469747564652020204C6F6E6769DD
:104E4000747564650048444F503A20004669783ACA
:104E50002000584572723A20005361743A20006372
:104E60006F6E6E656374204572726F7200636F6E51
:104E70006E6563746564202020202000636F6E6E71
:104E8000656374207374617475730074727920742F
:104E90006F20636F6E6E656374004D41433A00444A
:104EA00065766963653A00737563686520425420CE
:104EB0004465766963650077E4686C652042542038
:104EC00044657669636500130012002052452D4940
:104ED00044204E6F74697A2020202020202020203A
:104EE000003A004D41433A002042544D2D323232B7
:104EF000204D41432D416472657373652000425417
:104F000020496E6974204572726F720042542049C4
:104F10006E6974206F6B0020426C7565746F6F74DE
:104F2000682050696E202020202020200020426C24
:104F30007565746F6F7468204E616D652020202048
:104F4000202000130012001300120020425420738E
:104F5000656C656374204465766963652020202054
:104F6000002017202020202016202020202019207B
:104F70002020204F4B0020202020202020202020F7
:104F800020202043002000130012002057692E32F9
:104F9000333220536574757020202020202020207B
:104FA00000130012001300120020504B542D5365C3
:104FB0007475702020202020202020202020002513
:104FC0000057693233320057693233320034383097
:104FD0003020200031313532303000353736303036
:104FE0002000333834303020003139323030200066
:104FF00039363030202000323430302020004D69E6
:105000006B726F6B6F70740042542D4D6F757365CA
:1050100031002020206E69636874206DF6676C692A
:105020006368202020200020204D69742048617290
:10503000647761726520312E78202020000E0F0EDB
:105040004E0E0F0E4F0E0F0E530E0F0E570E0F0E6D
:105050004E0E0F0E4F0E0F0E530E0F0E570E0F0E5D
:105060004E0E0F0E4F0E0F0E530E0F0E574E4500E5
:105070004520005345005320005357005720004E51
:1050800057004E20006D5070507350765079507C10
:10509000507F50825000496E666F003A006D416843
:1050A0000020202030006B6D6800537461746973B8
:1050B00074696373003344204C616765004F534447
:1050C00032004F534431004F534430006D00486F5D
:1050D0006D653A00416C743A004E6176696761749F
:1050E000696F6E006D00206B6D68004100202049E3
:1050F0003A004469723A00416C743A00206D4100F4
:1051000047656E6572616C005750006D73006D20CD
:105110002D005A69656C00205361740050430020D3
:1051200020001F006D202D00486F6D65004B6D68DD
:10513000006D0041006D4168005600560056005356
:105140000048F66865006D00532100475000465343
:1051500000454C004659004D520053540043410055
:105160004241006F32006F31004348004346005017
:1051700048004148002E002E002E002E002E002E4A
:10518000005374617465203A0056657273696F6EDE
:105190003A0054656D70657261747572653A0043CA
:1051A000757272656E74202020203A005365745029
:1051B0006F696E742020203A001D00200020001D21
:1051C00000416C6C00416C6C001D001A201B0056E5
:1051D000616C75653A20202030004D6F746F723A13
:1051E000202020310020424C2D4374726C205465E5
:1051F0007374202020202020202000456E6465202C
:10520000436865636B0054656D7020203A004D6102
:105210007850574D203A00437572726E743A0052BE
:105220006561644D6F643A005374617465203A009F
:10523000536574506F694C3A00536574506F693A06
:105240000056657273696F6E3A00466F756E642022
:10525000424C2D4374726C3A00537563686520426A
:105260004C2D4374726C0000000000000000007EB2
:105270008195B1B195817E7EFFEBCFCFEBFF7E0EA6
:105280001F3F7E3F1F0E00081C3E7F3E1C0800385B
:105290003A9FFF9F3A38001038BCFFBC381000001E
:1052A00000000000000000000000000000000000FE
:1052B000000000000000000000000000000000707E
:1052C000F88888FD7F070F004E5FF1F15F4E000008
:1052D00000000000000000C0FF7F0505657F3F99CA
:1052E0005A3CE7E73C5A997F3E3E1C1C08080008E0
:1052F000081C1C3E3E7F00002466FFFF6624000061
:105300005F5F00005F5F00060F097F7F017F7FDA2C
:10531000BFA5A5FD59030200707070707070008009
:1053200094B6FFFFB694800004067F7F0604000059
:1053300010307F7F3010000808082A3E1C08000843
:105340001C3E2A080808003C3C20202020200008A1
:105350001C3E08083E1C0830383C3E3E3C383006B7
:105360000E1E3E3E1E0E0600000000000000000063
:10537000065F5F0600000000070700070700001433
:105380007F7F147F7F1400242E6B6B3A120000463F
:105390006630180C666200307A4F5D377A48000438
:1053A00007030000000000001C3E634100000000F5
:1053B00041633E1C000000082A3E1C1C3E2A0808CF
:1053C000083E3E0808000000A0E060000000000861
:1053D0000808080808000000006060000000006085
:1053E00030180C060301003E7F594D7F3E000042FD
:1053F000427F7F40400000627359496F660000227F
:105400006349497F360000181C16137F7F10002760
:105410006745457D3900003C7E4B497930000003EB
:105420006371190F070000367F49497F3600000677
:105430004F49693F1E000000006C6C000000000036
:10544000A0EC6C00000000081C3663410000001452
:1054500014141414140000004163361C08000002E8
:105460000351590F0600003E7F415D5D1F1E007C09
:105470007E13137E7C0000417F7F49497F36001CEC
:105480003E634141632200417F7F41637F1C0041B5
:105490007F7F495D416300417F7F491D0103001CFF
:1054A0003E6341517372007F7F08087F7F000000D8
:1054B000417F7F41000000307040417F3F0100414B
:1054C0007F7F081C776300417F7F41406070007FD1
:1054D0007F060C067F7F007F7F060C187F7F001CF5
:1054E0003E6341633E1C00417F7F49090F06001E59
:1054F0003F21717F5E0000417F7F19396F46002692
:10550000674D597B32000003417F7F410300007FDC
:105510007F40407F7F00001F3F60603F1F00007F93
:105520007F3018307F7F0063771C081C776300078B
:105530004F78784F0700006773594D47637100003B
:105540007F7F41410000000103060C18306000001D
:1055500041417F7F000000080C0603060C08008014
:10556000808080808080800000030704000000208D
:105570007454543C784000413F7F44447C380038A8
:105580007C44446C280000307848493F7F40003814
:105590007C54545C180000487E7F49030200009848
:1055A000BCA4A4F87C0400417F7F08047C78000040
:1055B000447D7D4000000040C484FD7D000000412A
:1055C0007F7F10386C440000417F7F400000007CEA
:1055D0007C0C180C7C78007C7C04047C78000038FF
:1055E0007C44447C38000084FCF8A4243C18001857
:1055F0003C24A4F8FC8400447C78441C1800004837
:105600005C54547424000000043E7F442400003C99
:105610007C40403C7C40001C3C60603C1C00003CEA
:105620007C6030607C3C00446C3810386C44009CDA
:10563000BCA0A0FC7C00004C64745C4C64000008BE
:10564000083E7741410000000000777700000041EC
:1056500041773E08080000020301030203010078BD
:105660007C4643467C78001EBFE161331200003A5D
:105670007A40407A7A4000387C56575D1800000224
:10568000237555557D7B42217554547D794000200A
:105690007557567C78400000227755557F7A401C1C
:1056A000BEE26236140000023B7D55555D1B023997
:1056B0007D54545D190000387D57565C1800000178
:1056C000457C7C410100000203457D7D43020000D2
:1056D000457F7E40000000797D26267D79000070A0
:1056E0007A2D2D7A700000447C7E575544000020AE
:1056F0007454547C7C54547C7E0B097F7F49003267
:105700007B49497B320000327A48487A32000030C7
:10571000794B4A783000003A7B41417B7A4000382F
:1057200079434278784000BABAA0A0FA7A000039EA
:105730007D4444447D39003D7D40407D3D0000383E
:105740007C64544C7C3800687E7F49436620005C52
:105750003E7349673E1D00446C38386C440000407D
:10576000C888FE7F090B02207456577D78400000E0
:10577000447E7F410000003078484A7B3100003889
:105780007840427B7940007A7B090B7A7301007A7A
:105790007B19337A7B010000262F292F2F28000048
:1057A000262F29292F260030784D45602000001C27
:1057B000227D4B5B65221C08080808383800006110
:1057C0003F1FCCEEABB990613F1F4C6673D9F80018
:1057D0000060FAFA600000081C3622081C362222FB
:1057E000361C0822361C08AA005500AA005500AA3B
:1057F00055AA55AA55AA5555FFAAFF55FFAAFF005D
:105800000000FFFF000000101010FFFF00000070FC
:10581000782C2E7B71000072792D2D797200007129
:105820007B2E2C787000001C225D555541221C14E3
:1058300014F7F700FFFF000000FFFF00FFFF001458
:1058400014F4F404FCFC0014141717101F1F0018A4
:105850003C24E7E72424002B2FFCFC2F2B00001016
:105860001010F0F00000000000001F1F10101010BA
:1058700010101F1F101010101010F0F0101010005A
:105880000000FFFF1010101010101010101010105A
:105890001010FFFF101010227755577E7B410072C9
:1058A0007B2D2F7A73010000001F1F1017171400A3
:1058B00000FCFC04F4F41414141717101717141434
:1058C00014F4F404F4F4140000FFFF00F7F71414C8
:1058D000141414141414141414F7F700F7F71466BE
:1058E0003C3C243C3C6600052772577D380000494B
:1058F0007F7F49637F1C00467D7D555546000045EE
:105900007D7C5455450000447D7F56544400000A78
:105910000E08000000000000447E7F4500000002E9
:10592000457D7D4502000001457C7C45010000105D
:1059300010101F1F000000000000F0F0101010FFFA
:10594000FFFFFFFFFFFFFFF0F0F0F0F0F0F0F000DE
:105950000000777700000000457F7E440000000FC4
:105960000F0F0F0F0F0F0F387C4647457C3800FC98
:10597000FE2A2A3E1400003A7D4545457D3A00380E
:105980007C4547467C3800327B494B7A3301003AEC
:105990007F4547467F390080FE7E20203E1E004224
:1059A0007E7E541C080000417F7F55141C08003C7B
:1059B0007C42437D3C00003A794141793A00003C09
:1059C0007D43427C3C0000B8B8A2A3F97800000CEB
:1059D0005C72735D0C000002020202020200000011
:1059E000000203010000001010101010100000440D
:1059F000445F5F44440000282828282828000071BC
:105A0000351F4C6673D9F8060F097F7F017F7FDA57
:105A1000BFA5A5FD59030208086B6B08080000002C
:105A200080C0400000000000060F090F06000002C1
:105A30000200000202000000000010100000000040
:105A400012131F1F101000001115151F1F0A000050
:105A5000191D151712000000003C3C3C3C000000E2
:105A60000000000000000000000000000078151495
:105A70001578002055545578003845444538003095
:105A800049484930003C4140413C00384140217880
:105A9000007E1515150A0022170F172200008482B8
:105AA000FF828400000000000000000000000010E1
:105AB000385410101E0000000000001010101010CC
:105AC000101010107C1010000000000000081400DE
:105AD0000014081008040408100810202010080002
:105AE000081422410000412214080004027F02042D
:105AF0000010207F201000103854101010101010CB
:105B000054381010181C1C181008183838180800C1
:105B1000081C3E7F00007F3E1C080006090909069C
:105B20000006497D49060000000000000000002F2B
:105B3000000000000700070000147F147F140024F9
:105B40002A6B2A120023130864620036495522503A
:105B500000000503000000001C224100000041225B
:105B60001C000014083E08140008083E0808000045
:105B700050300000000808080808000060600000BD
:105B8000002010080402003E5149453E0000427FBB
:105B90004000004261514946002141454B31001807
:105BA00014127F10002745454539003C4A494930C9
:105BB0000003017109070036494949360006494981
:105BC000291E00003636000000005636000000088E
:105BD000142241000014141414140000412214086B
:105BE00000020151090600324979413E007E11113F
:105BF000117E007F49494936003E41414122007FE4
:105C00004141221C007F49494941007F090909019E
:105C1000003E4149497A007F0808087F0000417F23
:105C20004100002040413F01007F08142241007FD5
:105C300040404040007F020C027F007F0408107F3C
:105C4000003E4141413E007F09090906003E4151A5
:105C5000215E007F09192946004649494931000162
:105C6000017F0101003F4040403F001F2040201FB6
:105C7000003F4038403F0063140814630007087079
:105C80000807006151494543007F4141000000027F
:105C900004081020000041417F00000402010204BA
:105CA00000404040404000000102040000205454E5
:105CB0005478007F48444438003844444420003835
:105CC0004444487F00385454541800087E090102A7
:105CD000000C5252523E007F080404780000447DBC
:105CE0004000002040443D00007F10284400000098
:105CF000417F4000007C04180478007C080404788C
:105D0000003844444438007C141414080008141467
:105D1000187C007C080404080048545454200004F3
:105D20003F444020003C4040207C001C2040201C80
:105D3000003C4038403C004428102844000C50509F
:105D4000503C004464544C440000083641000000BC
:105D5000007F00000000413608000008082A1C08E7
:105D600000081C2A08080031313532303000353740
:105D70003630300033383430300031393230300092
:105D80003936303000343830300032343030002092
:105D90001A202020201B2020202020457869740014
:105DA000202030313233343536373839414243449C
:105DB00045460D0A006D002E002E006B6D2F680009
:105DC0002E00636D002020006F6B00200044006EE9
:105DD0006F0032440033440020002D00780058004A
:105DE0004F00416C742020202020203A20004C617C
:105DF000742020202020203A20004C6F6E67202045
:105E00002020203A20005370656564202020203A2D
:105E1000200050444F5020202020203A2000416391
:105E2000637572616379203A2000536174202020E9
:105E30002020203A20004669782054797065203A65
:105E400020004E7572206D6974204E432021002180
:105E500021216E6F7420696D706C656D656E74655F
:105E600064212121002E002E004D4B3A004469731D
:105E7000743A0053706565643A00466C7974696DD4
:105E8000653A004F4B002121436865636B205061E8
:105E900072616D65746572212120003030303000F0
:105EA000303030302D30302D303030303030005008
:105EB0004B54204365627261200030303030005313
:105EC00074616E646172647765727465206765736E
:105ED00065747A740077657264656E20617566001A
:105EE00020454550524F4D20506172616D6574657B
:105EF00072202020200020202057726974652045E0
:105F00004550524F4D20202020004F4B00636865C4
:105F1000636B207468652073657474696E677321A0
:105F20000020202020202056657273696F6E20208B
:105F30002020202000454550726F6D5570646174BB
:105F40006520746F206E6577004F4B000D0A00725C
:105F50000A00496E717569727920456E64000D0AF8
:105F600000496E717569727920526573756C74732E
:105F70003A0D0A002E004552524F520D0A004F4B67
:105F80000D0A000D004154423F004154533100417D
:105F9000544E3D004154523100415452300041545E
:105FA0004F300041544F31004154463F004154446A
:105FB0003D004154443000415448004154410041A7
:105FC0005400415445310041545130004154453052
:105FD00000415451310041544C350041544C34007F
:105FE00041544C330041544C320041544C31004137
:105FF000544C300041544C2A0041545A3000415412
:10600000503D0054696D65206F75742C4661696C54
:1060100020746F20636F6E6E6563742100434F4E72
:106020004E45435400444953434F4E4E454354005C
:106030000D0A00425420696E697469616C69736964
:106040006572656E2E2E00736574204261756472F0
:10605000617465204572726F7200736574204261CD
:10606000756472617465206F6B004572726F723176
:10607000207365742042617564726174652E2E0010
:10608000425420736574206E657720426175647296
:106090006174652E2E0014BE88E10FB6F8948093CB
:1060A0006000109260000FBE11241FBECFEFD0E43D
:1060B000DEBFCDBF11E2A0E0B1E0E4E3FAEB01E026
:1060C0000BBF02C007900D92AC32B107D9F71AE3AB
:1060D000ACE2B1E201C01D92A432B107E1F70E9427
:1060E00068380C9418DD0C9400008FEF81B914B857
:1060F00017B81AB880B18093B92883B18093BB28B0
:1061000086B18093B82889B18093A628379B02C0B6
:1061100081E001C082E08093BA2808958091BA2876
:10612000813009F447988091BA28823009F45F9849
:1061300008958091BA28813009F4479A8091BA284D
:10614000823009F45F9A08958091BA28813081F4F1
:106150008091EF32882359F48091B0008368809356
:10616000B0008091B10081608093B10001C05F9A5E
:106170008091BA28823009F4479A08958091BA280C
:10618000813051F48091EF32882329F41092B000CD
:106190001092B10001C05F988091BA28823009F452
:1061A0004798089580912C21882369F4439881E0D1
:1061B00080932C2180E29EE424EF31E0F9013197B5
:1061C000F1F70197D9F70895439A10922C21089579
:1061D0000F930E94753082B1806F82B90C98099834
:1061E0008FEF84B988B1806988B987B18C6E87B91F
:1061F0003C9843985E9A8AB1806F8AB9299A0E9426
:10620000167281E08093A12A84E190E00E940C55EF
:1062100084E190E00E94E65381E00E9477B280E042
:106220000E944CB80E942CCB84E10E94AD5A789415
:106230008091E83280934E268091E8320E94045487
:106240008091E8320E943D5580917632843080F012
:1062500081E0809376328091763290E060E070E069
:1062600043E050E02FE50AE00E9476888093763282
:106270008091EF328823C9F48091BA288130A9F443
:106280000E943C7260917F3270E0882777FD809594
:10629000982F0E94EFD623E333E343E250E40E94B9
:1062A000DCD70E94C1D66093B3008091EF32813079
:1062B00011F40E94767F81E00E944CB880E991E061
:1062C00060E870E040E00E946A7310926F2C0E94B8
:1062D00013B68091BA28813071F482E060E049E021
:1062E00052E020E00E947EBB87E061E041E052E0A6
:1062F00020E00E947EBB8091BA28823069F460E081
:106300004FEE51E020E00E947EBB87E061E047EE67
:1063100051E020E00E947EBB80E063E04DED51E063
:1063200020E00E947EBB88E063E046ED51E023E080
:106330000E947EBB86E090E00E94903EAC0180E02F
:1063400065E020E00E94ACBB87E090E00E94903EB8
:10635000AC0180E066E020E00E94ACBB80E49FE1FD
:1063600024EF31E0F9013197F1F70197D9F7079957
:10637000299888EE93E024EF31E0F9013197F1F7A5
:106380000197D9F780E991E060E870E040E00E9471
:106390006A7380EF0E9405738091EF324091F13271
:1063A00089EF91E064E670E00E94E07D4091F13277
:1063B00083E092E064E670E00E94E07D4091F1327B
:1063C0008DE092E064E670E00E94E07D4091F13261
:1063D00087E192E064E670E00E94E07D4091F13256
:1063E0008DE092E064E670E00E94E07D4091F13241
:1063F00083E092E064E670E00E94E07D4091F1323B
:1064000089EF91E064E670E00E94E07D0E9483B72E
:10641000439A10922C2180918332813041F48091F3
:106420008532882321F48091E8320E946F4F0E94C8
:1064300083B780918432813031F480918632882311
:1064400011F40E9484D30E947CCB0E9483B7809178
:106450008332813051F58091A528882331F585E07C
:106460000E947D328091D932813009F042C088E0AB
:1064700090E00E94903EAC0180E060E020E00E944D
:10648000ACBB89E090E00E94903EAC0180E061E00E
:1064900020E00E94ACBB80E29EE424EF31E0F901F1
:1064A0003197F1F70197D9F724C086E00E947D3239
:1064B0008091D9328130E9F488E090E00E94903EEA
:1064C000AC0180E060E020E00E94ACBB8AE090E09C
:1064D0000E94903EAC0180E061E020E00E94ACBBF5
:1064E00080E29EE424EF31E0F9013197F1F7019762
:1064F000D9F70E9483B70F910895429A289A469A35
:10650000459A823051F0833018F48823F9F00895C9
:106510008530C1F0863071F517C08091C9008F7E3B
:106520008093C9008091C900877F8093C9008091C2
:10653000C9008F778093C900529853985A985B98F6
:106540004298089545980895469808958091C90005
:106550008F7E8093C9008091C900877F8093C90096
:106560008091C9008F778093C900529853985A98A8
:106570005B98289808950E9483B78AE490E00E946F
:10658000903EAC0180E060E022E00E94ACBB88E479
:1065900090E00E94903EAC0180E061E022E00E9429
:1065A000ACBB87E490E00E94903EAC0180E063E0E9
:1065B00020E00E94ACBB80E064E041E352E020E0D8
:1065C0000E947EBB80E065E04BE152E020E00E944B
:1065D0007EBB8BE490E00E94903EAC0180E066E0E0
:1065E00020E00E94ACBB8DE290E00E94903EAC01A6
:1065F0008CE067E020E00E94ACBB80E00E947D322E
:106600005E9880E20E9405738823D9F380EF0E9490
:1066100005735E9A80918132813011F486E001C069
:1066200085E00E947D3208950E9483B780E490E067
:106630000E94903EAC0180E060E022E00E94ACBB92
:1066400088E490E00E94903EAC0180E061E022E0AE
:106650000E94ACBB87E490E00E94903EAC0180E0D9
:1066600063E020E00E94ACBB85E490E00E94903E95
:10667000AC0180E064E020E00E94ACBB89E490E0E3
:106680000E94903EAC0180E065E020E00E94ACBB3F
:1066900080E066E047E452E020E00E947EBB40914B
:1066A000E8328AE066E020E00E94C4BE8DE290E01D
:1066B0000E94903EAC018CE067E020E00E94ACBB01
:1066C00080E00E947D320E94F2B680E20E94057353
:1066D0008823C9F380EF0E94057380918132813055
:1066E00011F486E001C085E00E947D3208950E9489
:1066F00083B780E490E00E94903EAC0180E060E0CF
:1067000022E00E94ACBB86E490E00E94903EAC0187
:1067100080E061E020E00E94ACBB87E490E00E9452
:10672000903EAC0180E063E020E00E94ACBB83E4DB
:1067300090E00E94903EAC0180E064E020E00E9486
:10674000ACBB89E490E00E94903EAC0180E065E043
:1067500020E00E94ACBB8DE290E00E94903EAC0134
:106760008CE067E020E00E94ACBB82E00E947D32BA
:106770000E94F2B680E20E9405738823C9F380EF7D
:106780000E94057380918132813011F486E001C04E
:1067900085E00E947D3208950E9483B780E060E02A
:1067A00040EC52E022E00E947EBB80E061E04AEAD9
:1067B00052E022E00E947EBB80E063E044E952E0C8
:1067C00020E00E947EBB80E064E04EE752E020E0E3
:1067D0000E947EBB80E065E048E652E020E00E9437
:1067E0007EBB80E066E042E552E020E00E947EBB96
:1067F0008DE290E00E94903EAC018CE067E020E0EA
:106800000E94ACBB0E94D23082E00E947D3280E2C6
:106810000E9405738823D9F380EF0E94057380914D
:106820008132813011F486E001C085E00E947D3222
:106830000E94E4300895CF93DF930E9483B780E4F1
:1068400090E00E94903EAC0180E060E022E00E9477
:10685000ACBB84E490E00E94903EAC0180E061E03B
:1068600022E00E94ACBB85E062E041EE52E020E015
:106870000E947EBBC0E0D0E0FE01ED58FD4C9E01C1
:10688000245F822F62E045A120E00E94B5BB2196E3
:10689000C430D10589F782E490E00E94903EAC01BB
:1068A00080E063E020E00E94ACBB85E490E00E94C1
:1068B000903EAC0180E064E020E00E94ACBB89E443
:1068C00090E00E94903EAC0180E065E020E00E94F4
:1068D000ACBB80E066E046ED52E020E00E947EBB6B
:1068E0004091E8328AE066E020E00E94C4BE8DE27A
:1068F00090E00E94903EAC018CE067E020E00E94B6
:10690000ACBB0E94D23080E29EE424EF31E0F9017A
:106910003197F1F70197D9F780918732882319F4DD
:1069200081E00E944ECF80E00E947D320E94F2B64C
:1069300080E20E9405738823C9F380EF0E940573EB
:1069400080918132813011F486E001C085E00E949F
:106950007D320E94E430DF91CF9108950E9483B789
:1069600080918432813009F075C080E490E00E940B
:10697000903EAC0180E060E022E00E94ACBB81E48C
:1069800090E00E94903EAC0180E061E020E00E9437
:10699000ACBB82E490E00E94903EAC0180E063E0FA
:1069A00020E00E94ACBB83E490E00E94903EAC01EA
:1069B00080E064E020E00E94ACBB89E490E00E94AB
:1069C000903EAC0180E065E020E00E94ACBB80E03E
:1069D00066E049EE52E020E00E947EBB4091E83242
:1069E0008AE066E020E00E94C4BE8DE290E00E9452
:1069F000903EAC018CE067E020E00E94ACBB0E94BE
:106A0000D23080E29EE424EF31E0F9013197F1F7D2
:106A10000197D9F780918732882319F481E00E9489
:106A20004ECF82E00E947D320E94F2B680E20E9448
:106A300005738823C9F380EF0E940573809181322A
:106A4000813011F486E001C085E00E947D320E9411
:106A5000E43008958EE390E00E94903EAC0180E027
:106A600061E020E00E94ACBB8FE390E00E94903E8A
:106A7000AC0180E061E020E00E94ACBB89E390E0E3
:106A80000E94903EAC0180E062E020E00E94ACBB3E
:106A90008AE390E00E94903EAC0180E063E020E059
:106AA0000E94ACBB8BE390E00E94903EAC0180E082
:106AB00064E020E00E94ACBB8CE190E00E94903E3C
:106AC000AC018CE067E020E00E94ACBB80E20E9459
:106AD00005738823D9F380EF0E9405730895A1E020
:106AE000B0E0E5E7F5E30C9486DA88E480932D21A5
:106AF0000E9483B783E090E00E94903EAC0180E06A
:106B000067E020E00E94ACBB80912F21813061F4CE
:106B100080E060E041EA53E022E00E947EBB83E136
:106B200067E04EE953E01BC080912E21823061F472
:106B300080E060E048E853E022E00E947EBB83E111
:106B400067E045E853E00BC080E060E04FE653E0CB
:106B500022E00E947EBB83E167E04CE653E020E048
:106B60000E947EBB1092882584EF91E09093A32A27
:106B70008093A22A8CEF898310E058E6452E3324B7
:106B800033944E010894811C911C41E0A42EB12C39
:106B900055245A9434EFC32E31E0D32E24EFE22E45
:106BA00021E0F22E9EEF692E0DEF8CEF782E2DB79F
:106BB0003EB7275030400FB6F8943EBF0FBE2DBFF2
:106BC000EDB7FEB73196ADB7BEB711964C921182B4
:106BD000328294828382B682A5820E943356598281
:106BE00084EC99E02DB73EB7295F3F4F0FB6F8947C
:106BF0003EBF0FBE2DBFF6013197F1F70197D9F7D0
:106C0000809188258823E9F10E94985580912E2152
:106C1000882341F51091C628115610932E2111306A
:106C200081F460E046E553E022E00E947EBB83E110
:106C300067E043E553E020E00E947EBB10932F21E4
:106C400011C080E060E04DE353E022E00E947EBB93
:106C500083E167E04AE353E020E00E947EBB82E0EC
:106C600080932F211092182980E062E048EC58E2CE
:106C70000E94DBBB10928825F092A32AE092A22A00
:106C800011E080E80E940573882331F480E862E017
:106C90000E945E73882311F0698239C080E40E94EB
:106CA0000573882331F480E462E00E945E738823D8
:106CB00011F009832CC080912E21813041F580E1B3
:106CC0000E940573882319F180912F21813071F47E
:106CD0000E94AA5780E060E044E253E022E00E9474
:106CE0007EBB83E167E041E253E00DC00E94F355B3
:106CF00080E060E04BE053E022E00E947EBB83E155
:106D000067E048E053E020E00E947EBB798280E2A9
:106D10000E940573882339F48091A22A9091A32AB6
:106D2000892B09F044CF80EF0E94057310922D212A
:106D3000109288258091A22A9091A32A892BB9F4D8
:106D4000112311F00E9483B780E062E044EF52E02B
:106D500020E00E947EBB84E690E09093A32A80937B
:106D6000A22A8091A22A9091A32A892BD1F70E946E
:106D7000F3552196E1E10C94A2DAA0E0B0E0E3EC57
:106D8000F6E30C9490DA8BE10E9476558BE10E9439
:106D9000765585E50E9476558AEA0E94765580E010
:106DA0000E94765586E580932D2100E096E7D92E46
:106DB00084E1E82EF12CCAE5D0E00E9483B78BE194
:106DC00090E00E94903EAC0180E064E020E00E94F0
:106DD000ACBB8CE190E00E94903EAC018CE067E09F
:106DE00020E00E94ACBB12E33BC000D00F92EDB795
:106DF000FEB73196ADB7BEB71196DC921182128202
:106E00000E943356F092A32AE092A22A0F900F908C
:106E10000F908091A22A9091A32A892BD1F7053156
:106E200048F4802F66E049ED53E020E00E947EBBED
:106E30000F5F06C080E066E045E10E9413BC00E001
:106E400080E20E940573882351F080EF0E94057351
:106E50001092823210922E210E945F3CF9CF115085
:106E600080918825882321F4112309F0BECF02C028
:106E70001123A9F480E290E00E94903EAC0180E0F2
:106E800065E020E00E94ACBBD093A32AC093A22A65
:106E90008091A22A9091A32A892BD1F78ECF0E94AC
:106EA000985580918A2590918B259093BD28809349
:106EB000BC288091D9328130B1F40E9483B781E23D
:106EC00090E00E94903EAC0180E060E020E00E94F3
:106ED000ACBB82E290E00E94903EAC0180E061E0B9
:106EE00020E00E94ACBB8091C628823681F480915C
:106EF000D932813051F483E290E00E94903EAC019F
:106F000080E062E020E00E94ACBB82E015C080918E
:106F1000C628833611F010E014C08091D932813038
:106F200051F484E290E00E94903EAC0180E062E087
:106F300020E00E94ACBB81E080932E2180932F2122
:106F400011E08091D9328130B1F585E290E00E9464
:106F5000903EAC0180E063E020E00E94ACBBE09199
:106F6000BC28F091BD2889E063E040810E946FBE9B
:106F70008AE063E047ED53E020E00E947EBBE091B1
:106F8000BC28F091BD288BE063E041810E946FBE78
:106F9000E091BC28F091BD2844814F598EE063E018
:106FA0000E946FBE88EA91E624EF31E0F901319743
:106FB000F1F70197D9F70E94AA578FEF0E94213F5E
:106FC00080918232882309F06DC0E091BE28F09153
:106FD000BF2880818B3509F465C00E9483B780E0AB
:106FE00060E04CEC53E020E00E947EBB8BE50E9409
:106FF00038BE86E290E00E94903EAC018DE060E0F9
:1070000020E00E94ACBB80E062E041EC53E020E075
:107010000E947EBBE091BE28F091BF2880810E9433
:1070200038BE87E290E00E94903EAC018DE062E0C5
:1070300020E00E94ACBB88E290E00E94903EAC0150
:1070400080E064E020E00E94ACBB89E290E00E9416
:10705000903EAC0180E065E020E00E94ACBB8CE09B
:1070600065E04BEB53E020E00E947EBB8AE290E0BB
:107070000E94903EAC0180E066E020E00E94ACBB44
:1070800010922E218CED95E060E470E040E00E94CB
:107090006A7380E49CE924EF31E0F9013197F1F75C
:1070A0000197D9F710922D211092882582E390E064
:1070B0009093A32A8093A22A8091A22A9091A32A36
:1070C000892BD1F7812FCDB7DEB7E7E00C94ACDA8E
:1070D000EF920F930E94E83010922E2110922F21F0
:1070E0008091D932813009F03DC00E9483B78BE096
:1070F00090E00E94903EAC0180E060E020E00E94C1
:10710000ACBB8CE090E00E94903EAC0180E061E07E
:1071100020E00E94ACBB8DE090E00E94903EAC016C
:1071200080E063E020E00E94ACBB85E190E00E943B
:10713000903EAC0180E064E020E00E94ACBB80E1C6
:1071400090E00E94903EAC0180E065E020E00E946B
:10715000ACBB88E99AE324EF31E0F9013197F1F70C
:107160000197D9F78091D0329091D132A091D2324B
:10717000B091D3320097A105B10509F444C18091C3
:10718000D4329091D532A091D632B091D7320097B7
:10719000A105B10509F437C10E9483B786E190E0EB
:1071A0000E94903EAC0180E060E022E00E94ACBB17
:1071B00089E190E00E94903EAC0180E061E022E035
:1071C0000E94ACBB87E190E00E94903EAC0180E061
:1071D00062E022E00E94ACBB88E190E00E94903E19
:1071E000AC0180E067E020E00E94ACBB6091D4324B
:1071F0007091D5328091D6329091D73220E836E91D
:1072000048E950E00E9448DA81E064E0A90122E008
:1072100030E000E0EE240E945BC183E064E049EBD3
:1072200053E020E00E947EBB6091D4327091D53251
:107230008091D6329091D73228EE33E040E050E092
:107240000E9448DACA01B90120E137E240E050E08B
:107250000E9448DA9B01AC0184E064E0A90124E0CB
:1072600030E001E00E945BC16091D4327091D53270
:107270008091D6329091D7322AE030E040E050E061
:107280000E9448DACA01B90124E630E040E050E04B
:107290000E9448DA9B01AC0188E064E0A90122E089
:1072A00030E00E945BC16091D0327091D132809108
:1072B000D2329091D33220E836E948E950E00E947A
:1072C00048DA8CE064E0A90122E030E000E00E94AE
:1072D0005BC18EE064E047EB53E020E00E947EBBA0
:1072E0006091D0327091D1328091D2329091D3326C
:1072F00028EE33E040E050E00E9448DACA01B901CC
:1073000020E137E240E050E00E9448DA9B01AC0106
:107310008FE064E0A90124E030E001E00E945BC15D
:107320006091D0327091D1328091D2329091D3322B
:107330002AE030E040E050E00E9448DACA01B9019A
:1073400024E630E040E050E00E9448DA9B01AC01C6
:1073500083E164E0A90122E030E00E945BC180E8A3
:107360000E9405738823A9F160E070E080E090E05E
:1073700020E030E040E050E00E94BAC980E060E2E6
:1073800040E828E000E00E94DCB980E068E240E8E4
:1073900028E00E94DCB98AE190E00E94903EAC01B6
:1073A00080E065E020E00E94ACBB80E066E045E163
:1073B0000E9413BC80E067E045E10E9413BC80E1BD
:1073C00097E224EF31E0F9013197F1F70197D9F70E
:1073D0001AC080E10E940573882309F4C0CF80E0C1
:1073E00064E045E10E9413BC80E065E045E10E9455
:1073F00013BC80E066E045E10E9413BC80E067E0DA
:1074000045E10E9413BC0E94BD360E945F3CFDCF47
:107410000F931F93982F062F142F842F692F45E168
:107420005AE020E00E947EBB812F602F43E15AE0AA
:1074300020E00E947EBB1F910F9108958F929F9232
:10744000AF92BF92DF92EF92FF920F931F93CF9371
:10745000DF930E9483B780E060E04EE059E022E0D5
:107460000E947EBB8DE060E047E059E022E00E9490
:107470007EBB80E061E041EF58E022E00E947EBBED
:107480008CE090E00E94903EAC0180E061E022E060
:107490000E94ACBB81E090E00E94903EAC0180E095
:1074A00067E020E00E94ACBBDD2486E1882E912CB1
:1074B000ED2CFF24E89C8001E99C100DF89C100D38
:1074C00011240352184FC0E0D0E05701CE018E0DB9
:1074D0009F1D0C9744F4CE018D5F682F80E0A801BA
:1074E00020E00E947EBB21960A5E1F4FC330D1056B
:1074F00069F7DD2009F057C080E062E04FEE58E008
:1075000020E00E947EBB80E066E04DEE58E00BC0BC
:1075100080E062E04BEE58E020E00E947EBB80E01D
:1075200066E049EE58E020E00E947EBB99E0A91693
:10753000B10474F080E062E047EE58E020E00E9481
:107540007EBB80E066E045EE58E020E00E947EBB16
:1075500080E40E940573882329F089E0A816B1040D
:107560000CF4D39480E80E940573882311F0D110A5
:10757000DA9480E20E940573882331F480E10E944E
:107580000573882309F494CF80EF0E940573DF917F
:10759000CF911F910F91FF90EF90DF90BF90AF9030
:1075A0009F908F90089599E0A916B1041CF6B0CF72
:1075B0000E9483B780E062E049E359E020E00E9446
:1075C0007EBB80E063E049E259E020E00E947EBBA0
:1075D0008CE067E044E259E020E00E947EBB80E25C
:1075E0000E9405738823D9F380EF0E9405730895E4
:1075F0000E9483B780E060E046EA59E022E00E9402
:107600007EBB80E390E00E94903EAC0180E061E0B0
:1076100020E00E94ACBB81E390E00E94903EAC0170
:1076200080E062E020E00E94ACBB80E063E040E9E3
:1076300059E020E00E947EBB80E064E04AE759E028
:1076400020E00E947EBB80E065E044E659E020E057
:107650000E947EBB80E066E04EE459E020E00E949C
:107660007EBB82E390E00E94903EAC0180E067E048
:1076700020E00E94ACBB80E20E940573882321F0C9
:1076800080EF0E940573089580E10E9405738823AE
:1076900091F32CE088E190E00FB6F894A8958093E0
:1076A00060000FBE20936000FFCFBF92CF92DF92A9
:1076B000EF92FF920F931F93D82EE62E142FB22E27
:1076C000C02E842F642F41E00E94083A012FF12E32
:1076D00080E40E940573182F80E461E00E945E73CD
:1076E000182B51F00E1510F40F5F06C081E0C8167C
:1076F00011F40EEF24C00E2D80E80E940573182FA0
:1077000080E861E00E945E73182B51F0D01610F4EF
:10771000015006C081E0B81611F40DEF10C00D2D18
:107720000F1529F08F2D602F41E00E94083A80E369
:107730000E940573F02E882359F285FD0FEF802FEC
:107740001F910F91FF90EF90DF90CF90BF90089521
:10775000CF92DF92EF92FF920F931F93C82ED62EF7
:10776000E42E122F822F622F0E94083A012FF12E51
:1077700080E40E940573182F80E461E00E945E732C
:10778000182B29F00D1510F00D2D01C00F5F80E8AA
:107790000E940573182F80E861E00E945E73182B29
:1077A00029F0C01610F00C2D01C001500F1529F062
:1077B0008F2D602F4E2D0E94083A80E30E940573A2
:1077C000F02E8823A9F285FD0FEF802F1F910F91D6
:1077D000FF90EF90DF90CF900895BF92CF92DF920D
:1077E000EF92FF920F931F93D82EE62E142FB22EF6
:1077F000C02E842F642F41E00E94083A012FF12E01
:1078000080E40E940573182F80E461E00E945E739B
:10781000182B51F00E1510F40F5F06C081E0C8164A
:1078200011F40EEF43C00E2D80E80E940573182F4F
:1078300080E861E00E945E73182B51F0D01610F4BE
:10784000015006C081E0B81611F40DEF2FC00D2DC8
:1078500080E20E942073882329F080EF0E94057344
:107860000AEF24C080E10E942073882329F080EF72
:107870000E9405730BEF1AC080E20E940F738823E9
:1078800029F080EF0E9405730CEF10C00F1529F04E
:107890008F2D602F41E00E94083A0E94F2B680E1ED
:1078A0000E940F73F02E882309F4AACF802F1F9116
:1078B0000F91FF90EF90DF90CF90BF900895A4E0DC
:1078C000B0E0E5E6FCE30C9485DA20912E212A83D2
:1078D00080EF0E940573552444241982AA24A3949E
:1078E00001C0A12E80918232813011F480932E212B
:1078F00080918232882319F43A8130932E2180912D
:107900002E21882319F456E0452E09C0813019F440
:1079100049E0442E04C0823011F434E0432E0E942A
:1079200083B780E060E046E05AE022E00E947EBB40
:107930008CE060E040E05AE022E00E947EBB81E003
:1079400090E00E94903EAC0180E067E020E00E9461
:10795000ACBB8CE290E00E94903EAC018CE067E012
:1079600020E00E94ACBB642C77241301089421080A
:107970003108552039F081E061E04EEF59E020E018
:107980000E947EBBE52CFF24E6E3F0E0EE9EC00102
:10799000EF9E900DFE9E900D11249C838B8300E042
:1079A00010E0BB24B394670148018E0C9F1C861421
:1079B00097048CF580912E21813069F440917632C4
:1079C000F2E14F9FA00111242B813C81420F531FF4
:1079D00045525C4F1BC0823069F44091763232E1EF
:1079E000439FA00111248B819C81480F591F4F5345
:1079F0005A4F0CC04091763292E1499FA001112468
:107A0000EB81FC814E0F5F1F4756594F83E06B2D72
:107A100020E00E947EBB053051F4821493043CF4B4
:107A200081E066E04CEF59E020E00E947EBB0E94BE
:107A3000F2B60F5F1F4FB3942B813C812A5C3F4FFE
:107A40003C832B8337E0B31609F0AECF89818823BE
:107A500079F45520D1F496E0941528F481E065E09E
:107A60004A2D20E016C081E0642D4A2D20E00BC095
:107A7000E6E0F0E0CE0EDF1EC614D70434F082E05C
:107A800066E04A2D21E000E005C082E065E04A2D75
:107A900021E001E00E94ED3B182F8E3F31F453941A
:107AA000F1E0F98325E0A22E64CF8D3F29F45A94AA
:107AB000198292E0A92E5DCF8C3F09F04BC00E9445
:107AC00083B78EE290E00E94903EAC0180E062E0DD
:107AD00020E00E94ACBB8FE290E00E94903EAC019F
:107AE0008CE067E020E00E94ACBB80E10E9405735F
:107AF000882319F00E94CBC9299880E20E940F7355
:107B0000882399F380EF0E9405730E9483B780E079
:107B100060E04FEE59E022E00E947EBB8CE060E026
:107B200049EE59E022E00E947EBB81E090E00E9495
:107B3000903EAC0180E067E020E00E94ACBB8CE2AC
:107B400090E00E94903EAC018CE067E020E00E9453
:107B5000ACBB0FCF8B3F19F40E94B34BDDC08A3F03
:107B600009F4DAC080912E21813009F055C0E12E50
:107B7000FF24E50CF11C21E0E216F10419F40E9447
:107B800010AB15C032E0E316F10419F40E946F3512
:107B900028C083E0E816F10419F40E94E57128C0BA
:107BA00094E0E916F10419F40E94074A28C0E5E0C0
:107BB000EE16F104B1F487E00E94D1B880E067E0EE
:107BC00043ED59E020E00E947EBB80E197E2E4EFC4
:107BD000F1E03197F1F70197D1F787E00E94F6B80D
:107BE00015C0F6E0EF16F10419F40E948EC614C019
:107BF00027E0E216F10419F40E9484C70DC038E0B2
:107C0000E316F10419F40E94507706C089E0E816E3
:107C1000F10411F40E94904C80912E21823069F57C
:107C2000812F90E0850D911D8130910519F40E94FE
:107C30006F3523C08230910519F40E94074A1DC098
:107C400083309105B1F487E00E94D1B880E067E00D
:107C50004CEB59E020E00E947EBB80E197E2E4EF2C
:107C6000F1E03197F1F70197D1F787E00E94F6B87C
:107C700004C0049711F40E94904C80912E21882317
:107C800009F02FCEE12EFF24E50CF11C91E0E9165E
:107C9000F10441F40E94BD36882359F0E0912E2171
:107CA000EA831FCEF2E0EF16F10419F482E00E949D
:107CB000F8AE80918132882371F423E0E216F1045A
:107CC00019F40E941B3420C034E0E316F104A9F437
:107CD0000E94143319C080918132813071F483E0A5
:107CE000E816F10419F40E94AE340EC094E0E916CF
:107CF000F10419F40E94773307C0E5E0EE16F104B1
:107D000019F40E945693EDCDF6E0EF16F10409F058
:107D1000E8CD0E941E3AE5CD2496E2E10C94A1DA6A
:107D200020917632FC01EE0FFF1FEE0FFF1FE20FD6
:107D3000F11DEE0FFF1FE75EF54F25913491C9014C
:107D40000895A1E0B0E0E7EAFEE30C9489DA8983C4
:107D500083E580932D211092882512E333E7632E6B
:107D60007724739402E04E010894811C911C21E059
:107D7000A22EB12C9CE7C92ED12C84E1E82EF12C47
:107D800032C08DB79EB70B970FB6F8949EBF0FBE4B
:107D90008DBFEDB7FEB73196ADB7BEB711966C92F9
:107DA0007182028394828382B682A5828091BE28EA
:107DB0009091BF2890878783D286C1860E943356D0
:107DC000F092A32AE092A22A8DB79EB70B960FB627
:107DD000F8949EBF0FBE8DBF8091A22A9091A32AD6
:107DE000892BD1F7115080918825882319F411230C
:107DF00041F60AC0112341F00E949855E0918A256E
:107E0000F0918B25808117C083E890E00E94903E1E
:107E1000AC0180E062E020E00E94ACBB84E690E030
:107E20009093A32A8093A22A8091A22A9091A32AB8
:107E3000892BD1F78FEF898389812196EEE00C940D
:107E4000A5DAA1E0B0E0E7E2FFE30C948CDA8983E5
:107E500081E580932D211092882512E361E7962E0B
:107E600001E05E010894A11CB11C51E0C52ED12C8B
:107E700044E1E42EF12C2AC08DB79EB707970FB6C8
:107E8000F8949EBF0FBE8DBFEDB7FEB73196ADB76C
:107E9000BEB711969C9201830283B482A382D682DC
:107EA000C5820E943356F092A32AE092A22A8DB78F
:107EB0009EB707960FB6F8949EBF0FBE8DBF8091F8
:107EC000A22A9091A32A892BD1F71150809188255D
:107ED000882319F4112381F60FC0112369F00E9441
:107EE0009855E0918A25F0918B2581918983F093B3
:107EF000BF28E093BE2818C083E890E00E94903E1F
:107F0000AC0180E062E020E00E94ACBB84E690E03F
:107F10009093A32A8093A22A8091A22A9091A32AC7
:107F2000892BD1F78FEF898389812196EBE00C941F
:107F3000A8DAEF920F930E9483B784E990E00E9441
:107F4000903EAC0180E060E022E00E94ACBB81E0AA
:107F500090E00E94903EAC0180E067E020E00E944B
:107F6000ACBB81E020C0809136210E94213F482F88
:107F70008F3FC9F16091362183E050E021E030E08D
:107F800000E0EE240E945BC1609136214091BE2842
:107F90005091BF2841595F4F85E020E00E942FBBE0
:107FA000809136218F5F80933621809136218630F3
:107FB000D0F28CE890E00E94903EAC0183E066E055
:107FC00020E00E94ACBB8FEF0E94213F282F8F3F03
:107FD00051F081E066E041E00E94A83B80933621A9
:107FE0008091362101C08FEF0F91EF9008950F938C
:107FF0001F93CF93DF9300E0CDE2D0E01FE00E941B
:1080000083B783E990E00E94903EAC0180E060E09D
:1080100022E00E94ACBB81E090E00E94903EAC0167
:1080200080E067E020E00E94ACBB1092302180919C
:108030003121882339F081E061E040ED53E320E015
:108040000E947EBB1092302133C080913121262FB7
:1080500030E0280F311D2E303105ACF4809176329E
:108060006F5F2C9FA0012D9F500D3C9F500D112440
:10807000819FC0011124480F591F495B5E4E83E068
:1080800020E00E947EBB80913021853061F4809198
:10809000312190E008973CF481E066E04EEC53E338
:1080A00020E00E947EBB809130218F5F8093302141
:1080B00060913021663048F280913321882399F411
:1080C00080913121882331F481E065E04091000105
:1080D00020E005C082E065E04091000121E001E080
:1080E0000E94553B082F809133218130A9F4809163
:1080F000312190E008973CF082E066E04091000179
:1081000021E000E006C082E065E04091000121E04E
:1081100001E00E94553B082F0E3F51F48091312120
:108120008F5F8093312181E08093332185E00AC005
:108130000D3F59F48091312181508093312110926B
:10814000332182E0809300015ACF0F3F29F0009342
:10815000000180913121080F802FDF91CF911F9175
:108160000F910895A4E1B0E0E8EBF0E40C9486DA16
:10817000782EFF2440E0282F30E021503040BE010F
:108180006F5F7F4F15C0E42FF0E053E0EE0FFF1F4D
:108190005A95E1F7EB58F14DE4918E2F90E082175C
:1081A000930729F4FB01EF0DF11D4083F3944F5F1A
:1081B000483948F34093302110E0CF2CDD245E0194
:1081C0000894A11CB11C3DE2332E4601089481089D
:1081D00091080E9483B782E990E00E94903EAC0132
:1081E00080E060E022E00E94ACBB81E090E00E9471
:1081F000903EAC0180E067E020E00E94ACBB1092B2
:10820000302180913421882339F081E061E04DE014
:1082100054E320E00E947EBB109230212FE0622EBA
:10822000412C91E0592E03C2E62FF0E080913421D9
:108230009F01280F311D2C153D050CF0E1C1209147
:108240003421809176326F5FEA0DFB1DE20FF11D44
:108250004081439DA0011124869DC0011124480F37
:10826000591F43545C4E83E020E00E947EBB609126
:108270003021262F30E080913421D501A20FB31F89
:10828000FD01E80FF11DE081F0E083E0EE0FFF1F3C
:108290008A95E1F7EA58F14D8491882309F065C089
:1082A00080913421A80FB11DEC91F0E073E0EE0F46
:1082B000FF1F7A95E1F7E758F14DE4916F5FA091C8
:1082C000BE28B091BF28AE0FB11D4C9182E150E0A5
:1082D00023E030E000E0EE240E945BC139E0731639
:1082E00009F08EC160913021262F30E08091342139
:1082F000A901480F511D4830510509F081C18091F5
:108300003421D501A20FB31FFD01E80FF11D8481B7
:10831000E82FF0E053E0EE0FFF1F5A95E1F7E75822
:10832000F14D249180913421A80FB11D14968C91A8
:10833000E82FF0E043E0EE0FFF1F4A95E1F7E85821
:10834000F14D9491E091BE28F091BF28E20FF11D0C
:10835000808198236F5F992321F081E14BE054E302
:108360002EC181E149E054E32AC1813049F5809171
:108370003421A80FB11DEC91F0E033E0EE0FFF1FA8
:108380003A95E1F7E758F14DE491A091BE28B091FC
:10839000BF28AE0FB11D0C916F5F083F08F45CC0A1
:1083A00082E146E054E320E00E947EBB60913021F0
:1083B0006F5FA201401B510984E121E030E01CC144
:1083C000823081F580913421FD01E80FF11DE081BB
:1083D000F0E023E0EE0FFF1F2A95E1F7E758F14D9B
:1083E000249180913421A80FB11DEC91F0E093E02D
:1083F000EE0FFF1F9A95E1F7E858F14D9491E09147
:10840000BE28F091BF28E20FF11D808198236F5F95
:10841000992321F082E142E054E3D1C082E14EEFA2
:1084200053E3CDC08330B9F580913421A80FB11D3D
:10843000EC91F0E083E0EE0FFF1F8A95E1F7E7583B
:10844000F14DE491A091BE28B091BF28AE0FB11DAF
:108450000C910D3020F46F5F82E1402FCAC00931CA
:1084600090F46F5F82E14CEF53E320E00E947EBB0B
:10847000609130216F5F402F50E04C50504083E1BD
:1084800022E030E0B9C0093109F0BAC06F5F82E183
:1084900048EF53E394C08430D1F480913421F50146
:1084A000E80FF11DE20FF31FE081F0E003E0EE0FB3
:1084B000FF1F0A95E1F7E758F14DE4916F5FA09136
:1084C000BE28B091BF28AE0FB11D4C9191C0853030
:1084D000F1F480913421F501E80FF11DE20FF31F53
:1084E000E081F0E0B3E0EE0FFF1FBA95E1F7E75847
:1084F000F14DE4916F5FA091BE28B091BF28AE0FFF
:10850000B11D4C91469DA001112482E173C08630BB
:1085100009F076C04091BE285091BF288091342147
:10852000A80FB11DEC91F0E0A3E0EE0FFF1FAA959C
:10853000E1F7E758F14DE491CA018E0F911DFC015E
:10854000E081EE2329F46F5F82E144EF53E337C00B
:10855000E13029F46F5F82E140EF53E330C0E23055
:1085600029F46F5F82E14CEE53E329C0E33029F434
:108570006F5F82E148EE53E322C0E43029F46F5F7D
:1085800082E144EE53E31BC0E53029F46F5F82E1E2
:1085900040EE53E314C0E63029F46F5F82E14CED06
:1085A00053E30DC0E73029F46F5F82E148ED53E3F8
:1085B00006C06F5FE83039F482E144ED53E320E018
:1085C0000E947EBB1DC0809134212A0D3B1D280FC7
:1085D000311DD901EC91F0E073E0EE0FFF1F7A95A9
:1085E000E1F7E758F14DE4914E0F511DFA0140813A
:1085F00082E150E023E030E000E0EE240E945BC125
:1086000080913021853071F48091342190E005967D
:10861000881599053CF481E066E042ED53E320E0E3
:108620000E947EBB809130218F5F809330216091CA
:108630003021663008F4F8CD809135218823E9F4A3
:1086400080913421882381F4F6E0FF1530F44091C5
:108650009B1F81E065E020E00CC040919B1F81E002
:108660006F2D20E000E006C040919B1F82E065E096
:1086700021E001E00E94553B182F80913521813087
:10868000B9F48091342190E006968C159D053CF05C
:1086900040919B1F82E066E021E000E006C040912F
:1086A0009B1F82E065E021E001E00E94553B182F0E
:1086B0001E3F51F4809134218F5F8093342181E0FB
:1086C0008093352185E00AC01D3F59F48091342103
:1086D0008150809334211092352182E080939B1F3A
:1086E00078CD1F3F59F010939B1FE0913421F0E0AB
:1086F0003197E10FF11DEC0FFD1F1181812F649661
:10870000E1E10C94A2DAA3E0B0E0E9E8F3E40C9430
:1087100085DA082F0E9483B7802E9924740183E0A4
:10872000EE0CFF1C8A95E1F7F701EA58F14D149120
:1087300081E990E00E94903EAC0180E060E022E0A0
:108740000E94ACBB81E090E00E94903EAC0180E0D2
:1087500067E020E00E94ACBB163009F497C320917B
:1087600076328DE290E0889EA001899E500D989E01
:10877000500D11248FE0289F90011124420F531FA8
:1087800043545C4E80E062E020E00E947EBB1123F7
:1087900009F0DCC084E064E04EE754E320E00E948E
:1087A0007EBB8CE066E049E754E320E00E947EBB9C
:1087B00082E090E00E94903EAC0180E067E020E023
:1087C0000E94ACBB4701F701E958F14D149128E72D
:1087D0003EE2E20EF31EF701B490C4010496B5E741
:1087E0006B2EBEE27B2E680E791EF3012491E09180
:1087F000BE28F091BF28E20FF11D50802091362154
:10880000820F911D8B58914DFC01A49085E064E08E
:10881000412F50E023E030E000E0EE240E945BC1F5
:1088200089E064E04B2D50E023E030E00E945BC122
:1088300081E164E04A2D50E023E030E00E945BC11A
:10884000F52CCB2CDD24812E992480E064E04F2D83
:1088500050E023E030E000E0EE240E945BC12F2CCA
:108860003324C1019695982F882797958795B6014F
:108870000E9435DA462F80E068E226E001E00E949F
:10888000DCB9F1E3FB15A8F480E40E940573182F0E
:1088900080E463E00E945E73182B21F02C143D04E9
:1088A0000CF4F39480E80E940573182F80E863E0CD
:1088B00014C080E40E940573182F80E462E00E94D7
:1088C0005E73182B21F02C143D040CF4F39480E813
:1088D0000E940573182F80E862E00E945E73182BD7
:1088E000B1F08F2D90E0881699068CF4019796953B
:1088F000982F882797958795B6010E9435DA862F9D
:1089000068E240E826E000E00E94DCB9FA9480E2E8
:108910000E942073882341F080E068E240E826E06E
:1089200000E00E94DCB9FA2C80E10E940F738823DA
:1089300031F0F51409F4D3C3F301849114C180E23A
:108940000E940F73882309F480CFC9C3113009F046
:1089500019C184E064E047E654E320E00E947EBB56
:108960008CE066E042E654E320E00E947EBB82E0B9
:1089700090E00E94903EAC0180E067E020E00E9421
:10898000ACBBE3E0880C991CEA95E1F7F401E958E7
:10899000F14DD49028E73EE2E20EF31EF701149168
:1089A000C401049665E7662E6EE2762E680E791E87
:1089B000F3012491E091BE28F091BF28E20FF11D50
:1089C000808020913621820F911D8B58914DFC01A2
:1089D0009490F7EFF91580F481E164E04DE554E3FC
:1089E00020E00E947EBB40E051E04919510983E13B
:1089F00064E021E030E006C081E164E0492D50E010
:108A000023E030E000E0EE240E945BC1F82CA12EB0
:108A1000BB244D2C55245FEF252E312C2F2D30E01B
:108A20003B832A8337EF3F1508F0F5C380E064E00D
:108A30004AE554E320E00E947EBBC12C41E0D42EE5
:108A40008A819B81C81AD90A82E064E0A60121E0EC
:108A500030E000E0EE240E945BC134E0CC0CDD1C71
:108A60003A95E1F780E068E24C2D26E001E00E94B3
:108A7000DCB980E40E940573182F80E461E00E9455
:108A80005E73182BA1F539C0EA81FB81EA15FB055D
:108A90006CF4F394F8EFFF1649F480E068E240E8E4
:108AA00026E000E00E94DCB9FF24FA9480E80E94EE
:108AB0000573182F80E863E00E945E73182BE1F1C4
:108AC0008F2D90E048165906BCF501979695982F82
:108AD000882797958795B5010E9435DA862F68E239
:108AE00040E826E000E00E94DCB9FA9425C02A8123
:108AF0003B81283F310509F0FA9480E80E94057314
:108B0000182F80E861E00E945E73182BA9F0C10164
:108B10008F1991098295807F68E240E826E000E0A5
:108B20000E94DCB9F39441F480E068E240E826E07A
:108B30000E94DCB987EFF82E80E20E942073882320
:108B400041F080E068E240E826E000E00E94DCB905
:108B5000F92C80E10E940F73882369F0F81409F45E
:108B6000BEC2F3018491E091BE28F091BF28E80FC6
:108B7000F11DF082AAC280E20E940F73882309F4DB
:108B80004DCFADC2123009F09AC08FE690E00E943E
:108B9000903EAC0183E064E020E00E94ACBB80E743
:108BA00090E00E94903EAC0183E065E020E00E94EE
:108BB000ACBB81E090E00E94903EAC0180E067E0B9
:108BC00020E00E94ACBB28E73EE2E20EF31EF70174
:108BD0000491C401B3E0880F991FBA95E1F7049698
:108BE000A5E7CA2EAEE2DA2EC80ED91EF6012491F0
:108BF000E091BE28F091BF28E20FF11DE0802091A6
:108C00003621820F911D8B58914DFC0144914130CA
:108C100029F488E064E048E554E306C0442339F4CD
:108C200088E065E046E554E320E00E947EBB1E2D0F
:108C3000F12EF02261F081E064E044E554E320E0AD
:108C40000E947EBB81E065E042E554E30BC081E019
:108C500064E040E554E320E00E947EBB81E065E0F3
:108C60004EE454E320E00E947EBB80E80E9405733E
:108C7000882319F0FF2009F4102780E40E9405736F
:108C8000882321F0812F802309F0102780E10E94A2
:108C90000573882369F01E1509F421C2F601849139
:108CA000E091BE28F091BF28E80FF11D10830DC29E
:108CB00080E20E940F73882309F4BACF10C21330E8
:108CC00009F0E4C084E064E04CE354E320E00E9457
:108CD0007EBB8CE066E047E354E320E00E947EBB6D
:108CE00082E090E00E94903EAC0180E067E020E0EE
:108CF0000E94ACBBF3E0880C991CFA95E1F7F401F3
:108D0000E958F14D149128E73EE2E20EF31EF70117
:108D10003490C401049675E7A72E7EE2B72EA80E04
:108D2000B91EF5012491E091BE28F091BF28E20F11
:108D3000F11D408020913621820F911D8B58914D5D
:108D4000FC01549081E164E0452D50E023E030E0E7
:108D500000E0EE240E945BC1F42CC32CDD2464EF00
:108D6000662E6FEF762E6C0C7D1C812E99242F2D94
:108D700030E03B832A83261537053CF480E064E02D
:108D80004F2D50E023E030E014C08A819B818C1588
:108D90009D059CF480E064E045E354E320E00E94FC
:108DA0007EBB4A815B814C50504081E064E022E010
:108DB00030E000E0EE240E945BC1F31439F480E05F
:108DC00064E041E354E320E00E947EBB8A819B8102
:108DD0009695982F882797958795B6010E9435DA42
:108DE000462F80E068E226E001E00E94DCB980E4E2
:108DF0000E940573182F80E462E00E945E73182BB6
:108E000031F0EA81FB81EC15FD050CF4F39480E868
:108E10000E940573182F80E862E00E945E73182B91
:108E2000B1F08F2D90E0881699068CF401979695F5
:108E3000982F882797958795B6010E9435DA862F57
:108E400068E240E826E000E00E94DCB9FA9480E2A3
:108E50000E942073882341F080E068E240E826E029
:108E600000E00E94DCB9F52C80E10E940F7388239A
:108E700031F0F41409F433C1F501849174CE80E229
:108E80000E940F73882309F472CF29C1143009F0AE
:108E9000A9C080E067E04BE154E320E00E947EBB84
:108EA000F02FFD55F983F23050F48FE190E00E94ED
:108EB000903EAC0185E066E020E00E94ACBB402E15
:108EC000552433E0440C551C3A95E1F729E73EE27E
:108ED000420E531EF2018491E091BE28F091BF280A
:108EE000E80FF11DE0800E2DFF2428E0722E97E0A0
:108EF000892E912C81E0A82EB12C10923021C02E09
:108F0000DD241CC0C601022E02C0959587950A94E7
:108F1000E2F780FF06C0872D821B64E049E154E33D
:108F200005C0872D821B64E047E154E320E00E94E6
:108F30007EBB809130218F5F809330212091302142
:108F4000283000F31F2D1F5F812F65E045E154E3BA
:108F500020E00E947EBB80E80E940573882311F404
:108F60001F2D0AC0812F65E043E154E320E00E94F9
:108F70007EBB183009F410E0F981F23050F480E43F
:108F80000E942073882329F0002311F40AEA01C00B
:108F900000E080E40E940F73882351F0C401811B1C
:108FA0009109950102C0220F331F8A95E2F702272B
:108FB00080E10E940F73882369F00E1509F48FC0B9
:108FC000F2018491E091BE28F091BF28E80FF11DD5
:108FD00000837BC080E20E940F73882309F07FC06A
:108FE000F12E8BCF153009F07EC082E090E00E9418
:108FF000903EAC0180E067E020E00E94ACBB802E98
:10900000992403E0880C991C0A95E1F729E73EE2D0
:10901000820E931EF4018491E091BE28F091BF2846
:10902000E80FF11DB08086E690E063E270E040E179
:1090300050E021E00E9457C3FB2C1FE0A12E0AC084
:10904000FE1439F086E663E24FE0960100E00E94EC
:10905000BDC3FE2CFA9C6001112486E663E24FE05A
:10906000960101E00E94BDC380E40E940573182FA1
:1090700080E461E00E945E73182B11F4EF2C06C0AF
:10908000EF2CE394F8E1EF1609F4EE2480E80E9457
:109090000573182F80E861E00E945E73182B29F099
:1090A000EE2011F4B8E1EB2EEA9480E10E940F73F8
:1090B000882379F0EB1499F0F4018491E091BE28B3
:1090C000F091BF28E80FF11DE08281E08093372105
:1090D00006C080E20E940F73882309F4B1CF80EFAD
:1090E0000E940573BFC0163009F0BCC0802E9924C1
:1090F000A3E0880C991CAA95E1F729E73EE2820ECD
:10910000931E81E090E00E94903EAC0180E067E019
:1091100020E00E94ACBBBB245524AA24A39409C020
:10912000BB2039F081E061E041E154E320E00E949E
:109130007EBBEB2CFF248701F4E0000F111FFA9592
:10914000E1F70E0D1F1D0B5C1C4C2224332437014C
:109150006101CE0CDF1C39E0C316D1043CF4622D52
:109160006F5F83E0A80120E00E947EBB85E02816A7
:1091700059F498E0C916D1043CF481E066E04FE070
:1091800054E320E00E947EBB0894211C311C0F5E3A
:109190001F4FE6E02E163104D9F6552039F4BB20D6
:1091A00079F481E065E04A2D20E00EC0F3E06F160F
:1091B000710434F082E066E04A2D21E000E005C051
:1091C00082E065E04A2D21E001E00E94ED3B982F0E
:1091D0008E3F31F4B39455245394E5E0AE2EA0CFE6
:1091E0008D3F29F4BA94552472E0A72E99CF8C3F75
:1091F000C9F18A3008F094CFF4018491E091BE283F
:10920000F091BF28E80FF11DB90EBA94B08281E049
:109210008093372127C080E064E04F2D50E023E0A9
:1092200030E000E0EE240E945BC18A819B8196952C
:10923000982F882797958795B5010E9435DA462F94
:1092400080E068E226E001E00E94DCB980E40E9450
:109250000573182F80E463E00E945E73182B09F0F9
:1092600013CC24CC2396E2E10C94A1DAEF92FF9286
:109270000F931F930E9483B78CE890E00E94903E6A
:10928000AC0180E061E020E00E94ACBB8DE890E0A2
:109290000E94903EAC0180E063E020E00E94ACBB05
:1092A0008EE890E00E94903EAC0180E067E020E014
:1092B0000E94ACBB13E095E0F92E85E063E0412FFE
:1092C00050E021E030E000E0EE240E945BC18EE03F
:1092D00063E04F2D50E021E030E00E945BC180E868
:1092E0000E940573882321F01F5F163009F411E0F6
:1092F00080E40E940573882331F0F39486E0F81629
:1093000011F4FF24F39480E10E940573882309F48B
:1093100070C080E065E046EA54E320E00E947EBB36
:109320008FE890E00E94903EAC0180E065E020E094
:109330000E94ACBB84E090E00E94903EAC018CE0C7
:1093400067E020E00E94ACBB80E10E9405738823A7
:10935000C1F1812F0E94213F8117B9F48F2D0E9406
:10936000A13E8F1591F480E065E040E954E320E0F0
:109370000E947EBB80E990E00E94903EAC0180E0BC
:1093800065E020E00E94ACBB0FC08EE190E00E943F
:10939000903EAC0180E065E020E00E94ACBB86E03E
:1093A00065E04EE00E9413BC84E690E09093A32A0F
:1093B0008093A22A8091A22A9091A32A892BD1F787
:1093C00021C080E20E940573882309F4BDCF80EF9D
:1093D0000E94057380E065E045E10E9413BC8EE8C1
:1093E00090E00E94903EAC0180E067E020E00E94A7
:1093F000ACBB80E20E940573882309F45ECF80EF46
:109400000E9405731F910F91FF90EF900895EF92C6
:109410000F931F930E94AA570E94993F8093362171
:10942000809136218F3F09F425C180913621863005
:1094300019F40E9436491EC10E9483B786E890E065
:109440000E94903EAC0180E060E022E00E94ACBB54
:1094500040913621405D8FE060E022E00E94B5BB84
:1094600087E890E00E94903EAC0183E062E020E05B
:109470000E94ACBB88E890E00E94903EAC0183E083
:1094800063E020E00E94ACBB81E090E00E94903E4F
:10949000AC0180E067E020E00E94ACBB82E063E0CA
:1094A00042E020E000E00E94553B8F3F09F4E2C01B
:1094B000833009F03CC0809136210E94213F809189
:1094C00036210E94A13E90913621891791F480E0C7
:1094D00062E045E10E9413BC80E063E045E10E9448
:1094E00013BC89E890E00E94903EAC0185E062E008
:1094F00011C080E062E045E10E9413BC80E063E0BF
:1095000045E10E9413BC8EE190E00E94903EAC01C8
:1095100080E064E020E00E94ACBB80E29EE424EFA7
:1095200031E0F9013197F1F70197D9F7A3C08091A4
:1095300036218F3F09F49EC0809136210E94213F41
:109540008F3F09F497C0109231211092332181E0AE
:10955000809300011092372111E00E94F73F082FFD
:109560008F3F71F0109234211092352110939B1F80
:10957000802F0E94B2408F3F81F30E948343F8CF37
:1095800080913721813009F075C00E9483B78AE845
:1095900090E00E94903EAC0180E060E022E00E94FA
:1095A000ACBB40913621405D89E060E022E00E9442
:1095B000B5BB4091362189E060E050E021E030E029
:1095C00000E0EE240E945BC18FE690E00E94903E96
:1095D000AC0183E062E020E00E94ACBB80E790E059
:1095E0000E94903EAC0183E063E020E00E94ACBBAF
:1095F00081E090E00E94903EAC0180E067E020E0D6
:109600000E94ACBB82E063E042E020E00E94553B58
:10961000823081F5809136210E94A13E90913621C1
:10962000891791F48BE890E00E94903EAC0183E0B2
:1096300064E020E00E94ACBB89E890E00E94903E8C
:10964000AC0183E065E007C08EE190E00E94903EAF
:10965000AC0180E064E020E00E94ACBB84E690E0D6
:109660009093A32A8093A22A8091A22A9091A32A60
:10967000892BD1F71F910F91EF900895EF920F93DF
:109680001F930E9483B78CE067E042E056E320E03E
:109690000E947EBB80918B2690918C2680509041B9
:1096A00084F00E941FB66091852670918626809175
:1096B0008726909188260E94C1D670938E2660934B
:1096C0008D260E94F2B640918D2650918E2685E01F
:1096D00065E020E030E000E00E94B9BE8AE065E08D
:1096E0004DEF55E320E00E947EBB4091DA3250916D
:1096F000DB3280E066E025E030E0EE240E945BC1D2
:1097000080E40E940573182F80E463E00E945E737A
:10971000182B49F08091DA329091DB320A969093BF
:10972000DB328093DA3280E80E940573182F80E8DC
:1097300063E00E945E73182B49F08091DA329091B9
:10974000DB320A979093DB328093DA3280E20E9418
:109750000573882309F49ECF80EF0E9405731F9143
:109760000F91EF9008951F9311E00E9483B783E358
:1097700090E00E94903EAC0180E068E022E00E9410
:10978000ACBB83E063E04FE156E320E00E947EBB88
:1097900083E064E04FE056E320E00E947EBB81E07E
:1097A00090E00E94903EAC0180E067E020E00E94E3
:1097B000ACBB113061F481E063E04DE056E320E0A2
:1097C0000E947EBB81E064E04BE056E30BC081E089
:1097D00063E049E056E320E00E947EBB81E064E064
:1097E00047E056E320E00E947EBB80E80E940573BC
:1097F000811111E080E40E940573811112E080E183
:109800000E940F738823F9F080918132882359F4E4
:10981000113019F40E941B34A8CF123009F0A5CFE3
:109820000E941433A2CF80918132813009F09DCF04
:10983000113019F40E94AE3498CF123009F095CF50
:109840000E94773392CF80E20E940573882309F447
:10985000B0CF80EF0E9405731F9108950F9310926F
:1098600031211092332181E0809300011092C028B1
:109870001092302180913121882339F081E061E01C
:1098800049E456E320E00E947EBB80E001C08F5F88
:109890008630E8F380933021809133218823A9F426
:1098A00080913121882339F481E060E0409100010A
:1098B00020E000E006C082E065E04091000121E088
:1098C00001E00E94553B8093C02880913321813074
:1098D00051F482E066E04091000121E000E00E9446
:1098E000553B8093C0288091C0288E3F51F48091D1
:1098F00031218F5F8093312181E08093332185E096
:109900000AC08D3F59F480913121815080933121DB
:109910001092332182E080930001AACF0F91089525
:10992000A0E0B0E0E6E9FCE40C9489DAAA249924EA
:10993000BB24B39436E3632E712C22E1822E01C046
:10994000B12E0E9483B780E060E043E356E322E05B
:109950000E947EBB81E090E00E94903EAC0180E0DE
:1099600067E020E00E94ACBBAA2039F081E061E012
:1099700041E356E320E00E947EBBCA2CDD24C69C56
:109980008001C79C100DD69C100D1124C0E0D0E0C2
:109990007E01EC0CFD1C86E0E816F10484F4409195
:1099A0007632CE018F5F682F489DA0011124400FB1
:1099B000511F47545B4C83E020E00E947EBBC530C2
:1099C00059F495E0E916F1043CF481E066E04FE2D9
:1099D00056E320E00E947EBB21960A5C1F4FC630F2
:1099E000D105B1F6992069F4AA2029F481E066E056
:1099F0004B2D20E00AC082E065E04B2D21E001E024
:109A000005C082E066E04B2D21E000E00E94553B5E
:109A1000182F8E3F31F4A3949924939495E0B92E96
:109A2000A3CF8D3F29F4AA94992482E0B82E9CCF2D
:109A30008F3FE1F1C82FD0E0CA0DD11DC130D10553
:109A400021F482E00E94F8AE05C0C230D10511F4C5
:109A50000E94AC5A80918132882361F4C330D105D1
:109A600019F40E941B341CC0C430D10599F40E9423
:109A7000143316C080918132813061F4C330D10536
:109A800019F40E94AE340CC0C430D10519F40E9400
:109A9000773306C0C530D10519F40E94569350CFD4
:109AA000269709F04DCF0E941E3A4ACFCDB7DEB7B8
:109AB000EEE00C94A5DA1F93CF93DF93182F0E944A
:109AC000B4548FEF0E94765582E00E9476558EEF57
:109AD0000E947655812F0E94765584EF91E024EF05
:109AE00031E0F9013197F1F70197D9F710E0C4EFB0
:109AF000D1E00E94B45490E028EE33E0FE013197AB
:109B0000F1F721503040D1F71F5F009719F41A3058
:109B100081F70AC01A3041F0069719F426E030E0C8
:109B200005C02FEF30E002C020E030E0C901DF9136
:109B3000CF911F9108950F931F93CF93DF93082F19
:109B4000162F67FD0BC08FEF0E94765582E00E94B2
:109B50007655802F0E947655812F0EC08FEF0E9480
:109B6000765583E00E947655802F0E9476558EEFC1
:109B70000E947655812F80580E94765510E0C4EFE0
:109B8000D1E00E94B45490E028EE33E0FE0131971A
:109B9000F1F721503040D1F7009721F41F5F1A30C0
:109BA00081F705C0069719F420E030E019C080E085
:109BB00062E04BE456E320E00E940ABC88EE93E0AA
:109BC00060E470E040E00E946A7380E29EE424EF6B
:109BD00031E0F9013197F1F70197D9F72FEF30E034
:109BE000C901DF91CF911F910F9108951F93182FF5
:109BF00080E063E046E556E320E00E940ABC812F46
:109C000060E00E9400BE1093392184EF91E060E48F
:109C100070E040E00E946A7388E893E124EF31E04D
:109C2000F9013197F1F70197D9F71F910895FF9244
:109C30000F931F93082F0E943D5580E061E04AE793
:109C400057E320E00E940ABC0230C1F0033028F440
:109C5000002351F0013041F50CC00430C9F004304C
:109C600090F0053009F519C086E061E043E757E35D
:109C700018C086E061E04CE657E313C086E061E07F
:109C800045E657E30EC086E061E04EE557E309C0C4
:109C900086E061E047E557E304C086E061E040E527
:109CA00057E320E00E940ABC88E790E00E945B4DE9
:109CB000182FF92E80E062E0412F20E00E94DBBDEA
:109CC000212F3F2DC90101978E3F910528F482E095
:109CD0008093382100933A21C9011F910F91FF9081
:109CE00008951F93CF93DF93182F0E9426565E98F6
:109CF00080ED97E024EF31E0F9013197F1F701971A
:109D0000D9F70E9483B7812F0E943D5580E060E023
:109D10004CE357E320E00E940ABC812F0E94174EBB
:109D2000EC01009721F081E08093382124C080E08D
:109D30000E94174EEC010097F1F481E00E94174E4B
:109D4000EC010097C1F482E00E94174EEC010097ED
:109D500091F483E00E94174EEC01009761F484E0D7
:109D60000E94174EEC01009731F485E00E94174ED7
:109D7000EC01009721F0CF3FD10589F515C00E9475
:109D800083B780E060E04CE257E320E00E940ABC29
:109D90001092382180E29EE424EF31E0F9013197FE
:109DA000F1F70197D9F71BC00E9483B780E060E00C
:109DB00047E157E320E00E940ABC88EE93E060E4AC
:109DC00070E040E00E946A7380E29EE424EF31E09C
:109DD000F9013197F1F70197D9F7C0E0D0E0CE0152
:109DE00001978E3F910508F075C00E9483B780915E
:109DF0003A210E943D5580913821813039F480E02C
:109E000060E049E057E320E00E940ABC80913821DD
:109E1000823009F04DC01092853280E060E043EF5F
:109E200056E320E00E940ABC6091E83283E00E9481
:109E30009B4D892BB9F080E061E042EE56E320E0D3
:109E40000E940ABC88EE93E060E470E040E00E946B
:109E50006A7380E29EE424EF31E0F9013197F1F773
:109E60000197D9F76091E8328EE40E949B4D892BCF
:109E7000B9F080E063E04FEC56E320E00E940ABCBA
:109E800088EE93E060E470E040E00E946A7380E254
:109E90009EE424EF31E0F9013197F1F70197D9F70A
:109EA0008091E8320E943D558091E83280934E26A1
:109EB00080E061E045E10E9413BC80E061E046EC97
:109EC00056E320E00E940ABC89E061E04C2F20E0CC
:109ED0000E94DBBD5E9ADF91CF911F910895EF92B2
:109EE000FF920F931F93E82E85E00E947D328091B0
:109EF0004E260E94714E80913821882309F4B4C106
:109F000080E062E042EB56E320E00E940ABC5E98EB
:109F100080ED97E024EF31E0F9013197F1F70197F7
:109F2000D9F70E94265681E56EE70E949B4D892B4A
:109F300011F410E008C080E064E040EB56E320E05C
:109F40000E940ABC11E06091773280E00E949B4D34
:109F5000892B19F081E00E94F64DF12EF394812FA8
:109F600064E04EEA56E320E00E940ABC609177323A
:109F70008BE40E949B4D892B19F082E00E94F64DE4
:109F80000F2D0F5F8F2D64E04CEA56E320E00E9416
:109F90000ABC6091773281E00E949B4D892B19F0B9
:109FA00083E00E94F64D102F1F5F802F64E04AEA85
:109FB00056E320E00E940ABC609177328CE40E9454
:109FC0009B4D892B19F084E00E94F64D012F0F5F05
:109FD000812F64E048EA56E320E00E940ABC8DE04D
:109FE00060E00E949B4D892B19F085E00E94F64DA0
:109FF000102F1F5F802F64E046EA56E320E00E94A6
:10A000000ABC82E063E00E949B4D892B19F086E038
:10A010000E94F64D012F0F5F812F64E044EA56E362
:10A0200020E00E940ABC60917A3285E00E949B4D3C
:10A03000892B19F087E00E94F64D102F1F5F802FAB
:10A0400064E042EA56E320E00E940ABC60917A3262
:10A0500080E50E949B4D892B19F088E00E94F64D07
:10A06000012F0F5F812F64E040EA56E320E00E9459
:10A070000ABC60917B3289E00E949B4D892B19F0CC
:10A0800089E00E94F64D102F1F5F802F64E04EE99B
:10A0900056E320E00E940ABC60917B3284E50E9476
:10A0A0009B4D892B19F08AE00E94F64D012F0F5F1E
:10A0B000812F64E04CE956E320E00E940ABC6091E5
:10A0C000793284E00E949B4D892B19F08BE00E942D
:10A0D000F64D102F1F5F802F64E04AE956E320E021
:10A0E0000E940ABC609179328FE40E949B4D892BBB
:10A0F00019F08CE00E94F64D012F0F5F812F64E074
:10A1000048E956E320E00E940ABC88E061E00E9432
:10A110009B4D892B19F08DE00E94F64D102F1F5F8B
:10A12000802F64E046E956E320E00E940ABC8BE001
:10A1300061E00E949B4D892B19F08EE00E94F64D44
:10A14000012F0F5F812F64E044E956E320E00E9475
:10A150000ABC6091783286E00E949B4D892B19F0F1
:10A160008FE00E94F64D102F1F5F802F64E042E9C0
:10A1700056E320E00E940ABC6091783281E50E949B
:10A180009B4D892B19F08FE00E94F64D012F0F5F38
:10A19000812F64E040E956E320E00E940ABC83E09E
:10A1A0006E2D0E949B4D892B19F080E10E94F64D87
:10A1B000802F64E04EE856E320E00E940ABC80ED68
:10A1C00097E024EF31E0F9013197F1F70197D9F7E2
:10A1D0008EE46E2D0E949B4D892B19F081E10E9427
:10A1E000F64D802F8F5F64E04CE856E320E00E943C
:10A1F0000ABC5E9A809139218823E9F080E062E010
:10A200004AE756E320E00E940ABC8091392160E0D1
:10A210000E9400BE88EE93E060E470E040E00E949F
:10A220006A7380E29EE424EF31E0F9013197F1F79F
:10A230000197D9F70DC080E062E048E656E320E0E0
:10A240000E940ABC0E94ABC98E2D60E00E9400BE35
:10A250008E2D0E943D5580E29EE424EF31E0F9010D
:10A260003197F1F70197D9F71F910F91FF90EF9078
:10A27000089510923C2110923D2110923E2110929F
:10A28000402110923F2110924121E091C128F0918C
:10A29000C22811AA10AAEFE2F3E389E691E02FEFBA
:10A2A00014861482158216821782108211821282FD
:10A2B00013821086118612861386968785871786E5
:10A2C000108A238B118A158A7E9636E3E13DF307C7
:10A2D00039F781E008950E943951089580913F2116
:10A2E0000895982F8823A1F080913F21891780F04D
:10A2F000892F90E001979C0155E0220F331F5A955A
:10A30000E1F7880F991F281B390B215D3C4C02C0D7
:10A3100020E030E0C901089510923C218091412154
:10A32000882309F46AC010923D2180913F2188233F
:10A3300009F449C0ABE3B3E3FD0190E087818823D2
:10A3400039F48081882321F09F5F90933C2104C0E1
:10A350009F5F7E969F3191F790913C21E091C128BB
:10A36000F091C2289923E1F081E080AB892F90E041
:10A370000197FC01B5E0EE0FFF1FBA95E1F7880FDA
:10A38000991FE81BF90BE45CFC4C8081918197FFDD
:10A3900004C0819580933D211DC010923D211AC0BB
:10A3A00010AA90E017968C911797813039F48C9110
:10A3B000882321F09F5F90933D210CC09F5F5E96A4
:10A3C0009F3181F707C010923D21E091C128F091A3
:10A3D000C22810AA80913C21882379F090E001974F
:10A3E0009C0175E0220F331F7A95E1F7880F991FC2
:10A3F000281B390B215D3C4C02C020E030E0C90134
:10A40000089510923C2110923D2180914121882392
:10A4100009F46AC080913F21882309F44BC0AFEB57
:10A42000B6E3FD0191E08781882341F48081882390
:10A4300029F080E2891B80933C2104C09F5F7E97B6
:10A44000903289F790913C21992309F1E091C1283C
:10A45000F091C22880913E2180AB892F90E0019736
:10A46000FC0175E0EE0FFF1F7A95E1F7880F991F49
:10A47000E81BF90BE45CFC4C8081918197FF04C0E0
:10A48000819580933D211DC010923D211AC091E01D
:10A4900017968C911797813041F48C91882329F07D
:10A4A00080E2891B80933D2107C09F5F5E979032B9
:10A4B00079F702C010923D21E091C128F091C228A5
:10A4C00010AA80913C21882379F090E001979C01AB
:10A4D00055E0220F331F5A95E1F7880F991F281B6B
:10A4E000390B215D3C4C02C020E030E0C9010895E9
:10A4F00080914121882309F450C020913C212F31C3
:10A5000008F044C0822F90E0FC0165E0EE0FFF1FD1
:10A510006A95E1F7880F991FE81BF90BEE5BFC4C7D
:10A520008081882379F5822F90E0FC0145E0EE0FD1
:10A53000FF1F4A95E1F7880F991FE81BF90BE55CAF
:10A54000FC4C80818823F1F02F5F20933C21E09127
:10A55000C128F091C22880A98F5F80AB822F90E044
:10A560000197FC01B5E0EE0FFF1FBA95E1F7880FE8
:10A57000991FE81BF90BE45CFC4C808191819923C5
:10A580009CF40EC02F5F2F3109F0BCCFE091C128A1
:10A59000F091C22810AA10923D2120E030E015C0B1
:10A5A000819580933D2102C010923D21822F90E041
:10A5B00001979C01F5E0220F331FFA95E1F7880F10
:10A5C000991F281B390B215D3C4CC9010895882334
:10A5D00031F081E0809341210E948C5108951092C6
:10A5E000412110923D21089580913D210E94715199
:10A5F0000895CF93DF93EC012A89822F81508F3108
:10A6000010F080E07AC0822F90E00197FC0135E0E5
:10A61000EE0FFF1F3A95E1F7880F991FE81BF90B22
:10A62000EE5BFC4CE081E13089F1E130C8F0EF3FB6
:10A6300009F046C08B89882321F0813009F040C0A1
:10A6400006C080913E218F5F80933E2105C080919E
:10A6500040218F5F8093402180913F218F5F23C0F5
:10A660008B89813041F08F3F59F580913E21815097
:10A6700080933E2115C0809140218F5F80934021BF
:10A6800080913E21815080933E211AC08B8988237E
:10A6900069F08F3FA9F4809140218150809340213F
:10A6A00080913F21815080933F210AC080913E21BB
:10A6B0008F5F80933E218091402181508093402183
:10A6C000822F90E00197FC01A5E0EE0FFF1FAA95F5
:10A6D000E1F7880F991FE81BF90BE15DFC4CDE01E7
:10A6E0008EE10D9001928150E1F7E091C128F09147
:10A6F000C22880913E2181AB8A89DF91CF91089554
:10A700001F920F920FB60F920BB60F9211242F9338
:10A710008F939F93EF93FF939091C8002091CE0069
:10A72000E0918525EF5F80918625E81759F48091A7
:10A73000C3289091C42801969093C4288093C3287D
:10A7400082E008C0892F8871E0938525F0E0ED57FD
:10A75000FE4D208380938725FF91EF919F918F91EC
:10A760002F910F900BBE0F900FBE0F901F9018955A
:10A770001F920F920FB60F920BB60F9211248F9368
:10A780009F93EF93FF939091832580918425981751
:10A7900069F0E0918425EF5FEF73E0938425F0E0AA
:10A7A000ED5BFE4D80818093CE0005C08091C90095
:10A7B0008F7D8093C900FF91EF919F918F910F90B2
:10A7C0000BBE0F900FBE0F901F9018959C0110921A
:10A7D000832510928425109285251092862510924B
:10A7E000C4281092C32897FF04C082E08093C80059
:10A7F0003F773093CD002093CC0088E98093C90047
:10A8000086E08093CA0008958330D1F0843028F424
:10A81000813081F0823088F407C08530C9F08530FE
:10A8200090F08630C9F403C087E092E00EC083E068
:10A8300091E00BC081E890E008C080E490E005C0A2
:10A840008FE190E002C084E190E00E94E653089519
:10A850008AE090E00E94E6530895909185258091CA
:10A860008625981719F420E031E011C0E091862583
:10A87000EF5FE0938625F0E0ED57FE4D30812091AB
:10A880008725922F80E0AC01430F511D9A01C90129
:10A890000895482F909183259F5F9F738091842511
:10A8A0009817E1F3E92FF0E0ED5BFE4D40839093C4
:10A8B00083258091C90080628093C900809187259B
:10A8C000382F20E0240F311DC9010895CF93DF9365
:10A8D000EC0103C021960E94495488818823D1F756
:10A8E000DF91CF910895CF93DF93EC0102C00E94D6
:10A8F0004954FE01219684918823C9F7DF91CF91B5
:10A900000895809185252091862590E081509C4F67
:10A91000821B91096FEF73E00E9435DA08958091F0
:10A920008625809385250895CF93DF93EC01FB0165
:10A930009A013197E80FF91F1082C9016AE070E0AF
:10A940000E9421DA805D8293C9016AE070E00E9472
:10A9500021DA9B016115710519F0CE17DF0768F345
:10A96000CF01DF91CF9108952091D5253091D62543
:10A970008091D7259091D8252817390711F4E0E068
:10A980001BC0E091D725F091D825E0818091D72593
:10A990009091D82501969093D8258093D7258091C2
:10A9A000D7259091D825855D954231F485E995E2CA
:10A9B0009093D8258093D7258E2F0895DC01209180
:10A9C000D5253091D6258091D7259091D825281767
:10A9D000390711F480E00895E091D725F091D8254A
:10A9E00080818C938091D7259091D8250196909362
:10A9F000D8258093D7258091D7259091D825855D3E
:10AA0000954211F081E0089585E995E29093D8256B
:10AA10008093D72581E008959093C5008093C4006A
:10AA20008091C0008D7F8093C00086E08093C2003B
:10AA30008091C1008B7F8093C10002C08091C600CD
:10AA40008091C00087FDFACF8091C100886180931A
:10AA5000C1008091C10080688093C10085E995E2C2
:10AA60009093D8258093D7258091D7259091D8258C
:10AA70009093D6258093D52508958330D1F08430E6
:10AA800028F4813081F0823088F407C08530C9F025
:10AA9000853090F08630C9F403C087E092E00EC0A4
:10AAA00083E091E00BC081E890E008C080E490E092
:10AAB00005C08FE190E002C084E190E00E940C5557
:10AAC00008958AE090E00E940C550895E1ECF0E0D2
:10AAD0008081877F808323982B980895239A2B98D1
:10AAE000E1ECF0E08081886080830895982F809168
:10AAF000C00085FFFCCF9093C6000895FC0107C0FD
:10AB00008091C00085FFFCCF9093C6003196908164
:10AB10009923B1F70895FC0107C08091C00085FF1B
:10AB2000FCCF9093C600319694919923B1F7089584
:10AB300050918925565033E043E048C0E32FF0E0C0
:10AB4000EB53F74D80813F5FE32FF0E0EB53F74D80
:10AB500020812D533F5FE32FF0E0EB53F74D7081E1
:10AB60003F5FE32FF0E03350EB53F74D6081E42F6C
:10AB7000F0E0922F92959F708D53880F880F892B4C
:10AB8000EB53F74D8083E42FEF5F513081F0972F27
:10AB90009D53F0E02295207F892F86958695282B5E
:10ABA000EB53F74D2083E42FEE5F523011F44E2F1C
:10ABB00010C03C5F5350F0E09295990F990F907C34
:10ABC0006D53962BEB53F74D90834D5F552309F052
:10ABD000B5CF88EC98E290938B2580938A254350DB
:10ABE00040938C25089580912E21813071F58091BC
:10ABF000C00085FFFCCF8BE18093C6008091C00030
:10AC000085FFFCCF8BE18093C6008091C00085FF5B
:10AC1000FCCF85E58093C6008091C00085FFFCCF06
:10AC20008AEA8093C6008091C00085FFFCCF109215
:10AC3000C60081E080932F2184EF91E024EF31E082
:10AC4000F9013197F1F70197D9F7089585E08093DD
:10AC50002F2184EF91E024EF31E0F9013197F1F7F2
:10AC60000197D9F70895A0E0B0E0E9E3F6E50C9488
:10AC700090DA8B857C8593E2909398298F59809305
:10AC800099298A8580939A29DE011D96772329F4D4
:10AC9000EE24FF2440E050E007C0ED84FE84DE0196
:10ACA00051964F855889715030E003E010E07DC027
:10ACB000F701E30FF11D90813F5F4150504091F447
:10ACC000772309F4BFC0FD013296ED90FC90DF01BF
:10ACD00012960190F081E02D7150309709F4B1C0C7
:10ACE000AF0130E0F701E30FF11DD0803F5F41502D
:10ACF000504091F4772369F0FD013296ED90FC907D
:10AD0000DF0112964081518171504115510519F4AE
:10AD100030E060E015C030E0F701E30FF11D608125
:10AD20003F5F4150504061F4772351F0FD0132966E
:10AD3000ED90FC90DF01129640815181715030E01E
:10AD4000892F86958695835CF801E856F64D8083B9
:10AD50002D2D22952F70892F90E083709070F4E054
:10AD6000880F991FFA95E1F7282B235CF801E75625
:10AD7000F64D20838D2D90E08F709070880F991F75
:10AD8000880F991F262F2295269526952370282B0C
:10AD9000235CF801E656F64D20836F73635CF8017F
:10ADA000E556F64D60830C5F1F4F4115510509F0C4
:10ADB0007FCF20E030E090E006C0E856F64D80817D
:10ADC000280F311D9F5FE92FF0E0E017F107A8F38E
:10ADD0003F70C90136E0969587953A95E1F7835C17
:10ADE000F801E856F64D8083C80101962F73235C65
:10ADF000FC01E856F64D20830196FC01E856F64D1D
:10AE00002DE02083AC014F5F5F4F10929C1F20E02C
:10AE10000CC08091C00085FFFCCFE22FF0E0E85627
:10AE2000F64D80818093C6002F5F822F90E08417BB
:10AE3000950778F381E080939C1F2096E7E00C94BF
:10AE4000ACDA30E060E0DD247BCFA1E0B0E0EBE203
:10AE5000F7E50C9495DA20912F212130A9F592E0A5
:10AE600099834DB75EB7475050400FB6F8945EBF18
:10AE70000FBE4DBFEDB7FEB7319685E7ADB7BEB794
:10AE800011968C9391832283CE01019694838383C0
:10AE900081E090E0968385830E94335684E080931E
:10AEA0002F2124EF31E04DB75EB7495F5F4F0FB6FA
:10AEB000F8945EBF0FBE4DBF44EF51E0CA01019749
:10AEC000F1F721503040D1F72196E2E00C94B1DA4D
:10AED000A1E0B0E0EEE6F7E50C9495DA90912F2131
:10AEE0009130A1F599832DB73EB7275030400FB66A
:10AEF000F8943EBF0FBE2DBFEDB7FEB7319685E784
:10AF0000ADB7BEB711968C9382E081839283CE0158
:10AF100001969483838381E090E0968385830E94E9
:10AF2000335683E080932F2124EF31E08DB79EB715
:10AF300007960FB6F8949EBF0FBE8DBF44EF51E049
:10AF4000CA010197F1F721503040D1F72196E2E094
:10AF50000C94B1DAA1E0B0E0E0EBF7E50C9494DA00
:10AF600090912F21913099F519822DB73EB7275036
:10AF700030400FB6F8943EBF0FBE2DBFEDB7FEB701
:10AF8000319685E7ADB7BEB711968C9312E0118369
:10AF90009283CE0101969483838381E090E096832F
:10AFA00085830E94335610932F2124EF31E08DB713
:10AFB0009EB707960FB6F8949EBF0FBE8DBF44EFA5
:10AFC00051E0CA010197F1F721503040D1F72196A5
:10AFD000E3E00C94B0DAA1E0B0E0E1EFF7E50C9427
:10AFE00092DA082FF62E142F0E946E55812F6AE0F8
:10AFF0000E9415DA89838DB79EB707970FB6F8942C
:10B000009EBF0FBE8DBFEDB7FEB73196ADB7BEB7D1
:10B0100011960C93F18281E08283CE010196948394
:10B02000838381E090E0968385830E9433568DB7B9
:10B030009EB707960FB6F8949EBF0FBE8DBF809146
:10B040009C1F8823E1F30E9466552196E5E00C944D
:10B05000AEDA1F920F920FB60F920BB60F92112419
:10B060001F932F933F934F935F936F937F938F9390
:10B070009F93AF93BF93CF93DF93EF93FF93809111
:10B080002F21853011F0843089F54091C600209140
:10B09000D5253091D6258091D7259091D825281B8C
:10B0A000390B37FF02C0205C3F4F2F3331050CF0C6
:10B0B000B5C0E091D525F091D62540838091D52566
:10B0C0009091D62501969093D6258093D525809191
:10B0D000D5259091D625855D954209F09FC085E9DB
:10B0E00095E29093D6258093D52598C01091C600FF
:10B0F00080916F2C882339F08091E032882319F0F9
:10B10000812F0E94495480918825882309F086C0A8
:10B1100060919225662371F4133279F41093C52857
:10B1200081E08093922583E290E090939425809330
:10B13000932574C0643B08F064C0A62FB0E0209152
:10B140009325309194251D3069F0AB53B74D1C9376
:10B150006F5F60939225210F311D309394252093CA
:10B1600093255CC0FD01ED53F74D9081ED01CC536B
:10B17000D74D8881A901491B5109481B51095F70AE
:10B1800050939425409393252081CA0136E09695EB
:10B1900087953A95E1F7835C821729F59881842F8A
:10B1A0008F73835C8917F9F4AB53B74D1C936F5FB2
:10B1B0006093892590912D218091C7289817F1F4EB
:10B1C00081E0809388258091C7288235B9F42CE0EE
:10B1D00088E190E00FB6F894A895809360000FBEC8
:10B1E000209360000BC080918D2590918E25019653
:10B1F00090938E2580938D2510928825109292250C
:10B200000DC080918F259091902501969093902567
:10B2100080938F251092922510928825FF91EF91AF
:10B22000DF91CF91BF91AF919F918F917F916F915E
:10B230005F914F913F912F911F910F900BBE0F90F7
:10B240000FBE0F901F901895A0E0B0E0EAE2F9E57C
:10B250000C948DDA5B016C01C0E0D0E800E010E8EE
:10B260009FE0E92EF12C169507959E0140E050E0F5
:10B27000CA01B9010E94F6D9A616B706C806D906B2
:10B2800018F4C01BD10B02C0C00FD11F0894E108F5
:10B29000F108E114F10439F79E0140E050E0CA01E1
:10B2A000B9010E94F6D9A616B706C806D90608F451
:10B2B0002197CE01CDB7DEB7EAE00C94A9DA2AE5F2
:10B2C00030E0281B390B37FD02C041E004C0309547
:10B2D00021953F4F4FEFC90168E671E00E9435DAD2
:10B2E000FC018B3591055CF08B5590408A359105BA
:10B2F00040F484EB90E09C012E1B3F0BF90181E0B0
:10B3000010C0CF01855B90408A35910518F4E45B4D
:10B31000F04006C088E691E09C012E1B3F0BF9012E
:10B320008FEF8402C0011124EE0FFF1FE356F04E91
:10B3300020813181A901849F9001859F300D949FC8
:10B34000300D1124C9010895AAE0B0E0EAEAF9E558
:10B350000C9485DA69837A838B839C8319012A0193
:10B3600029813A8137FF03C0309521953F4FB901BC
:10B37000882777FD8095982F0E94EFD65B016C019E
:10B3800020E030E040E050E00E944DD6882341F4B8
:10B3900057FC03C060E070E0DAC064EB70E0D7C037
:10B3A000910137FE03C0309521953F4FB9018827A1
:10B3B00077FD8095982F0E94EFD67B018C01A60126
:10B3C00095010E944DD688238CF4C801B701A601CF
:10B3D00095010E9454D60F2EF0E0EF2EF0E0FF2EE4
:10B3E000F0E80F2FFFE31F2FF02D0CC0C601B501B1
:10B3F000A80197010E9454D67B018C0160E070E0A7
:10B4000080E89FE320E038ED4BED56E40E94DCD766
:10B410000E94BCD63B014C01C801B70120E038EDC9
:10B420004BED56E40E94DCD70E94BCD69B01AC01D8
:10B430000CE817E31E830D83EE24FF24870160E0F0
:10B4400070E064015301062E04C0D694C794B794EB
:10B45000A7940A94D2F7AF82B886C986DA865901D2
:10B460006A01062E04C0D594C794B794A7940A9491
:10B47000D2F757FF17C06A187B088C089D088F8188
:10B480009885A985BA85280F391F4A1F5B1FED8152
:10B49000FE8185919491A0E0B0E0E81AF90A0A0BC8
:10B4A0001B0B16C06A0C7B1C8C1C9D1CAF80B884C7
:10B4B000C984DA842A193B094C095D09ED81FE81B2
:10B4C00085919491A0E0B0E0E80EF91E0A1F1B1FC1
:10B4D0006F5F7F4F8D819E8102969E838D836F303B
:10B4E000710509F0AECFC801B7010E94EDD621EE7B
:10B4F0003EE245E652E40E94DCD720E038ED4BED19
:10B5000056E40E9454D60E94C1D69B01AC0112148D
:10B5100013041404150464F084EB90E0A0E0B0E0A0
:10B520005C016D01A21AB30AC40AD50AA6019501ED
:10B53000C980DA80EB80FC801C141D041E041F04EB
:10B540002CF066277727621B730B01C0B901CB0172
:10B550002A96E2E10C94A1DA0895EF92FF920F93FC
:10B560001F93E82E80916F008D7F80936F008091F4
:10B570000033882309F059C0809181008C7F80932B
:10B5800081008091810084608093810080E18093BC
:10B590004C2A80E28093582A1092652A1092642ADD
:10B5A000E0910033FF2400E010E0F0E083E0EE0FD4
:10B5B000FF1F8A95E1F7ED5AFF4D2681378140E064
:10B5C00050E060E07DE281E391E00E9448DAC8014A
:10B5D000B7010E94F6D90E94EDD62FE632E143E88A
:10B5E0005AE30E94DCD70E94C1D6AB017093672A50
:10B5F0006093662A3091880020918900922F80E024
:10B60000830F911D840F951F90938900809388006C
:10B6100080916F00826080936F0081E080937C2A2C
:10B620001F910F91FF90EF900895809181008B7F83
:10B6300080938100809181008360A6CFE0910033E8
:10B64000F0E023E0EE0FFF1F2A95E1F7ED5AFF4DE2
:10B6500026813781829FB001839F700D929F700D6C
:10B66000112480E090E00E94EDD620E030E040EA36
:10B6700051E40E9454D620E030E040E05FE30E94B5
:10B68000E9D50E94C1D6CB010895E0910033F0E0E6
:10B6900033E0EE0FFF1F3A95E1F7E95AFF4D808145
:10B6A0009181089590E0FC01EE0FFF1FE80FF91F54
:10B6B000EE0FFF1FEE0FFF1FE45BF54D617063831C
:10B6C0000895E091003390E0DC01AA0FBB1FA80FA2
:10B6D000B91FAA0FBB1FAA0FBB1FA05BB54DF0E09F
:10B6E00083E0EE0FFF1F8A95E1F7EB5AFF4D808153
:10B6F0009181860F971F8D939C930895E09100335D
:10B7000090E0DC01AA0FBB1FA80FB91FAA0FBB1F37
:10B71000AA0FBB1FA45BB54DF0E033E0EE0FFF1F97
:10B720003A95E1F7ED5AFF4D80819181861B970B89
:10B7300017969C938E931697089590E0ECE4FAE2A6
:10B740009C01220F331F280F391FD901AA0FBB1FDD
:10B75000AA0FBB1FAE0FBF1F1B967C936E931A9749
:10B760002F5F3F4F220F331F220F331FE20FF31FB4
:10B7700040815181E0910033F0E083E0EE0FFF1F44
:10B780008A95E1F7E95AFF4D8081918190958195E5
:10B790009F4F841B950B16962D913C911797820F06
:10B7A000931F660F771F860F971F73E0880F991FEF
:10B7B0007A95E1F764E0969587956A95E1F7840FAD
:10B7C000951F19969C938E9318970895EFE6F0E0D5
:10B7D00080818D7F80830895482F50E0FA01EE0F1D
:10B7E000FF1FE40FF51FEE0FFF1FEE0FFF1FE05BC3
:10B7F000F54D0190F081E02DCB016E177F0708F425
:10B80000CF01FA01EE0FFF1FE40FF51FEE0FFF1F30
:10B81000EE0FFF1FE45BF54D2681378128173907AE
:10B8200008F4C901928381830895FF920F931F93B7
:10B83000CF93DF93AB01C82FD0E0FE01EE0FFF1FC7
:10B84000EC0FFD1FEE0FFF1FEE0FFF1FE45BF54D2A
:10B850008381882381F0E0910033F0E073E0EE0F04
:10B86000FF1F7A95E1F7E95AFF4D808191819C0194
:10B87000241B350BA901E0910033F0E063E0EE0FEB
:10B88000FF1F6A95E1F7E95AFF4D808191819695F6
:10B890008795FE01EE0FFF1F4817590770F5EC0F53
:10B8A000FD1FEE0FFF1FEE0FFF1FDF01A05BB54D69
:10B8B0000D911C91F0900033E45BF54D608571852E
:10B8C000601B710B80E090E0660F771F881F991F47
:10B8D0009A0140E050E00E94F6D9EF2DF0E0A3E09D
:10B8E000EE0FFF1FAA95E1F7E95AFF4D2081318144
:10B8F00040E050E00E946ADA3AC0A0910033EC0FB9
:10B90000FD1FEE0FFF1FEE0FFF1FE45BF54D0085DF
:10B910001185F090003366817781601B710B80E0A8
:10B9200090E0660F771F881F991FB0E023E0AA0FF1
:10B93000BB1F2A95E1F7A95ABF4D2D913C91369531
:10B940002795421B530B9A0140E050E00E94F6D924
:10B95000EF2DF0E0A3E0EE0FFF1FAA95E1F7E95A03
:10B96000FF4D2081318140E050E00E9448DAC8015B
:10B97000820F931FFE01EE0FFF1FEC0FFD1FEE0F56
:10B98000FF1FEE0FFF1FE05BF54D0190F081E02DF2
:10B990008E179F0708F4CF01FE01EE0FFF1FEC0F7B
:10B9A000FD1FEE0FFF1FEE0FFF1FE45BF54D26811D
:10B9B00037812817390708F4C90192838183CDB7ED
:10B9C000DEB7E5E00C94AEDA0F931F93E0910033FD
:10B9D000F0E033E0EE0FFF1F3A95E1F703E510E2E8
:10B9E000E00FF11F6481758180E00E94155C8091F9
:10B9F000003390E023E0880F991F2A95E1F7080FA4
:10BA0000191FF8016481758181E00E94155C1F9106
:10BA10000F9108951F93182FE0910033882777FD29
:10BA20008095982FF0E043E0EE0FFF1F4A95E1F775
:10BA3000E95AFF4D2081318140E050E00E94F6D963
:10BA400024EB30E040E050E00E9448DA812FB90159
:10BA50000E94155C1F9108951F920F920FB60F92CE
:10BA60000BB60F9211242F933F934F935F938F93B5
:10BA70009F93EF93FF933091D925323090F42BB1FF
:10BA8000832F90E0FC01EE0FFF1FE80FF91FEE0F70
:10BA9000FF1FEE0FFF1FE45BF54D80818095822331
:10BAA0008BB9832F8F5F8093D9258230C9F0833083
:10BAB00010F01092D9252BB18091D92590E0FC018E
:10BAC000EE0FFF1FE80FF91FEE0FFF1FEE0FFF1F16
:10BAD000E45BF54D8081282B2BB9418152810AC04E
:10BAE0004091662A5091672A8091642A9091652A34
:10BAF000481B590B3091880020918900922F80E0DB
:10BB0000830F911D840F951F909389008093880067
:10BB10008091642A9091652A840F951F9093652ADD
:10BB20008093642A2091662A3091672A82179307AE
:10BB300020F01092652A1092642AFF91EF919F9154
:10BB40008F915F914F913F912F910F900BBE0F906E
:10BB50000FBE0F901F90189597FF03C0261B370B41
:10BB600004C0CA01821B930B9C01C9010895A82F30
:10BB7000B0E0A330B10514F080E001C08F5FA95799
:10BB8000BF4DAC91B0E0AA0FBB1FA60FB71FE82FA7
:10BB9000F0E0E957FF4DE081F0E0EE0FFF1FE60F08
:10BBA000F71F2D913C91808191818217930714F4A6
:10BBB0008FEF089581E00895892B29F480E162E0F8
:10BBC0004BE850E204C080E162E040E950E220E04E
:10BBD0000E94ACBB08950E9483B78091682A882395
:10BBE00019F48DEC90E002C08EEC90E00E94903E43
:10BBF000AC0180E060E022E00E94ACBB0895892B9C
:10BC000019F48CE290E002C08BE290E00E94903E3A
:10BC1000AC0181E162E020E00E94ACBB08950F938B
:10BC20001F938C0180E062E04EE95BE320E00E941C
:10BC30007EBB012B29F48EE062E046E95BE304C0A1
:10BC40008EE062E04EE85BE320E00E947EBB1F9145
:10BC50000F9108950E94AD5A80E00895EF92FF92EF
:10BC60000F931F93CF93DF93E82EC0E0D0E0FC2E1C
:10BC7000FE0103E0EE0FFF1F0A95E1F7EE2039F514
:10BC8000EC1BFD0BED58FD4CDF01A058BF4F8D9113
:10BC90009C911197969587959695879511969C936B
:10BCA0008E93DF01AE57BF4F8D919C911197969562
:10BCB00087959695879511969C938E93EC57FF4F99
:10BCC00080819181969587959695879527C0EC1BE5
:10BCD000FD0BED58FD4CDF01A058BF4F8D919C919D
:10BCE0001197880F991F880F991F11969C938E9317
:10BCF000DF01AE57BF4F8D919C911197880F991F0F
:10BD0000880F991F11969C938E93EC57FF4F80815B
:10BD10009181880F991F880F991F039691838083C3
:10BD20008E0123E0000F111F2A95E1F70C1B1D0B5C
:10BD30000D581D4C00581F4FF801619171918F01F2
:10BD40008F2D0E94615BF801619171918F018F2DA0
:10BD50000E947E5BF801608171818F2D0E949D5B46
:10BD60002196C230D10509F082CF0E94E45CCDB7A4
:10BD7000DEB7E6E00C94ADDA0E94E45C0895EF9241
:10BD8000FF920F931F937C010E94455B96958795C8
:10BD9000B701681B790B882777FD8095982F44E0C1
:10BDA00020E000E00E946E68AC0180E162E020E0EB
:10BDB0000E94ACBB8091682AB7010E949D5B1091E4
:10BDC000682A0E94455BBC0176956795812F0E9489
:10BDD000155C1F910F91FF90EF9008950F9390E0E5
:10BDE000A0E0B0E0BC01CD0144E020E000E00E9412
:10BDF0006E68AC0180E162E020E00E94ACBB0F9174
:10BE000008950F93A0E0B0E0BC01CD0143E020E035
:10BE100000E00E946E68AC0180E162E020E00E94D8
:10BE2000ACBB0F910895009759F48CE290E00E940A
:10BE3000903EAC0181E162E020E00E94ACBB08953D
:10BE40000E94015F08950E94135F08950F93BC0143
:10BE50008A30910578F0BC0180E090E043E021E079
:10BE600001E00E946E68AC0180E162E020E00E9487
:10BE7000ACBB0CC084E690E09C01629FC001639F54
:10BE8000900D729F900D11240E94015F0F910895F3
:10BE9000CF92DF92EF920F93CF93DF936C010E94CA
:10BEA000455BEC0180E162E0A60125E030E000E0C6
:10BEB000EE240E945BC18091682AB6010E947E5BDD
:10BEC0002091682A822F90E0FC0133E0EE0FFF1FE3
:10BED0003A95E1F7E81BF90BEE50FD4C8081882381
:10BEE00011F0C0E0D0E0822FBE010E94155CDF910E
:10BEF000CF910F91EF90DF90CF900895CF92DF9286
:10BF0000EF920F936C0180E162E0A60125E030E042
:10BF100000E0EE240E9497C08091682AB6010E943A
:10BF2000615B8091682A90E0FC0143E0EE0FFF1F07
:10BF30004A95E1F7E81BF90BEE50FD4C8081882310
:10BF400019F460E070E003C00E94455BBC01809181
:10BF5000682A0E94155C0F91EF90DF90CF900895B2
:10BF60002F923F925F926F927F928F929F92AF92A9
:10BF7000BF92CF92DF92EF92FF920F931F93DF93C6
:10BF8000CF9300D000D000D0CDB7DEB7809103337F
:10BF90000E94AD5A0E9483B786ED90E00E94903EC9
:10BFA000AC0180E060E022E00E94ACBB82E090E067
:10BFB0000E94903EAC0180E067E020E00E94ACBBB4
:10BFC000809105330E94EE5E1A8219820E94455BC1
:10BFD000969587959C838B830E94455B9E838D837A
:10BFE00080E08E010F5F1F4FB8010E94B75D682E81
:10BFF000E0918720F0E0EE0FFF1FE00FF11F80803F
:10C0000091805090053377247394180197C08091E4
:10C01000682AB4010E94155CE72DF0E0E957FF4D56
:10C02000E081F0E0EE0FFF1FE20DF31D0190F081C3
:10C03000E02D8E169F0609F46CC080910433262DE6
:10C04000332727FD309590E0AC01249FC001259F48
:10C05000900D349F900D1124880E991E67FE04C028
:10C060008E169F0654F005C0662019F0E815F905F4
:10C0700024F080910433882309F44F012091033385
:10C080006091073370E0620F711D6F5F7F4F8827EB
:10C0900077FD8095982F0E94EFD65B016C0120E020
:10C0A00030E44CE955E40E94DCD77B018C0120E0B0
:10C0B00030E040E85FE30E944DD688231CF461E045
:10C0C00070E023C0C801B70120E03FEF4FE757E41D
:10C0D0000E94D8D71816ACF4C601B50120E030E0B4
:10C0E00040E251E40E94DCD70E94C1D606C084EF32
:10C0F00091E00197F1F76150704061157105B9F752
:10C100001DC0C801B7010E94C1D6CB010197F1F74C
:10C1100015C0872DB1010E94B75D682E52E05715FA
:10C1200010F4772407C0772021F45A94852D0E94BB
:10C13000EE5E7394809106330E94A56980E10E94AF
:10C140000573882331F480E20E940573882309F483
:10C150005ECFF89484E10E94AD5A78940E94E45C2A
:10C1600026960FB6F894DEBF0FBECDBFCF91DF91FC
:10C170001F910F91FF90EF90DF90CF90BF90AF9005
:10C180009F908F907F906F905F903F902F90089539
:10C19000CF92DF92EF92FF920F93CF93DF93EC0158
:10C1A0008091682ABE010E94EC5B8091003390E090
:10C1B000FC01EE0FFF1FE80FF91FEE0FFF1FE55800
:10C1C000FF4D848195816E01C81AD90A8091003390
:10C1D00090E0FC01EE0FFF1FE80FF91FEE0FFF1FAD
:10C1E000E558FF4D608171818091003390E0FC0142
:10C1F000EE0FFF1FE80FF91FEE0FFF1FE358FF4D73
:10C20000408151818091003390E0FC01EE0FFF1FCF
:10C21000E80FF91FEE0FFF1FE558FF4D2481358110
:10C22000D7FE04C07901E61AF70A03C07A01E21AC0
:10C23000F30ACE010E941E5B23E0883E920718F4A9
:10C240000E94015F0EC0BC0180E090E045E023E069
:10C2500003E00E946E68AC018EE062E020E00E9484
:10C26000ACBBB601882777FD8095982F28EE33E088
:10C2700040E050E00E94F6D99701442737FD4095F1
:10C28000542F0E946ADAB901882777FD8095982F8C
:10C2900046E021E001E00E946E68AC018EE062E0C1
:10C2A00020E00E94ACBBDF91CF910F91FF90EF9007
:10C2B000DF90CF900895A0E0B0E0E1E6F1E60C94C5
:10C2C0008FDAEC018B016A0180E40E9405738823F8
:10C2D00031F480E463E00E945E73882361F0CC1542
:10C2E000DD0510F0E80104C081E080934A26219624
:10C2F000CE01F701099580E80E940573882331F487
:10C3000080E863E00E945E73882361F00C171D07CC
:10C3100010F0E60104C0219781E080934A26CE0107
:10C32000F7010995CE01CDB7DEB7E8E00C94ABDAA2
:10C330006F927F928F929F92AF92BF92CF92DF9235
:10C34000EF92FF920F93CF93DF93EC013B014A01F1
:10C350005901C880D980C601F90109950BC08881AF
:10C360009981B301A40120E102E075010E945B61A3
:10C370009983888380E10E940573882329F480E2F1
:10C380000E940573882359F3888199818C159D0536
:10C3900019F410924A2603C081E080934A2620E0D7
:10C3A00088819981C816D90609F021E0822FDF9192
:10C3B000CF910F91FF90EF90DF90CF90BF90AF9013
:10C3C0009F908F907F906F900895A2E0B0E0EBEE89
:10C3D000F1E60C9495DA0E9483B78CEC90E00E9411
:10C3E000903EAC0180E060E022E00E94ACBB8CECAF
:10C3F00090E00E94903EAC0180E062E020E00E946C
:10C40000ACBB82E090E00E94903EAC0180E067E02F
:10C4100020E00E94ACBB8091003389831A82CE0158
:10C42000019660E070E041E050E02CED3DE50E94B7
:10C430009861882361F0F89489818093003380911A
:10C4400000330E942E5E84E10E94AD5A78942296B9
:10C45000E2E00C94B1DAA2E0B0E0E1E3F2E60C94A1
:10C4600094DA82ED90E00E94903EAC0180E062E0C0
:10C4700020E00E94ACBB82E090E00E94903EAC01C4
:10C4800080E067E020E00E94ACBB84E10E94AD5AEE
:10C490001091682A0E94455BBC0176956795812FB3
:10C4A0000E94155C8091682A90E0FC0143E0EE0F49
:10C4B000FF1F4A95E1F7E81BF90BE950FD4C80811D
:10C4C00091819A838983809100332091003390E099
:10C4D000FC01EE0FFF1FE80FF91FEE0FFF1FEE0F1D
:10C4E000FF1FED59FF4D6085718530E0F901EE0FBA
:10C4F000FF1FE20FF31FEE0FFF1FEE0FFF1FED599F
:10C50000FF4D42855385CE0101962FEB3EE50E94FB
:10C510009861882389F08091682A90E029813A8186
:10C52000FC0173E0EE0FFF1F7A95E1F7E81BF90BB2
:10C53000E950FD4C318320830E94E45C2296E3E0C5
:10C540000C94B0DA0E94EB5D0E942B620895A2E089
:10C55000B0E0EDEAF2E60C9495DA81ED90E00E940D
:10C56000903EAC0180E062E020E00E94ACBB82E043
:10C5700090E00E94903EAC0180E067E020E00E94E5
:10C58000ACBB84E10E94AD5A8091682A60E070E003
:10C590000E94155C8091682A90E0FC0143E0EE0F58
:10C5A000FF1F4A95E1F7E81BF90BED50FD4C808128
:10C5B00091819A838983809100332091003390E0A8
:10C5C000FC01EE0FFF1FE80FF91FEE0FFF1FEE0F2C
:10C5D000FF1FED59FF4D6081718130E0F901EE0FD1
:10C5E000FF1FE20FF31FEE0FFF1FEE0FFF1FEB59B0
:10C5F000FF4D40815181CE0101962EE73FE50E941B
:10C6000098618823C9F08091682A282F30E04981F9
:10C610005A81F90163E0EE0FFF1F6A95E1F7E21B13
:10C62000F30BED58FD4CE058FF4F51834083349697
:10C63000608171810E949D5B0E94E45C2296E2E031
:10C640000C94B1DA0E94EB5D0E94A7620895A2E00B
:10C65000B0E0EDE2F3E60C9494DA80ED90E00E9415
:10C66000903EAC0180E062E020E00E94ACBB82E042
:10C6700090E00E94903EAC0180E067E020E00E94E4
:10C68000ACBB84E10E94AD5A1091682A0E94455BC0
:10C69000BC01812F0E94155C8091682A90E0FC010A
:10C6A00043E0EE0FFF1F4A95E1F7E81BF90BEB5053
:10C6B000FD4C808191819A83898380910033209100
:10C6C000003390E0FC01EE0FFF1FE80FF91FEE0FA3
:10C6D000FF1FEE0FFF1FE959FF4D6081718130E0B0
:10C6E000F901EE0FFF1FE20FF31FEE0FFF1FEE0F1A
:10C6F000FF1FED59FF4D46815781CE01019628E479
:10C700003FE50E9498618823C9F08091682A282F0C
:10C7100030E049815A81F90163E0EE0FFF1F6A950D
:10C72000E1F7E21BF30BED58FD4CEE57FF4F518341
:10C7300040833296608171810E949D5B0E94E45C1F
:10C740002296E3E00C94B0DA0E94EB5D0E9427632E
:10C750000895A2E0B0E0EFEAF3E60C9495DA8FECEE
:10C7600090E00E94903EAC0180E062E020E00E94F8
:10C77000ACBB82E090E00E94903EAC0180E067E0BC
:10C7800020E00E94ACBB84E10E94AD5A8091682AEF
:10C7900090E0FC0163E0EE0FFF1F6A95E1F7E81BF4
:10C7A000F90BEE50FD4C808189831A82CE010196EF
:10C7B00060E070E041E050E02FEF3DE50E949861BD
:10C7C000882391F08091682A282F30E06981F9014F
:10C7D00053E0EE0FFF1F5A95E1F7E21BF30BEE500B
:10C7E000FD4C60830E94525B0E94E45C2296E2E072
:10C7F0000C94B1DA0E94EB5D0E94A9630895A0E059
:10C80000B0E0E5E0F4E60C9488DA8093682A8823A7
:10C8100019F092E3892E02C081E3882EEE24992438
:10C82000FF24F39402E1502E16E3612E712C01C017
:10C83000F42E0E9483B780E060E045E55BE322E0F0
:10C840000E940ABC82E160E0482D22E00E94B5BB54
:10C8500081E090E00E94903EAC0180E067E020E043
:10C860000E94ACBBEE2039F081E061E043E55BE380
:10C8700020E00E947EBBAE2CBB24A69C8001A79C1E
:10C88000100DB69C100D1124C0E0D0E06E01CA0C52
:10C89000DB1C84E0C816D10484F440917632CE01CA
:10C8A0008F5F682F459DA0011124400F511F4659ED
:10C8B000554C83E020E00E947EBBC53059F493E0E4
:10C8C000C916D1043CF481E066E041E55BE320E079
:10C8D0000E947EBB21960A5C1F4FC630D105B1F67F
:10C8E000992069F4EE2029F481E064E04F2D20E0E6
:10C8F0000AC082E065E04F2D21E001E005C082E042
:10C9000066E04F2D21E000E00E94553B482F8E3F0E
:10C9100031F4E39499249394B5E0FB2EA3CF8D3F9B
:10C9200029F4EA949924A2E0FA2E9CCF8F3F39F49F
:10C9300080914A26813001F510924A261DC081302F
:10C9400029F40E94FA63FF24F39473CF823029F410
:10C950000E94A463F2E0FF2E6CCF833029F40E9482
:10C960002263E3E0FE2E65CF843009F061CF0E94A0
:10C97000A26274E0F72E5DCFCDB7DEB7EFE00C9486
:10C98000A4DAA2E0B0E0E7ECF4E60C9495DA0E94B9
:10C9900083B78AED90E00E94903EAC0180E060E0B9
:10C9A00022E00E94ACBB82E090E00E94903EAC018D
:10C9B00080E067E020E00E94ACBB80910733898370
:10C9C0001A82CE01019660E070E048EC50E023E26C
:10C9D0003FE50E949861882319F08981809307338D
:10C9E0002296E2E00C94B1DAA2E0B0E0EAEFF4E6DD
:10C9F0000C9495DA0E9483B789ED90E00E94903EF6
:10CA0000AC0180E060E022E00E94ACBB82E090E0FC
:10CA10000E94903EAC0180E067E020E00E94ACBB49
:10CA20008091063389831A82CE01019664E070E01A
:10CA300044E150E026E23FE50E949861882319F026
:10CA40008981809306332296E2E00C94B1DAA2E069
:10CA5000B0E0EDE2F5E60C9495DA80910533898338
:10CA60001A820E9483B788ED90E00E94903EAC014C
:10CA700080E060E022E00E94ACBB82E090E00E9497
:10CA8000903EAC0180E067E020E00E94ACBBCE01AC
:10CA9000019661E070E044E650E021E03FE50E944D
:10CAA0009861882319F08981809305332296E2E00A
:10CAB0000C94B1DAA2E0B0E0E0E6F5E60C9495DA89
:10CAC0000E9483B78091043389831A8287ED90E0B6
:10CAD0000E94903EAC0180E060E022E00E94ACBB8E
:10CAE00082E090E00E94903EAC0180E067E020E0B0
:10CAF0000E94ACBBCE01019660E070E044E150E0E2
:10CB000023E13FE50E949861882319F08981809391
:10CB100004332296E2E00C94B1DAA0E0B0E0E3E95D
:10CB2000F5E60C9489DAEE249924FF24F394F6E3D5
:10CB30006F2E712CE2E18E2E01C0F02E0E9483B781
:10CB400080E060E048E65BE322E00E940ABC81E00E
:10CB500090E00E94903EAC0180E067E020E00E94FF
:10CB6000ACBBEE2039F081E061E046E65BE320E01B
:10CB70000E947EBBAE2CBB24A69C8001A79C100DFE
:10CB8000B69C100D1124C0E0D0E06E01CA0CDB1C75
:10CB900085E0C816D10484F440917632CE018F5FCF
:10CBA000682F489DA0011124400F511F445A564C34
:10CBB00083E020E00E947EBBC53059F494E0C916A2
:10CBC000D1043CF481E066E044E65BE320E00E94AF
:10CBD0007EBB21960A5C1F4FC630D105B1F6992065
:10CBE00069F4EE2029F481E065E04F2D20E00AC0D1
:10CBF00082E065E04F2D21E001E005C082E066E0C3
:10CC00004F2D21E000E00E94553B082F8E3F31F46C
:10CC1000E3949924939475E0F72EA3CF8D3F29F4E4
:10CC2000EA94992462E0F62E9CCF8F3F39F48091EC
:10CC30004A26813029F510924A2622C0813019F403
:10CC40000E94B05F7ACF823029F40E945A6552E088
:10CC5000F52E74CF833029F40E94276543E0F42E2B
:10CC60006DCF843029F40E94F46434E0F32E66CF53
:10CC7000853009F062CF0E94C16425E0F22E5ECFBC
:10CC8000CDB7DEB7EEE00C94A5DAA2E0B0E0EBE4BD
:10CC9000F6E60C9495DA0E9483B783ED90E00E944B
:10CCA000903EAC0180E060E022E00E94ACBB82E0FC
:10CCB00090E00E94903EAC0180E067E020E00E949E
:10CCC000ACBB809103330E94AD5AA0E0B3E38C91DA
:10CCD00090E04BE750E2FC01EE0FFF1FE80FF91F59
:10CCE000EE0FFF1FE40FF51F848195819A838983DE
:10CCF0008C912C9190E0FC01EE0FFF1FE80FF91FC3
:10CD0000EE0FFF1FE40FF51F6081718130E0C90154
:10CD1000880F991F820F931F0196880F991F480F44
:10CD2000591FFA0140815181CE01019628EC30E66D
:10CD30000E949861F89484E10E94AD5A78940E9410
:10CD4000E45C2296E2E00C94B1DAA2E0B0E0EBEA17
:10CD5000F6E60C9495DA0E9483B784ED90E00E9489
:10CD6000903EAC0180E060E022E00E94ACBB82E03B
:10CD700090E00E94903EAC0180E067E020E00E94DD
:10CD8000ACBB8091682A89831A82CE01019660E04B
:10CD900070E041E050E02FE03EE50E94986188237A
:10CDA00019F089818093682A2296E2E00C94B1DA26
:10CDB000A2E0B0E0EEEDF6E60C9495DA0E9483B7BF
:10CDC00085ED90E00E94903EAC0180E060E022E0C2
:10CDD0000E94ACBB82E090E00E94903EAC0180E0FB
:10CDE00067E020E00E94ACBB8091033389831A8204
:10CDF000CE0101966AE070E04EE150E021E03FE5AF
:10CE00000E949861882319F08981809303332296C8
:10CE1000E2E00C94B1DAA0E0B0E0E1E1F7E60C94D6
:10CE200089DAEE249924FF24F39486E3682E712C8A
:10CE300002E1802E01C0F42E0E9483B780E060E002
:10CE40004CE75BE322E00E940ABC81E090E00E9494
:10CE5000903EAC0180E067E020E00E94ACBBEE2099
:10CE600039F081E061E04AE75BE320E00E947EBBAD
:10CE7000AE2CBB24A69C8001A79C100DB69C100D67
:10CE80001124C0E0D0E06E01CA0CDB1C84E0C8169F
:10CE9000D10484F440917632CE018F5F682F489D93
:10CEA000A0011124400F511F4C57574C83E020E044
:10CEB0000E947EBBC53059F493E0C916D1043CF4FE
:10CEC00081E066E048E75BE320E00E947EBB2196BC
:10CED0000A5C1F4FC630D105B1F6992069F4EE20E7
:10CEE00029F481E064E04F2D20E00AC082E065E093
:10CEF0004F2D21E001E005C082E066E04F2D21E0EA
:10CF000000E00E94553B482F8E3F31F4E394992472
:10CF1000939415E0F12EA3CF8D3F29F4EA94992440
:10CF2000B2E0FB2E9CCF8F3FE9F0813029F40E94C4
:10CF30004566FF24F39480CF823029F40E948D65EA
:10CF4000A2E0FA2E79CF833029F40E94A566F3E09F
:10CF5000FF2E72CF843009F06ECF0E94D866E4E0D5
:10CF6000FE2E6ACFCDB7DEB7EEE00C94A5DAA0E0D6
:10CF7000B0E0EDEBF7E60C9489DA10924A26EE2445
:10CF80009924FF24F39476E3672E712C62E1862EB8
:10CF900001C0F42E0E9483B780E060E046E45BE3CA
:10CFA00022E00E940ABC81E090E00E94903EAC0129
:10CFB00080E067E020E00E94ACBBEE2039F081E029
:10CFC00061E044E45BE320E00E947EBBAE2CBB2426
:10CFD000A69C8001A79C100DB69C100D1124C0E0EA
:10CFE000D0E06E01CA0CDB1C84E0C816D10484F4C6
:10CFF00040917632CE018F5F682F489DA0011124A9
:10D00000400F511F4455584C83E020E00E947EBBE6
:10D01000C53059F493E0C916D1043CF481E066E0D0
:10D0200042E45BE320E00E947EBB21960A5C1F4F36
:10D03000C630D105B1F6992069F4EE2029F481E0DB
:10D0400064E04F2D20E00AC082E065E04F2D21E032
:10D0500001E005C082E066E04F2D21E000E00E9483
:10D06000553B482F8E3F31F4E3949924939455E037
:10D07000F52EA3CF8D3F29F4EA94992442E0F42EB3
:10D080009CCF8F3F39F480914A26813011F5109260
:10D090004A261FC0813029F40E94E561FF24F394E1
:10D0A00079CF823031F480E00E94FF6332E0F32ECA
:10D0B00071CF833031F481E00E94FF6323E0F22ED0
:10D0C00069CF843009F065CF0E940B6794E0F92E98
:10D0D00061CFCDB7DEB7EEE00C94A5DAA0E0B0E00A
:10D0E000E4E7F8E60C9485DA6B017C01B42E122F8C
:10D0F000842E9924F401E652FA4D10820217B8F4F6
:10D10000E22FF0E0E01BF109EE0FFF1FEE0FFF1F13
:10D11000EB55F44C2591359145915491C701B601D9
:10D120000E946ADAC901DA016C017D01102FF7FC57
:10D1300002C033240AC0F094E094D094C094C11C7F
:10D14000D11CE11CF11C3324339449EA5BE321E058
:10D1500005C02F5F4C5F5F4F2A3051F0FA01859177
:10D160009591A591B491C816D906EA06FB068CF7ED
:10D1700031102F5F11112F5F022F0B1910160CF0B9
:10D180007BC0A02FBB27A7FDB095212F30E0A217B1
:10D19000B30729F0C9010196A817B90771F5A12FA6
:10D1A000B0E0AA0FBB1FAA0FBB1FCD018F55944C37
:10D1B000FC012591359145915491CA01B90112E0C4
:10D1C000660F771F881F991F1A95D1F7620F731F7B
:10D1D000841F951F6C0D7D1D8E1D9F1DFD01EB5540
:10D1E000F44C25913591459154910E946ADAC90118
:10D1F000DA016C017D0110E03FC0A217B30764F5AE
:10D20000AA0FBB1FAA0FBB1FCD018F55944CFC0169
:10D210002591359145915491CA01B901E2E0660F1B
:10D22000771F881F991FEA95D1F7620F731F841F1C
:10D23000951F6C0D7D1D8E1D9F1DFD01EB55F44C42
:10D2400025913591459154910E946ADAC901DA011C
:10D250006C017D01101B10C02B2D2150E22FFF27E8
:10D26000E7FDF095E652FA4D8AE203C08083215033
:10D27000319727FFFBCF62C02B2D2150822F99279A
:10D2800087FD9095EC01C652DA4D022FAA24BB24EB
:10D290002C01632C77240894810891088CE2282EB5
:10D2A0002FC0112349F0C401811B910928173907A8
:10D2B00019F4288210E01FC0C701B6012AE030E04F
:10D2C00040E050E00E946ADA605D6883C701B60101
:10D2D0002AE030E040E050E00E946ADAC901DA0159
:10D2E0006C017D01C114D104E104F10421F4112386
:10D2F00011F401500BC001500894A11CB11C2197DE
:10D3000092012A193B09261537055CF6332049F0AE
:10D31000E02FFF27E7FDF095E652FA4D8DE280837E
:10D320000150E02FFF27E7FDF095E652FA4D80E22D
:10D3300003C080830150319707FFFBCF8AED95E250
:10D34000CDB7DEB7E2E10C94A1DA90E044EF51E012
:10D3500009C028EE33E0FA013197F1F7215030404F
:10D36000D1F79F5F9817A8F30895A2E0B0E0EBEB28
:10D37000F9E60C948ADA5A016B01BE016F5F7F4FA8
:10D380004AE050E00E94C2DA7B018C01E981FA8117
:10D3900080818E3249F54F011AC0C801B7012AE0D9
:10D3A00030E040E050E00E94F6D97B018C01872DEF
:10D3B00090E0C097AA2797FDA095BA2FE80EF91E16
:10D3C0000A1F1B1F0894A108B108C108D108F40165
:10D3D0007180772049F00894811C911CA114B1043C
:10D3E000C104D104D1F616C0A114B104C104D10402
:10D3F00089F0F501EE0FFF1FEE0FFF1FEB55F44C08
:10D400002591359145915491C801B7010E94F6D9F3
:10D410007B018C01B701C8012296EDE00C94A6DADD
:10D42000BC0140E020E030E09AE3E42FF0E0E05679
:10D43000FF4DDB01A20FB31F8C9180834F5F213022
:10D4400011F0233031F4E42FF0E0E056FF4D9083EB
:10D450004F5F2F5F3F4F2630310539F7E42FF0E063
:10D46000E056FF4D10820895982F80538A3068F05F
:10D470008153863010F4865F0895892F8154863059
:10D4800010F080E00895892F87530895EF92FF925E
:10D490000F931F93CF93DF93809196268130E9F508
:10D4A0008091213A8823C9F100E091E002C00E2763
:10D4B0009F5F8091213A981738F4E92FF0E0E65900
:10D4C000F84CE081EA3299F7E92FF0E0EF0122967B
:10D4D0008091213A90E0C817D907FCF48AE6E82E3B
:10D4E00087E3F82EEE0EFF1EF70181810E94346A59
:10D4F000182FC659D84C88810E94346A1295107F23
:10D50000182B101751F4F701108282ED96E36BE6A9
:10D5100077E30E9458DC81E001C080E010929626FB
:10D52000CDB7DEB7E6E00C94ADDA8F929F92AF9262
:10D53000BF92CF92DF92EF92FF920F931F93FC0165
:10D540004B018281482F50E04051524080812AE0B7
:10D55000829FC00111242181820F911D805E914024
:10D560009C0173E0220F331F7A95E1F7880F991F12
:10D57000280F391F420F531F5A01CC24B7FCC09407
:10D58000DC2CCF01039646E050E060E070E00E94A2
:10D59000B5697B018C01C601B50120E836E948E98F
:10D5A00050E00E94F6D95B016C01C801B70126E08A
:10D5B00030E040E050E00E946ADA2A0D3B1D4C1D2D
:10D5C0005D1DF4018081873539F450954095309583
:10D5D00021953F4F4F4F5F4FB901CA011F910F91E6
:10D5E000FF90EF90DF90CF90BF90AF909F908F9083
:10D5F00008958F929F92AF92BF92CF92DF92EF9257
:10D60000FF920F931F93FC014B0190818AE0989F3A
:10D61000900111248181280F311D20513240590180
:10D62000CC24B7FCC094DC2CCF01029646E050E03D
:10D6300060E070E00E94B5697B018C01C601B50114
:10D6400020E836E948E950E00E94F6D95B016C0118
:10D65000C801B70126E030E040E050E00E946ADAFD
:10D660002A0D3B1D4C1D5D1DF4018081833539F46D
:10D6700050954095309521953F4F4F4F5F4FB901E1
:10D68000CA011F910F91FF90EF90DF90CF90BF9054
:10D69000AF909F908F900895AEE0B0E0E2E5FBE69A
:10D6A0000C9487DA7C012B01DC016D907D908D90CC
:10D6B0009C9013971496AD90BD90CD90DC901797E9
:10D6C000DB018D919D910D90BC91A02D8F8398874A
:10D6D000A987BA87DB0114968D919D910D90BC911D
:10D6E000A02D8B879C87AD87BE8780914D26882390
:10D6F000E1F5C601B5014AE027E007E00E946E6847
:10D70000AC0180E063E020E00E94ACBBF7016081E7
:10D710007181828193814AE027E00E946E68AC01AA
:10D720008BE063E020E00E94ACBBD20114966D91C7
:10D730007D918D919C9117974AE027E00E946E6839
:10D74000AC0180E064E020E00E94ACBBF2016081AB
:10D750007181828193814AE027E00E946E68AC016A
:10D760008BE064E020E00E94ACBB6B857C858D85FE
:10D770009E856A0D7B1D8C1D9D1D20E03DE241E3D1
:10D7800051E00E946ADADA01C9010E945F597C0106
:10D790008F819885A985BA85681A790A8A0A9B0AB1
:10D7A000C401B3012AE030E040E050E00E946ADAB0
:10D7B000CA01B9012FE435E040E050E00E94F6D9FB
:10D7C0000027F7FC0095102FA80197010E94F6D9B9
:10D7D00020E836E948E950E00E946ADA122F032F68
:10D7E000F42EE52E8B859C85AD85BE85A81AB90AD9
:10D7F000CA0ADB0AC601B50129E534E040E050E081
:10D800000E94F6D920E137E240E050E00E946ADA57
:10D81000D22EC32EB42EA52E612F702F8F2D9E2DAC
:10D820000E94A459845E9D4F68E671E00E9435DA3B
:10D830004C01612F702F8F2D9E2D212F302F4F2DBA
:10D840005E2D0E94F6D97B018C016D2D7C2D8B2DD8
:10D850009A2D2D2D3C2D4B2D5A2D0E94F6D9E60EDA
:10D86000F71E081F191FC801B7010E9424596C0137
:10D87000EE24FF2480914D268823C1F565E046E122
:10D880005DE320E00E947EBBB401882777FD809590
:10D89000982F43E020E000E00E946E68AC0185E034
:10D8A00065E020E00E94ACBB88E065E044E15DE318
:10D8B00020E00E947EBB89E065E04EE05DE320E071
:10D8C0000E947EBBC701B60143E021E001E00E9457
:10D8D0006E68AC018FE065E020E00E94ACBB84E1A3
:10D8E00065E04CE05DE320E00E947EBBC982DA8205
:10D8F000EB82FC829E828D822C2D3A814B815C8151
:10D90000682D7E8180E090E02E96E0E10C94A3DA11
:10D91000EF920F93DF93CF9300D000D000D0CDB71C
:10D92000DEB783E89AE26FE67AE20E944C6B2983C5
:10D930003A834B835C836D837E83ADE7BAE2FE015D
:10D94000319686E001900D928150E1F76091772A3F
:10D950007091782A8091792A90917A2A20918B2A45
:10D9600030918C2A40918D2A50918E2A621B730B24
:10D97000840B950B24E630E040E050E00E946ADA28
:10D98000CA01B90120917D2A30917E2A40917F2AD7
:10D990005091802A0E94A4599093982A8093972AA4
:10D9A00080917D2A90917E2AA0917F2AB091802A31
:10D9B00088329105A105B10544F0CC97A105B105C8
:10D9C0006CF58091E925882349F180918F2A909107
:10D9D000902A9093822A8093812A8091772A90912D
:10D9E000782AA091792AB0917A2A20918B2A3091B5
:10D9F0008C2A40918D2A50918E2A821B930BA40B66
:10DA0000B50B805A9F40A040B04024F41092982A51
:10DA10001092972A81E08093E92502C01092E925AF
:10DA20008091812A9091822A8E539E4F20918F2A35
:10DA30003091902A821B930B68E671E00E9435DAE0
:10DA40009C019093962A8093952A8091972A909191
:10DA5000982A97FF04C01092982A1092972A8091D2
:10DA6000972A9091982A853B910534F084EB90E0B9
:10DA70009093982A8093972A243B310594F0245B55
:10DA800030403093962A2093952A84EB90E02091A1
:10DA9000972A3091982A821B930B9093982A80930F
:10DAA000972A6091952A7091962A80E00E940A5DDB
:10DAB0006091972A7091982A81E00E940A5D809176
:10DAC0004D26882319F566E046E05DE320E00E94DC
:10DAD0007EBB4091952A5091962A86E066E023E02D
:10DAE00030E001E0EE240E945BC18BE066E040E0A4
:10DAF0005DE320E00E947EBB4091972A5091982AD6
:10DB000081E166E023E030E00E945BC126960FB61B
:10DB1000F894DEBF0FBECDBFCF91DF910F91EF9094
:10DB200008950F931F930E94466A882309F4B3C097
:10DB300082ED96E365E970E20E9443DC67E970E2FA
:10DB40000E944FDC009709F0A6C080E090E06DE9EC
:10DB500070E20E9443DC0E94106A80E090E065E978
:10DB600070E20E9443DC80E090E065E970E20E9490
:10DB700043DC8C0180E090E065E970E20E9443DCC8
:10DB8000BC01C8010E94F96A6093692A70936A2AED
:10DB900080936B2A90936C2A80E090E065E970E2B4
:10DBA0000E9443DC8C0180E090E065E970E20E9415
:10DBB00043DCBC01C8010E94956A6093912A70936E
:10DBC000922A8093932A9093942A80E090E065E9CA
:10DBD00070E20E9443DC0E94F1DB80936D2A80E0BA
:10DBE00090E065E970E20E9443DC0E94F1DB8093E3
:10DBF0006E2A80E090E065E970E20E9443DC41E03B
:10DC000050E060E070E00E94B56970939C2A6093D8
:10DC10009B2A80E090E065E970E20E9443DC41E0ED
:10DC200050E060E070E00E94B56970939E2A6093B6
:10DC30009D2A2091912A3091922A4091932A5091C5
:10DC4000942A2093832A3093842A4093852A5093E0
:10DC5000862A2091692A30916A2A40916B2A509134
:10DC60006C2A2093872A3093882A4093892A5093DC
:10DC70008A2A882777FD8095982F60938B2A709346
:10DC80008C2A80938D2A90938E2A1092902A10923B
:10DC90008F2A0E94886C1F910F910895A1E0B0E037
:10DCA000E4E5FEE60C9487DA81E080937C2A80E04C
:10DCB00061E04CEA52E320E00E94ACBB0E94D2300B
:10DCC00080918732813011F40E949BD082E161E023
:10DCD0004BEF5CE320E00E947EBB80EC92E30E946D
:10DCE000E4D2082F813051F482E161E046EF5CE339
:10DCF00020E00E947EBB0093422107C081E161E0E9
:10DD000041EF5CE322E00E947EBBD090422181E0A3
:10DD1000D81609F04FC180E062E04BED5CE322E0F1
:10DD20000E947EBB80E061E044E10E9413BC80E081
:10DD300063E049ED5CE320E00E947EBB80E064E0AC
:10DD400047ED5CE320E00E947EBB109296260E9485
:10DD5000F3558FE480932D211982ADB7BEB7179785
:10DD60000FB6F894BEBF0FBEADBFEDB7FEB731968C
:10DD700084E611968C931182D2828E010F5F1F4F21
:10DD80001483038321E0E22EF12CF682E5820E94C7
:10DD900033568AE08983EDB7FEB731968FE6ADB78B
:10DDA000BEB711968C9382E08183D2821483038361
:10DDB000F682E5820E94335688EC90E09093A32A85
:10DDC0008093A22A8CE291E09093A52A8093A42AC2
:10DDD0008DB79EB707960FB6F8949EBF0FBE8DBF46
:10DDE00098EC892E912C8AE0482EBFE65B2EA2E0AB
:10DDF0006A2E77247394F02EF1E0AF2EB12CECE272
:10DE0000CE2EE1E0DE2E0E9418CC882309F4A2C0B9
:10DE100080918825882309F482C09092A32A809259
:10DE2000A22A0E94985580918A2590918B259093E3
:10DE30009A2A8093992AAFE6BAE2FC0131968DE0E6
:10DE400001900D928150E1F70E94916D80914D26D5
:10DE50008823D9F58DE060E040EA50E222E00E949C
:10DE6000ACBB80E161E042ED5CE320E00E947EBB60
:10DE700040916E2A83E161E050E022E030E001E071
:10DE8000EE240E945BC180E061E04DEC5CE320E0A9
:10DE90000E947EBB40916D2A84E061E050E021E069
:10DEA00030E00E945BC186E061E047EC5CE320E08B
:10DEB0000E947EBB40919B2A50919C2A8BE061E09E
:10DEC00023E030E000E00E942CC010928825809171
:10DED000A42A9091A52A892B11F54982ADB7BEB726
:10DEE00017970FB6F894BEBF0FBEADBFEDB7FEB724
:10DEF000319611965C9261827282F3821483B682AB
:10DF0000A5820E943356D092A52AC092A42A8DB72A
:10DF10009EB707960FB6F8949EBF0FBE8DBF809137
:10DF2000A22A9091A32A892B29F480E00E94AFA411
:10DF30007092682680E10E940573882309F463CFFC
:10DF400080914221882309F45ECF80916826813038
:10DF500009F459CF80E061E045E10E9413BC80E004
:10DF600062E045E10E9413BC80E063E045E10E946D
:10DF700013BC80E064E045E10E9413BC80E065E0F2
:10DF800045E10E9413BC80E066E045E10E9413BCBD
:10DF900080914221882331F462E04AEB5CE320E087
:10DFA0000E947EBB80E063E04EEA5CE320E00E94DA
:10DFB0007EBB13C080E064E04AE95CE320E00E949D
:10DFC0007EBB80E065E045E85CE320E00E947EBB2C
:10DFD00080E10E9405738823D9F3109242210E94A8
:10DFE00072D2892B39F480E063E041E75CE320E002
:10DFF0000E947EBB0E94E43081E02196E0E10C9417
:10E00000A3DAA2E0B0E0E7E0F0E70C9485DADD24E3
:10E01000D394D0927C2A80E062E04BE55CE322E07E
:10E020000E947EBB80E061E044E10E9413BC0E943C
:10E03000F3558FE480932D2119828DB79EB70797F2
:10E040000FB6F8949EBF0FBE8DBFEDB7FEB73196E9
:10E0500084E6ADB7BEB711968C931182D2828E0141
:10E060000F5F1F4F1483038361E0E62EF12CF682CD
:10E07000E5820E9433568AE08983EDB7FEB7319678
:10E080008FE6ADB7BEB711968C9382E08183D282C2
:10E0900014830383F682E5820E94335688EC90E075
:10E0A0009093A32A8093A22A8CE291E09093A52AD0
:10E0B0008093A42A109268261A829924EDB7FEB79D
:10E0C00037960FB6F894FEBF0FBEEDBF5AE0252E6F
:10E0D000302E812E41E0642E712C3CE2432E31E043
:10E0E000532E80918825882309F41AC188EC90E08A
:10E0F0009093A32A8093A22A0E94985580918A2502
:10E1000090918B2590939A2A8093992A82E161E0DD
:10E1100041E00E94319B9A81913021F480E061E0DE
:10E120000E94DD940091992A10919A2A0C5B1F4F4E
:10E13000D8018C910454104087FD3FC19394B2E301
:10E140009B1609F440C1E9E19E1631F480E061E0DC
:10E1500048E45CE322E008C0F1E09F1639F480E077
:10E1600061E045E35CE320E00E947EBB10928825DD
:10E170001A82ABC00D5B1F4FD8018C910354104025
:10E1800083FF39C0F801878D90A1A1A1B2A180932E
:10E19000832A9093842AA093852AB093862A83A108
:10E1A00094A1A5A1B6A18093872A9093882AA093D1
:10E1B000892AB0938A2A87A190A5A1A5B2A58093A8
:10E1C0008B2A90938C2AA0938D2AB0938E2A86ADA9
:10E1D00097AD9093902A80938F2A10927C2A109268
:10E1E000882580E061E042E25CE320E00E947EBBA3
:10E1F000F1E0FA836AC080E061E04FE05CE320E098
:10E200000E947EBB1092882581E08A835EC0AFE6C3
:10E21000BAE2F80131968DE001900D928150E1F75C
:10E2200060918B2A70918C2A80918D2A90918E2AF0
:10E230000E94EFD65B016C01D801D3966D917C9161
:10E24000D497882777FD8095982F20EA3FE040E01B
:10E2500050E00E94F6D90E94EFD620E030E044EB77
:10E2600051E40E9454D67B018C016091772A709111
:10E27000782A8091792A90917A2A0E94EFD69B0180
:10E28000AC01C801B7010E94E9D5A60195010E9421
:10E29000E8D520E030E040EA50E40E9454D69B01EB
:10E2A000AC01C601B5010E94E9D50E94BCD66093BD
:10E2B000772A7093782A8093792A90937A2A0E94F9
:10E2C000886C10928825B1E0BA838091A42A90913D
:10E2D000A52A892B29F52982EDB7FEB737970FB606
:10E2E000F894FEBF0FBEEDBF31968FE6ADB7BEB757
:10E2F00011968C9392E0918381E0828333828482B1
:10E30000768265820E9433565092A52A4092A42AB2
:10E31000ADB7BEB717960FB6F894BEBF0FBEADBF70
:10E320008091A22A9091A32A892B31F481E00E9446
:10E33000AFA481E08093682680E10E940573882362
:10E3400029F480916826882309F4CBCE80E061E02F
:10E3500045E10E9413BC80E062E045E10E9413BCED
:10E3600080E063E045E10E9413BC80E064E045E1A9
:10E370000E9413BC80E065E045E10E9413BC80E090
:10E3800066E045E10E9413BC80916826813081F4EB
:10E3900080E062E04EEF5BE320E00E947EBB80E223
:10E3A0009EE424EF31E0F9013197F1F70197D9F7B5
:10E3B00081E02296E2E10C94A1DA80917C2A882304
:10E3C00009F0D8CE24CF9924D1CE80EF0E940573D6
:10E3D0000E9483B78091CF32882331F460E048EE09
:10E3E0005BE322E00E947EBB8091CF32813039F422
:10E3F00080E060E042ED5BE322E00E947EBB80E1D2
:10E4000067E04DEC5BE320E00E947EBB8091CF3261
:10E41000882311F40E944E6E8091CF32813011F426
:10E420000E94017080EF0E94057308951092A32A44
:10E430001092A22A82E084BD85E085BD83EC87BD71
:10E44000EEE6F0E080818260808308951F920F9253
:10E450000FB60F9211245F9A0F900FBE0F901F906E
:10E4600018951F920F920FB60F9211245F980F907C
:10E470000FBE0F901F9018958091EF328130A1F45C
:10E480001092B0001092B6001092B2008FEF8093FD
:10E49000B3008091B000836C8093B0008091B10094
:10E4A00081608093B1000895579A8091B00083688D
:10E4B0008093B0008091B10081608093B100809121
:10E4C00070008660809370008FEF8093B300089592
:10E4D000E0E9F0E0108288EF8093950010929400BC
:10E4E00087E0809399008FEF80939800808182600D
:10E4F0008083E1E9F0E0808181608083E1E7F0E002
:10E5000080818260808308951F920F920FB60F92D0
:10E510000BB60F9211242F933F934F935F938F93DA
:10E520009F93EF93FF931092950010929400809127
:10E53000CF2A882379F1579A9091E92B8091EA2B81
:10E54000890F8093E92B891728F48091E32B8F5F43
:10E550008093E32BE091F32B8091E32BE80FE09382
:10E56000E32BF0E0ED51F54D2081332727FD309569
:10E570008091E82B90E0AC01249FC001259F900D75
:10E58000349F900D1124892F990F990B80588093F7
:10E59000B30001C05798FF91EF919F918F915F91C8
:10E5A0004F913F912F910F900BBE0F900FBE0F9088
:10E5B0001F9018952091FD253091FE252F5F3F4F2C
:10E5C000280F391FC90108952091FD253091FE259E
:10E5D000821B930B80709078892F869508952091E7
:10E5E000FD253091FE252F5F3F4F280F391F809169
:10E5F000FD259091FE25A901481B590BCA01807089
:10E600009078892F869599F308952FB7F894909173
:10E61000EB25892398279093EB252FBF08954FB7BB
:10E62000F8943FB7F8942091EB259091EA259095C6
:10E630008923822328272093EB253FBF4FBF0895CE
:10E640002FB7F8949091EC25892398279093EC2587
:10E650002FBF2FB7F8949091ED2589239827909399
:10E66000ED252FBF2FB7F8949091EB25892398279C
:10E670009093EB252FBF08952FB7F8949091ED2537
:10E68000892398279093ED252FBF0895282F9FB7B2
:10E69000F8948091EE25282382278093EE259FBF52
:10E6A0003FB7F8949091ED258091EB2580958227D6
:10E6B000892398279093ED253FBF08952FB7F894AD
:10E6C0009091EF25892398279093EF256093F0256B
:10E6D0002FBF08950F931F939C018091F0328130DA
:10E6E00091F5442341F48091FB259091FC25892BE1
:10E6F00009F05BC00FC04130B1F48091FB259091CF
:10E70000FC25892B09F051C081E090E09093FC2515
:10E710008093FB253093FA252093F9257093AE2042
:10E720006093AD2042C0423009F03FC01092FC25FA
:10E730001092FB251092FA251092F9251092AE2026
:10E740001092AD2032C0442371F48091FB2590914A
:10E75000FC25892B51F5C9016AE070E00E9421DA9D
:10E7600084E893E020C04130B9F48091FB2590917A
:10E77000FC25892BD1F4C9016AE070E00E9421DAFE
:10E78000162F072F80EB94E040E00E94E07D8CE4A0
:10E7900094E0612F702F06C0423039F480E090E0A1
:10E7A00060E070E040E00E94E07D1F910F910895CD
:10E7B0008091F7259091F825019771F488EE93E008
:10E7C00060E270E040E00E946A7380E060E04CE14B
:10E7D0005DE322E00E947EBB4091F7255091F82531
:10E7E0002091A9203091AA2084E690E0BC01269FC8
:10E7F000C001279F900D369F900D1124481759078F
:10E8000021F41092F8251092F7258091F725909128
:10E81000F825892B49F08091F7259091F8250196EC
:10E820009093F8258093F725349B04C01092F62529
:10E830001092F52534991BC08091F5259091F6250D
:10E8400001969093F6258093F5258091F52590917A
:10E85000F6250A9761F48091F7259091F825892B88
:10E8600031F481E090E09093F8258093F725409172
:10E87000F5255091F6252091AB203091AC2084E60F
:10E8800090E0BC01269FC001279F900D369F900D00
:10E8900011244817590709F4299808951F920F92D7
:10E8A0000FB60F920BB60F9211242F933F934F93F5
:10E8B0005F936F937F938F939F93AF93BF93EF93E8
:10E8C000FF933091EA2520B12095232780910526DA
:10E8D0008223809580930526909104269223982781
:10E8E0009093042628232923922F93279093EA2597
:10E8F00092238091EB25892B8093EB258091FF2536
:10E9000081508093FF258F5F89F489E08093FF25F4
:10E910008091FD259091FE2501969093FE25809390
:10E92000FD258091AF208F5F8093AF20222309F1D6
:10E930008091F032813021F48091BA28813041F009
:10E940008091F0328823A9F48091BA28823089F42A
:10E950008091A12A882311F40E94A43081E0809341
:10E96000A12A1092F2251092F1251092F42510920E
:10E97000F32580917532882359F18091F0328130EE
:10E9800021F48091BA28813041F08091F0328823BF
:10E99000F9F48091BA288230D9F48091A12A81308B
:10E9A000B9F48091F1259091F22501969093F2258A
:10E9B0008093F1252091753264E670E00E9421DA9F
:10E9C00030E06217730721F40E94BE301092A12A32
:10E9D0008091F032813069F58091F9259091FA2586
:10E9E0000097D9F08B30910530F00A979093FA2573
:10E9F0008093F92504C01092FA251092F925809190
:10EA0000AD209091AE202091F9253091FA258223F6
:10EA10009323892B09F0B8C00AC08FEF9FEF909322
:10EA2000AE208093AD201092FC251092FB250E9411
:10EA300099308091AB2A9091AC2A892B51F080912A
:10EA4000AB2A9091AC2A01979093AC2A8093AB2A81
:10EA500013C01092CF2A0E94997E80919F2A909194
:10EA6000A02A892B49F080919F2A9091A02A019792
:10EA70009093A02A80939F2A4091EA25242F30E08A
:10EA8000207F30702115310519F486E48093032628
:10EA900080910326815080930326882339F4942F94
:10EAA000907F8091EC25892B8093EC2521153105F1
:10EAB00019F481E080930226809102268150809390
:10EAC0000226882351F48FE080930226942F907FB2
:10EAD0008091ED25892B8093ED252115310519F4C1
:10EAE00086E480930126809101268150809301263F
:10EAF000882351F48FE080930126942F907F80919A
:10EB0000EE25892B8093EE25232B19F486E4809340
:10EB10000026809100268150809300268823A9F446
:10EB20008091F025813011F484E107C0823011F426
:10EB300088E003C0833049F481E080930026407F61
:10EB40008091EF25842B8093EF258091A22A9091CC
:10EB5000A32A892B49F08091A22A9091A32A019798
:10EB60009093A32A8093A22A8091A42A9091A52A07
:10EB7000892B69F08091A42A9091A52A01979093FE
:10EB8000A52A8093A42A03C00E948E3052CFFF9101
:10EB9000EF91BF91AF919F918F917F916F915F9115
:10EBA0004F913F912F910F900BBE0F900FBE0F9082
:10EBB0001F901895A0E0B0E0E0EEF5E70C948CDA39
:10EBC000E0910726F0E0EE0FFF1FDF01A355B54DE2
:10EBD000CD91DC91EB53F54D0190F081E02DEC17D8
:10EBE000FD070CF044C0E639F1050CF040C026E901
:10EBF000E22EF12CB7016E1B7F0B882777FD8095E5
:10EC0000982F0E94EFD620E030E040E05FEB0E94BA
:10EC1000DCD720E030E04CE752E40E94E9D50E94C6
:10EC2000C1D65B016C01909006269394EC1AFD0A04
:10EC30000027F7FC0095102FC801B7010E94EFD6FE
:10EC400020E030E040E05FEB0E94DCD720E030E0E5
:10EC50004CE752E40E94E9D50E94C1D69B01AC0169
:10EC60008A2D692D422F24E000E00E94DCB9E0915A
:10EC70000726F0E0EE0FFF1FDF01A355B54D0D9005
:10EC8000BC91A02DEB53F54DC081D181AC17BD07D0
:10EC90000CF03FC0C739D105E4F1A659B040BD0121
:10ECA000882777FD8095982F0E94EFD620E030E0EE
:10ECB00040E05FE30E94DCD720E030E04CE752E424
:10ECC0000E94E9D50E94C1D67B018C01D090062616
:10ECD000D394C659D040BE01882777FD8095982FE0
:10ECE0000E94EFD620E030E040E05FE30E94DCD7F6
:10ECF00020E030E04CE752E40E94E9D50E94C1D602
:10ED00009B01AC018E2D6D2D422F24E000E00E946E
:10ED1000DCB9E0910726F0E0EE0FFF1FE355F54D5B
:10ED20000190F081E02D90900626E639F105B4F0CF
:10ED30009394E659F040BF01882777FD8095982F7E
:10ED40000E94EFD620E030E040E05FE30E94DCD795
:10ED50000E94C1D69B01AC018FE32AC066E970E036
:10ED60006E1B7F0B882777FD8095982F0E94EFD62A
:10ED70007B018C0120E030E040E05FEB0E94DCD7BB
:10ED800020E030E04CE752E40E94E9D50E94C1D671
:10ED90005B016C019394C801B70120E030E040E0D2
:10EDA0005FE30E94DCD70E94C1D69B01AC018A2D93
:10EDB000692D422F24E001E00E94DCB98EE36091CE
:10EDC000062642E026E00E94DCB92091062683E078
:10EDD000622F43E02A5F01E00E9428B920910626B5
:10EDE00087E1622F47E12A5F0E9428B92091062619
:10EDF0008BE2622F4BE22A5F0E9428B920910626FF
:10EE000083E5622F43E52A5F0E9428B920910626F8
:10EE100087E6622F47E62A5F0E9428B920910626DE
:10EE20008BE7622F4BE72A5F0E9428B9CDB7DEB788
:10EE3000EBE00C94A8DAE9E7F9E28CE0DF011D923F
:10EE40008A95E9F7ADEABAE28C91865981931296D8
:10EE50008AE2A73BB807C1F7ADB7BEB717970FB6A1
:10EE6000F894BEBF0FBEADBFEDB7FEB7319689E7D0
:10EE700011968C9381E08183828389E799E2948360
:10EE800083838CE090E0968385830E9433568DB710
:10EE90009EB707960FB6F8949EBF0FBE8DBF08951C
:10EEA000A4E1B0E0E6E5F7E70C9485DA8DEA9AE2B2
:10EEB00066E970E043E050E00E9448DCFE013196D4
:10EEC00085E0DF011D928A95E9F780911F33882341
:10EED00019F41098089802C0109A089A80912E335D
:10EEE000882349F480912033882319F411980998D4
:10EEF00002C0119A099A80912133882319F412983B
:10EF00000A9802C0129A0A9A80912233882371F4D7
:10EF100013980B98FE013B9630E000E4A2E3B0E0CA
:10EF200017EC64E970E04CE650E003C0139A0B9ACA
:10EF3000F1CF00937C0080917C00232F2F71807E85
:10EF4000822B80937C00B093A32AA093A22A809165
:10EF5000A22A9091A32A892BD1F710937A0080914D
:10EF60007A0086FDFCCF809178009091790096958B
:10EF70008795969587959070918380838D369105BE
:10EF80001CF45183408305C08439910514F07183CA
:10EF9000608380917C00807E282B20937C00809170
:10EFA0007A00806480937A0080917A0086FDFCCF9D
:10EFB00080917800909179009695879596958795A0
:10EFC0009070918380838D3691051CF4518340832A
:10EFD00005C08439910514F0718360833F5F3296D8
:10EFE000343009F0A6CF80917C00807E80937C0035
:10EFF00080917A00806480937A000E9483B786E3D0
:10F000009DE362E00E9489BB83E090E00E94903E15
:10F01000AC0180E067E020E00E94ACBB82E167E0E9
:10F0200042E35DE320E00E947EBB1CE010930626D5
:10F0300083E0612F48E726E001E00E9432BC209186
:10F04000062687E1622F47E12A5F0E9428B92091B6
:10F0500006268BE2622F4BE22A5F0E9428B98EE3DC
:10F060006091062642E026E00E94DCB92091062647
:10F0700083E5622F43E52A5F0E9428B92091062686
:10F0800087E6622F47E62A5F0E9428B9185F14338B
:10F0900069F686E990E09093AE2A8093AD2A1A82B1
:10F0A00019829093B22A8093B12A1E821D82909376
:10F0B000B62A8093B52A1A861986FF24FA94EE247C
:10F0C0005E010894A11CB11CE1E06E2E712C412C54
:10F0D0007CE3572E212C64EC362E56E9C52ED12C1C
:10F0E00048EC842E912C80917A0086FD03C10E2D70
:10F0F00010E0F801EC5DFC4C8081D801AA0FBB1F29
:10F100008823A1F08091780090917900F501EA0FB1
:10F11000FB1F969587959695879522853385281BA5
:10F120003109A355B54D2D933C9314C080917800BF
:10F130009091790096958795969587959070F501B1
:10F14000EA0FFB1F22853385821B930BA355B54D18
:10F150008D939C93F801EE0FFF1FE355F54D8081D1
:10F160009181BFEF89389B072CF488E89FEF91834A
:10F17000808307C08837910524F0A8E7B0E0B18309
:10F18000A083F801E75DFC4C8081882309F041C031
:10F19000F801EE0FFF1FE355F54D8081918168E086
:10F1A00070E00E9435DACB01AB0177FF04C0442741
:10F1B0005527461B570B489F9001499F300D589F7C
:10F1C000300D1124F801EE0FFF1FEA0DFB1D8081A9
:10F1D0009181280F391F31832083B4EC21303B0704
:10F1E0001CF43182208205C020503C4314F051822F
:10F1F0004082F801EE0FFF1FD501AE0FBF1F8D91AA
:10F200009C9160E870E00E9435DAE355F54D71831A
:10F210006083D801AA0FBB1FA355B54D2D913C911A
:10F2200011972A563F4F11963C932E93F801EE0FFB
:10F23000FF1FE55FFC4C808191818217930750F49A
:10F24000F801EE0FFF1FEB5EFC4C808191812817C7
:10F25000390720F0808191818D939C93F801EE0F06
:10F26000FF1FDF01AB53B54DE355F54D20813181D3
:10F270008D919C912817390741F0C301002E02C0DF
:10F28000880F991F0A94E2F7F82AE39493E0E916AD
:10F2900021F580912733882319F0039B03C007C011
:10F2A000039B05C080911B3390911C3304C0809157
:10F2B0001133909112339093B42A8093B32A209102
:10F2C000B32A3091B42A8091CB2A9091CC2A281766
:10F2D000390711F0A8E0FA2AEE2480917C009E2DD7
:10F2E0009F71807E982B90937C0080917A0080643F
:10F2F00080937A0080E40E940573182F80E463E015
:10F300000E945E73182BF1F180912D33882331F523
:10F3100080912833882331F48091B52A9091B62AC0
:10F32000019605C08091B52A9091B62A01979093D5
:10F33000B62A8093B52A2091B52A3091B62A8091B9
:10F340001333909114338217930788F480911D33FF
:10F3500090911E332817390790F004C0809128330C
:10F36000882329F480911D3390911E3304C080912D
:10F370001333909114339093B62A8093B52AB0E159
:10F38000FB2A47C080E80E940573182F80E863E0DD
:10F390000E945E73182BE9F180912D33882331F59B
:10F3A00080912833882331F48091B52A9091B62A30
:10F3B000019705C08091B52A9091B62A0196909345
:10F3C000B62A8093B52A2091B52A3091B62A809129
:10F3D0001333909114338217930760F480911D3397
:10F3E00090911E332817390790F009C08091283377
:10F3F000882329F4809113339091143304C08091B1
:10F400001D3390911E339093B62A8093B52A20E144
:10F41000F22A80912D33882389F08091B52A90912A
:10F42000B62A8639910551F0069B08C0079B06C095
:10F43000D092B62AC092B52A80E1F82A80E10E94D3
:10F4400005738823E9F0D092AE2AC092AD2A1A82C1
:10F450001982D092B22AC092B12A1E821D82D09205
:10F46000B62AC092B52A1A8619869092FA258092F9
:10F47000F92580E890E09093AE208093AD2003C002
:10F48000FF2009F473C09CE0909306261092072693
:10F490000E94DA75E0910726F0E0EE0FFF1FDF0112
:10F4A000A355B54D8D919C91EB53F54D9183808380
:10F4B000A4E1A0930626B1E0B093072680912E33F5
:10F4C000882311F40E94DA75E0910726F0E0EE0F30
:10F4D000FF1FDF01A355B54D8D919C91EB53F54D69
:10F4E000918380832CE12093062682E08093072677
:10F4F0000E94DA75E0910726F0E0EE0FFF1FDF01B2
:10F50000A355B54D8D919C91EB53F54D918380831F
:10F5100094E29093062683E0809307260E94DA7592
:10F52000E0910726F0E0EE0FFF1FDF01A355B54D78
:10F530008D919C91EB53F54D91838083ACE2A09328
:10F540000626B4E0B09307260E94DA75E0910726FC
:10F55000F0E0EE0FFF1FDF01A355B54D8D919C919B
:10F56000EB53F54D918380830E941B7780E20E94CC
:10F570000573FF24882309F4B6CD80EF0E9405733C
:10F5800080912E33813011F40E9413B66496E2E12B
:10F590000C94A1DAA8E0B0E0E0EDFAE70C9485DA8B
:10F5A00010924A26AA247724BB24B39490E09C01AD
:10F5B0002F5F3F4F3A83298312E1612E9C012D5822
:10F5C0003D4CA9014A545F4F5C834B83F901EF54D2
:10F5D000FF4FFE83ED83BCEA2B2E312C220E331E0F
:10F5E000880F991FF5E14F2EF3E35F2E480E591E49
:10F5F0004C012BE033E3820E931E01C0B12E0E941A
:10F6000083B780E060E047ED5FE322E00E940ABC40
:10F6100089E060E049815A8121E030E000E072E059
:10F62000E72E0E945BC181E090E00E94903EAC0119
:10F6300080E067E020E00E94ACBBAA2039F081E0C6
:10F6400061E045ED5FE320E00E947EBBCA2CDD2433
:10F6500046E350E0C49E8001C59E100DD49E100D5F
:10F66000112418861F82EF80F884EC0CFD1C55E0F5
:10F67000E516F1047CF4409176326F816F5F469D10
:10F68000A0011124400F511F4B53514C83E020E047
:10F690000E947EBB8F81853059F494E0E916F10415
:10F6A0003CF481E066E043ED5FE320E00E947EBB36
:10F6B000EF81F8853196F887EF830A5C1F4F369704
:10F6C00091F6772069F4AA2029F481E065E04B2DBA
:10F6D00020E00AC082E065E04B2D21E001E005C09A
:10F6E00082E066E04B2D21E000E00E94553B182FA0
:10F6F0008E3F31F4A3947724739495E0B92E9DCF77
:10F700008D3F29F4AA94772482E0B82E96CF8F3FBC
:10F7100051F480914A26813009F068C00E94CBC91B
:10F7200010924A2663C0E82EFF24EA0CF11CF1E097
:10F73000EF16F10479F4F4018081918160E070E0CA
:10F740004CE251E02EED00E00E947688F4019183B6
:10F75000808337C0F2E0EF16F10479F4F201808182
:10F76000918160E070E04CE251E02FED00E00E94FA
:10F770007688F2019183808341CFF3E0EF16F104A4
:10F7800069F4F101808190E060E070E041E050E0D8
:10F7900021EE0BE00E947688F10126C0F4E0EF161E
:10F7A000F10479F4ED81FE81808190E060E070E009
:10F7B00041E050E020EE07E00E947688ED81FE8176
:10F7C00013C0F5E0EF16F10409F018CFEB81FC81CE
:10F7D000808190E060E070E041E050E022EE05E0E2
:10F7E0000E947688EB81FC81808308CF2896E2E135
:10F7F0000C94A1DAA0E0B0E0E0E0FCE70C948FDA32
:10F800000E9483B780E060E048E450E422E00E9478
:10F810000ABC80E061E042E350E420E00E940ABCC0
:10F82000CC24DD24FC2C1C2D1E5FE6010894C11C99
:10F83000D11C80E0612FA60121E030E000E0EE2441
:10F840000E945BC1FE01EE0FFF1FE55FFC4C408193
:10F85000518182E0612F23E030E00E945BC1FE0114
:10F86000EE0FFF1FEB5EFC4C4081518186E0612F63
:10F8700023E030E00E945BC1FE01E15EFC4C808130
:10F88000882329F48AE0612F4DE250E404C08AE025
:10F89000612F48E250E420E00E940ABCFE01EC5DCA
:10F8A000FC4C8081882329F48FE0612F43E250E4EF
:10F8B00004C08FE0612F4FE150E420E00E940ABCB9
:10F8C000C75DDC4C8881882329F484E1612F4DE1F8
:10F8D00050E404C084E1612F4BE150E420E00E9439
:10F8E0000ABC81E0F81659F480912E33813039F446
:10F8F00083E0612F48E050E420E00E940ABC85E0EC
:10F90000C816D10409F08ECF82E167E045E050E4EB
:10F9100020E00E947EBB80E10E9405738823D9F31A
:10F92000CDB7DEB7E8E00C94ABDAA0E0B0E0EBE9ED
:10F93000FCE70C9487DA10924A26CC249924DD2423
:10F94000D39466E3462E512C52E1852E44EF642E6B
:10F9500041E0742E01C0D12E0E9483B780E060E0A8
:10F960004FEE5FE322E00E940ABC81E090E00E943B
:10F97000903EAC0180E067E020E00E94ACBBCC2070
:10F9800039F081E061E04DEE5FE320E00E947EBB54
:10F99000AC2CBB24A49C8001A59C100DB49C100D24
:10F9A0001124C0E0D0E07E01EA0CFB1C87E0E816E1
:10F9B000F10484F440917632CE018F5F682F489D28
:10F9C000A0011124400F511F455B524C83E020E001
:10F9D0000E947EBBC53059F496E0E916F1043CF470
:10F9E00081E066E04BEE5FE320E00E947EBB219663
:10F9F0000A5C1F4FC630D105B1F6992039F4CC20EE
:10FA000069F481E065E04D2D20E00CC0CC2031F0A0
:10FA100082E066E04D2D21E000E005C082E065E077
:10FA20004D2D21E001E00E94553B182F8E3F31F40F
:10FA3000C3949924939435E0D32EA1CF8D3F29F41C
:10FA4000CA94992422E0D22E9ACF8F3F51F480910C
:10FA50004A26813009F056C00E94CBC910924A262E
:10FA600051C0C82FD0E0CC0DD11DC130D10519F443
:10FA70000E94FA7B2AC0C230D10521F480E00E94A6
:10FA8000CA7A28C0C330D105D9F480912E33813091
:10FA9000A1F40E9483B783EE90E00E94903EAC01F7
:10FAA00080E063E022E00E94ACBB80E197E2F301DA
:10FAB0003197F1F70197D9F714C081E00E94CA7A13
:10FAC000C430D10511F482E009C0C530D10511F46C
:10FAD00083E004C0C630D10521F484E00E94CA7AD4
:10FAE0003ACF279709F037CF80912E3390E060E02E
:10FAF00070E041E050E023EE05E00E9476888093BC
:10FB00002E3329CFCDB7DEB7E0E10C94A3DAEF9224
:10FB1000FF920F931F936091D12A7091D22A80E0B7
:10FB200090E00E94EDD66093EB2B7093EC2B8093CA
:10FB3000ED2B9093EE2B2091DF2A3091E02A40911B
:10FB4000E12A5091E22A0E9454D67B018C016093F5
:10FB5000D32A7093D42A8093D52A9093D62A0E94D0
:10FB6000BCD66093F32B70E0882777FD8095982FA3
:10FB70000E94EFD69B01AC01C801B7010E94E8D5F5
:10FB800020E030E040E853E40E94DCD70E94C1D678
:10FB90006093EA2B1F910F91FF90EF900895282F0B
:10FBA000909148269F5F9F73809149269817E1F3B3
:10FBB000E92FF0E0E85FF94D2083909348260895FF
:10FBC000A4E0B0E0E6EEFDE70C9495DA9A83898331
:10FBD0007C836B83282F909148269F5F9F73809131
:10FBE00049269817E1F3E92FF0E0E85FF94D20830B
:10FBF00090934826FE0131962181909148269F5F7F
:10FC00009F73809149269817E1F3E92FF0E0E85FB0
:10FC1000F94D208390934826909148269F5F9F73CB
:10FC2000809149269817E1F3E92FF0E0E85FF94D5C
:10FC30004083909348262B81909148269F5F9F7325
:10FC4000809149269817E1F3E92FF0E0E85FF94D3C
:10FC5000208390934826FE01339621819091482677
:10FC60009F5F9F73809149269817E1F3E92FF0E099
:10FC7000E85FF94D2083909348262496E2E00C94A7
:10FC8000B1DACF93DF93C0E0D0E0BE0180E090E036
:10FC90000E94EDD62BED3FE049EC50E40E94DCD70A
:10FCA00020E030E040E85BE30E94DCD70E94ABD864
:10FCB00020E030E04EEF52E40E94DCD70E94C1D633
:10FCC000FE01ED51F54D6083219681E0C030D807EB
:10FCD000E1F6DF91CF9108956091DB2A7091DC2AE3
:10FCE0008091DD2A9091DE2A20E030E040EA51EC5C
:10FCF0000E9454D69B01AC0160E070E080E291E488
:10FD00000E943FD89B01AC012093EF2B3093F02B46
:10FD10004093F12B5093F22BCA01B90120E030E05F
:10FD20004FE753E40E94DCD70E94C1D66093E82BD2
:10FD30000895FF920F931F93909148268091492632
:10FD4000981709F47EC0E0914926EF5FEF73E093C6
:10FD50004926F0E0E85FF94D0081909148268091B6
:10FD60004926981709F46DC0E0914926EF5FEF73BB
:10FD7000E0934926F0E0E85FF94D20819091482614
:10FD800080914926981709F45CC0E0914926EF5FFD
:10FD9000EF73E0934926F0E0E85FF94DF080909131
:10FDA000482680914926981709F44BC0E0914926CE
:10FDB000EF5FEF73E0934926F0E0E85FF94D3081A3
:10FDC00090914826809149269817D9F1922F80E08A
:10FDD00010E0082B192BE0914926EF5FEF73E093B9
:10FDE0004926F0E0E85FF94D2081922F80E0232F33
:10FDF00030E0822B932B6AE070E00E9421DA70934E
:10FE0000AC2A6093AB2A1093D22A0093D12A0E9485
:10FE1000877D6F2D70E080E090E00E94EDD66093CA
:10FE2000DB2A7093DC2A8093DD2A9093DE2A0E94DD
:10FE30006C7E012B19F41092CF2A03C081E08093CD
:10FE4000CF2A1F910F91FF9008950F931F938C015C
:10FE50009093D22A8093D12A0E94877D80E090E0FF
:10FE6000A0E0B0E08093DB2A9093DC2AA093DD2A07
:10FE7000B093DE2A0E946C7E012B19F41092CF2AD7
:10FE800003C081E08093CF2A1F910F91089580E0F5
:10FE900094E9A8E9B6E48093D72A9093D82AA0934E
:10FEA000D92AB093DA2A8AE193ECA6E5B8E38093E5
:10FEB000E42B9093E52BA093E62BB093E72B80E007
:10FEC00094E9A8E9B2E48093DF2A9093E02AA09312
:10FED000E12AB093E22A80E991E09093D22A8093BC
:10FEE000D12A0E94877D0E946C7E08951092482638
:10FEF000109249260E94477F0E94417E0E943C72D8
:10FF00000E94687208950E9483B780E063E047E230
:10FF100050E522E00E947EBB80E064E042E150E5D3
:10FF200022E00E947EBB80E197E224EF31E0F901FC
:10FF30003197F1F70197D9F708950F931F93082F81
:10FF4000122F80930F2C1092102C0E9483B7812FB8
:10FF500090E00E94903EAC0180E062E020E00E94D0
:10FF6000ACBB013019F00330A9F522C089E590E05F
:10FF700063E170E043E050E021E00E9472BC85E65E
:10FF800090E063E170E043E050E020E00E94FEBCBE
:10FF900085E690E063E170E043E050E021E00E94FC
:10FFA00072BC85E690E063E170E041E050E00FC094
:10FFB00089E590E063E170E043E050E021E00E94D9
:10FFC00072BC85E690E063E170E043E050E021E040
:10FFD0000E94FEBC82E090E00E94903EAC0180E076
:10FFE00067E020E00E94ACBB80E40E940573882398
:10FFF000A9F0013099F489E590E063E170E043E015
:020000021000EC
:1000000050E021E00E9472BC85E690E063E170E080
:1000100043E050E021E00E94FEBC03E080E80E9443
:100020000573882339F1033029F589E590E063E110
:1000300070E043E050E021E00E9472BC85E690E071
:1000400063E170E043E050E020E00E94FEBC85E602
:1000500090E063E170E043E050E021E00E9472BC78
:1000600085E690E063E170E041E050E021E00E942D
:10007000FEBC01E080E10E940573882351F081E01D
:1000800080934A260093DF320E94CBC910924A2601
:100090000FC080E20E940573882309F4A5CF80EF8A
:1000A0000E94057310924A2600910F2C0093DF32B4
:1000B000802F1F910F9108951F93182F80930F2C5D
:1000C0001092102C0E9483B786E790E00E94903E29
:1000D000AC0180E062E020E00E94ACBB112319F08B
:1000E000113069F405C08FE062E048EC5DE404C0C3
:1000F0008FE062E043EC5DE420E00E947EBB82E0A2
:1001000090E00E94903EAC0180E067E020E00E9419
:10011000ACBB80E40E940573882351F0112341F4A5
:100120008FE062E04EEB5DE420E00E947EBB11E0D8
:1001300080E80E940573882351F0113041F48FE06C
:1001400062E049EB5DE420E00E947EBB10E080E1CC
:100150000E940573882321F081E080934A260CC019
:1001600080E20E9405738823A1F280EF0E9405734C
:1001700010924A2610910F2C1093DC32812F1F9180
:100180000895AF92BF92CF92DF92EF920F931F9399
:10019000CF93DF93EC015B016A010E9483B787E78D
:1001A00090E00E94903EAC0180E062E020E00E947E
:1001B000ACBB89E790E00E94903EAC0180E065E036
:1001C00020E00E94ACBB8AE790E00E94903EAC0128
:1001D00080E066E020E00E94ACBBD093F72BC09398
:1001E000F62B80E162E0AE0124E030E000E0EE2496
:1001F0000E945BC182E090E00E94903EAC0180E0F2
:1002000067E020E00E94ACBB86EF9FEFC80ED91ECE
:1002100011E080E40E940573882331F480E462E0F9
:100220000E945E73882399F0CC15DD0580F410934D
:100230004A262A96D093DB32C093DA3280E162E01C
:10024000AE0124E030E000E0EE240E945BC180E8D3
:100250000E940573882331F480E862E00E945E7397
:10026000882399F0AC16BD0680F410934A262A978D
:10027000D093DB32C093DA3280E162E0AE0124E059
:1002800030E000E0EE240E945BC180E10E94057333
:10029000882339F50E94F2B640918D2650918E2622
:1002A00088E063E020E030E000E00E94B9BE83E037
:1002B00063E044EB5DE420E00E947EBB80E20E94AC
:1002C0000573882309F4A5CF80EF0E94057310926F
:1002D0004A26C091F62BD091F72BD093DB32C093F6
:1002E000DA32CE01DF91CF911F910F91EF90DF9025
:1002F000CF90BF90AF900895A0E0B0E0E2E8F1E8C1
:100300000C9489DA1092F52B10924A260E9483B73A
:10031000BB249924AA24A39436E3632E712C22E1F2
:10032000822E01C0A12E0E9483B785E790E00E9433
:10033000903EAC0180E060E022E00E94ACBB81E036
:1003400090E00E94903EAC0180E067E020E00E94D7
:10035000ACBBBB2039F081E061E042EB5DE420E022
:100360000E947EBBCB2CDD24C69C8001C79C100D57
:10037000D69C100D1124C0E0D0E07E01EC0CFD1CD9
:1003800082E0E816F10484F440917632CE018F5F6A
:10039000682F489DA0011124400F511F4253574B15
:1003A00083E020E00E947EBBC53051F4E114F104EB
:1003B00039F481E066E040EB5DE420E00E947EBB22
:1003C00021960A5C1F4FC630D105B9F6992069F411
:1003D000BB2029F481E062E04A2D20E00AC082E0DF
:1003E00065E04A2D21E001E005C082E066E04A2D8B
:1003F00021E000E00E94553B182F8E3F31F4B3946A
:100400009924939495E0A92EA4CF8D3F29F4BA9412
:10041000992482E0A82E9DCF8F3F49F480914A26EF
:10042000813079F50E94CBC910924A262AC090E00B
:100430008B0D911D8130910549F48091DC3260E093
:1004400041E00E945C808093DC3211C0029709F089
:1004500069CF8091DA329091DB3260E070E04FE05A
:1004600057E20E94C1809093DB328093DA32809110
:100470004A26813009F056CF0E94CBC910924A26F5
:1004800051CFCDB7DEB7EEE00C94A5DA2F923F92B4
:100490005F926F927F928F929F92AF92BF92CF9214
:1004A000DF92EF92FF920F931F93CF93DF935090C1
:1004B00098261092F52B10924A260E9483B7BB24EF
:1004C000B39499248824652C772413010894210877
:1004D000310801C0BB240E9483B780E060E04BE498
:1004E0005FE422E00E947EBB81E090E00E94903EAB
:1004F000AC0180E067E020E00E94ACBB992039F0BD
:1005000081E061E049E45FE420E00E947EBBEE24EC
:10051000FF24AA24A394C92CDD24E701CC0DDD1D02
:10052000C615D70514F58E01000F111FCE0125E069
:10053000880F991F2A95E1F7080F191FC8018C5ED3
:10054000974C60EC72E34EE050E00E945FDCA80143
:100550004050584C009721F483E06A2D22E003C0FC
:1005600083E06A2D20E00E94ACBB85E0E81651F4E0
:10057000C215D3053CF481E066E047E45FE420E087
:100580000E947EBB0894E11CF11CA39497E0A9167D
:1005900021F6882079F49920D1F486E0851528F495
:1005A00081E065E04B2D20E016C081E0652D4B2DEC
:1005B00020E00BC086E090E0C80ED91EC614D70418
:1005C00034F082E066E04B2D21E000E005C082E0DF
:1005D00065E04B2D21E001E00E94553B482F8E3F06
:1005E00031F4939415E0B12E8824839487CF8D3F06
:1005F00029F49A94B2E0BB2E882480CF8F3F49F42F
:1006000080914A268130D1F50E94CBC910924A26AA
:1006100035C0882309F45ECF282F30E021503040C8
:10062000F901EE0FFF1FC90175E0880F991F7A9538
:10063000E1F7E80FF91FEC5EF74CC0ECD2E38191D3
:10064000899392E3CE3CD907D1F7D90165E0AA0F8F
:10065000BB1F6A95E1F7220F331FA20FB31FA050F3
:10066000B84CFE01B2978D91819382E3E03CF8078C
:10067000D1F781E080934A26B42E2DCFDF91CF9120
:100680001F910F91FF90EF90DF90CF90BF90AF90B0
:100690009F908F907F906F905F903F902F900895E4
:1006A000A0E0B0E0E6E5F3E80C9487DAF82EE92E56
:1006B000D62EC42E89010E9483B780E060E0A80195
:1006C00022E00E947EBB2F2D3E2DC901EC0198EF48
:1006D000E92E9BE2F92E01E0DD0CD39414C0102F1B
:1006E0001F5F802F63E0488120E00E94B5BB0E5F52
:1006F000812F63E045E85FE420E00E947EBB8991A2
:10070000F70181937F010D1551F783E066E14AE01F
:100710002AE001E00E9432BC80E066E046E75FE448
:1007200020E00E947EBB80E067E041E65FE420E0DD
:100730000E947EBB11E0FF24EE24E39489E3982E0F
:10074000B0E3AB2EA0E2DA2EFAE06F2EEAE55E2EE1
:1007500071E6472E61E4862E56E0B52E44E0742EF5
:10076000F1E0CF1609F074C0E1E0FCE29AE080818C
:10077000803219F090930E2C04C091503197992338
:10078000B1F780E40E940573882331F480E462E0CD
:100790000E945E73882379F1AF2DB0E0FD01E8502F
:1007A000F44D80818A3738F58F5F8083803208F47A
:1007B000D082FD01E850F44D808181528F3008F4E1
:1007C000A082FD01E850F44D80818A53873008F4FF
:1007D0008082FD01E850F44D80818B55863008F40D
:1007E0004082A850B44D812F63E04C9120E00E94DC
:1007F000B5BBE0924A2680E80E940573882339F44D
:1008000080E862E00E945E73882309F472C0AF2D15
:10081000B0E0FD01E850F44D8081813208F469C0F8
:10082000815080838B55863008F45082FD01E8505A
:10083000F44D80818A53873008F49082FD01E8509E
:10084000F44D808181528F3008F049C0D08247C07A
:1008500082E0C81609F04DC080E40E940573882329
:1008600031F480E461E00E945E738823F9F0AF2DDB
:10087000B0E0FD01E850F44D80818933B8F48F5F1A
:100880008083803208F4D082FD01E850F44D8081ED
:1008900081528F3008F4A082A850B44D812F63E0BC
:1008A0004C9120E00E94B5BBE0924A2680E80E946D
:1008B0000573882331F480E861E00E945E73882329
:1008C000C1F0AF2DB0E0FD01E850F44D80818133DF
:1008D00080F0815080838A53873008F49082A8503A
:1008E000B44D812F63E04C9120E00E94B5BBE092B3
:1008F0004A2680E20E9420738823E9F0E1E0CE16C8
:1009000031F4EF2DF0E0E850F44DD08208C0F2E071
:10091000CF1629F4EF2DF0E0E850F44DA082EF2D32
:10092000F0E0E850F44D812F63E0408120E00E9428
:10093000B5BBE0924A2680E20E940F73882309F437
:1009400040C081E0C81619F46092112C05C0E2E0A5
:10095000CE1611F47092112C212F269530E02F5FC6
:100960003F4F8091112C90E028173907A4F01B9D70
:10097000C0011124835066E14AE02AE000E00E94B1
:1009800032BC83E066E14AE02AE001E00E9432BC2A
:1009900011E0FF2416C01B9DC0011124835066E1A5
:1009A0004AE02AE000E00E9432BC1E5F1B9DC001AD
:1009B0001124835066E14AE02AE001E00E9432BC43
:1009C000F39480E10E940573882309F4C9CE81E085
:1009D000CDB7DEB7E0E10C94A3DA0E9483B780EFD5
:1009E0000E94057387E590E00E94903EAC0180E094
:1009F00062E020E00E94ACBB88E590E00E94903E5F
:100A0000AC0180E063E020E00E94ACBB86E590E0B2
:100A10000E94903EAC018CE067E020E00E94ACBBFD
:100A200080E10E940573882321F00E94E1C9299882
:100A3000089580E20E940573882391F380EF0E945D
:100A400005730895CF92DF92EF92FF920F931F9359
:100A5000F82EC62ED42E122F80930F2C1092102C0D
:100A6000682F70E0882777FD8095982F0E94EFD639
:100A700023E333E343E250E40E94DCD70E94C1D673
:100A80006093B3000E9483B7812F90E00E94903E54
:100A9000AC0180E062E020E00E94ACBB80E162E05B
:100AA0004F2D50E023E030E000E0EE240E945BC1D7
:100AB00081E162E04FEB5FE420E00E947EBB82E0D8
:100AC00090E00E94903EAC0180E067E020E00E9450
:100AD000ACBB80E162E04F2D50E023E030E000E06D
:100AE000EE240E945BC18F2D90E09695982F882769
:100AF0009795879564E670E00E9435DA462F80E08E
:100B000060E226E001E00E94DCB980E40E94057307
:100B1000882331F480E463E00E945E73882301F14E
:100B2000FD14F0F4F394FD1448F088EC90E060E8D4
:100B300070E040E00E946A73FD2C12C06F2D70E0DF
:100B4000882777FD8095982F0E94EFD623E333E323
:100B500043E250E40E94DCD70E94C1D66093B30008
:100B600080E80E940573882331F480E863E00E94E6
:100B70005E73882391F1CF1480F58F2D90E001975B
:100B80009695982F88279795879564E670E00E9440
:100B900035DA862F60E240E826E000E00E94DCB90A
:100BA000FA94FC1441F488EC90E060E870E040E0D6
:100BB0000E946A7312C06F2D70E0882777FD8095C0
:100BC000982F0E94EFD623E333E343E250E40E94E0
:100BD000DCD70E94C1D66093B30080E10E94057308
:100BE0008823E1F081E080934A266F2D70E088270A
:100BF00077FD8095982F0E94EFD623E333E343E2FD
:100C000050E40E94DCD70E94C1D66093B300F092FA
:100C10007F320E94CBC910924A2624C080E20E94F3
:100C20000573882309F455CF80EF0E940573109255
:100C30004A2600910F2C1091102CB80180E090E012
:100C40000E94EDD623E333E343E250E40E94DCD775
:100C50000E94C1D66093B30000937F320E94CBC93B
:100C6000F0900F2C8F2D1F910F91FF90EF90DF9040
:100C7000CF9008950F931F93182F80930F2C1092ED
:100C8000102C0E9483B784E390E00E94903EAC0158
:100C900080E061E020E00E94ACBB85E390E00E9430
:100CA000903EAC0180E062E020E00E94ACBB80910D
:100CB0008332882309F056C084E390E00E94903E7E
:100CC000AC0180E061E020E00E94ACBB86E390E0F4
:100CD0000E94903EAC0180E062E020E00E94ACBB4C
:100CE00087E390E00E94903EAC0180E061E020E06C
:100CF0000E94ACBB88E390E00E94903EAC0180E093
:100D000062E020E00E94ACBB89E390E00E94903E4C
:100D1000AC0180E061E020E00E94ACBB8AE390E09F
:100D20000E94903EAC0180E062E020E00E94ACBBFB
:100D30008BE390E00E94903EAC0180E061E020E017
:100D40000E94ACBB8CE190E00E94903EAC018CE034
:100D500067E020E00E94ACBB80E20E94057388231C
:100D6000D9F37BC0112319F0113099F408C08EE03B
:100D700062E047EC5FE420E00E947EBB0AC082E5AF
:100D800090E00E94903EAC018EE062E020E00E9484
:100D9000ACBB82E090E00E94903EAC0180E067E056
:100DA00020E00E94ACBB00918332013009F04FC0BB
:100DB00080E40E940573882391F0112381F400934D
:100DC0004A2682E590E00E94903EAC018EE062E00F
:100DD00020E00E94ACBB86E00E947D3211E080E8FA
:100DE0000E940573882379F0113069F410934A2624
:100DF0008EE062E041EC5FE420E00E947EBB85E093
:100E00000E947D3210E080E10E9405738823F9F092
:100E10008CE390E00E94903EAC0180E064E020E032
:100E20000E94ACBB8DE390E00E94903EAC0180E05C
:100E300065E020E00E94ACBB80E067E042E10E94F8
:100E400013BC80E10E9405738823D9F30DC080E2B2
:100E50000E940573882309F4A6CF80EF0E940573D2
:100E600010924A2610910F2C812F1F910F910895F7
:100E7000AF92BF92CF92DF92EF920F93CF93DF9317
:100E8000EC015B016A01E22FF0E0EC30F10508F0C3
:100E900024C1EA5BFF4F0C94BCDA80E162E0AE0152
:100EA00023E030E000E0EE240E945BC116C180E147
:100EB00062E0AE0123E030E000E0EE240E942CC0AE
:100EC0000CC1009729F08130910509F006C105C0D9
:100ED0008CE062E048E050E504C08CE062E04EEF58
:100EE0005FE420E00E947EBBF8C0009729F08130CB
:100EF000910509F0F2C003C083E590E002C084E5EB
:100F000090E00E94903EAC018FE0E3C0009729F092
:100F10008130910509F0E1C003C08CE290E00FC080
:100F20008BE290E00CC0009729F08130910509F028
:100F3000D4C003C080E790E002C08FE690E00E943A
:100F4000903EAC0181E1C5C0009729F08130910548
:100F500009F0C3C003C084E590E0B7C085E590E028
:100F6000B4C080E162E0AE0123E030E000E0EE24B6
:100F70000E945BC1CC15DD0580F088EC90E060E854
:100F800070E040E00E946A7380E162E0A60123E025
:100F900030E00E945BC1E60113C080E162E0AE0177
:100FA00023E030E000E0EE240E945BC1F8942B982F
:100FB00081E80E9475B78C2F0E9475B72B9A7894A0
:100FC000CA15DB0589F480E162E0AE0123E030E080
:100FD00000E0EE240E945BC188EC90E060E870E0E5
:100FE00040E00E946A7379C080E162E0AE0123E0D4
:100FF00030E000E0EE240E945BC1F8942B9881E879
:101000000E9475B78C2F0E9475B72B9A789465C093
:101010008330910521F18430910538F481309105B8
:10102000A1F082309105B0F40BC08530910509F133
:1010300085309105C8F08630910509F04EC01EC07C
:101040008FE062E047EF5FE44CCF8FE062E040EF7B
:101050005FE447CF8FE062E049EE5FE442CF8FE08C
:1010600062E042EE5FE43DCF8FE062E04BED5FE493
:1010700038CF8FE062E044ED5FE433CF8FE062E091
:101080004DEC5FE42ECF8130910551F08130910518
:1010900020F08230910509F506C089E590E005C091
:1010A0008AE590E002C08CE590E00E94903EAC01A1
:1010B0008AE00FC0009721F08130910571F403C0E0
:1010C00084EE90E002C085EE90E00E94903EAC017C
:1010D0008EE062E020E00E94ACBBDF91CF910F91E7
:1010E000EF90DF90CF90BF90AF900895A0E0B0E078
:1010F000ECE7F8E80C948FDAEC016B017A01122F1F
:101100009093102C80930F2C0E9483B7812F90E036
:101110000E94903EAC0180E062E020E00E94ACBB07
:10112000CE01B601A701202F0E94388782E090E00F
:101130000E94903EAC0180E067E020E00E94ACBBE2
:1011400011E080E40E940573882331F480E462E0BA
:101150000E945E738823A1F0CE15DF0588F41093FA
:101160004A262196CE01B601A701202F0E9438877A
:101170004091F13284EF91E064E170E00E94E07D03
:1011800080E80E940573882331F480E862E00E94C1
:101190005E738823A1F0CC16DD0688F410934A26EE
:1011A0002197CE01B601A701202F0E9438874091D8
:1011B000F13284EF91E064E170E00E94E07D80E133
:1011C0000E940573882379F480E20E9405738823C6
:1011D00009F4B7CF80EF0E94057310924A26C091A0
:1011E0000F2CD091102CCE01CDB7DEB7E8E00C94D7
:1011F000ABDAA0E0B0E0EFEFF8E80C9489DA1092F7
:10120000F52B10924A260E9483B7BB249924AA2466
:10121000A39476E3672E712C62E1862E01C0A12E85
:101220000E9483B781EC90E00E94903EAC0180E088
:1012300060E022E00E94ACBB81E090E00E94903E22
:10124000AC0180E067E020E00E94ACBBBB2039F03D
:1012500081E061E04AEA5DE420E00E947EBBCB2CA5
:10126000DD24C69C8001C79C100DD69C100D112456
:10127000C0E0D0E07E01EC0CFD1C83E0E816F10438
:1012800084F440917632CE018F5F682F489DA00193
:101290001124400F511F4258554B83E020E00E941B
:1012A0007EBBC53059F492E0E916F1043CF481E0CC
:1012B00066E048EA5DE420E00E947EBB21960A5C7D
:1012C0001F4FC630D105B1F6992069F4BB2029F42F
:1012D00081E063E04A2D20E00AC082E065E04A2D0B
:1012E00021E001E005C082E066E04A2D21E000E057
:1012F0000E94553B182F8E3F31F4B3949924939458
:1013000055E0A52EA3CF8D3F29F4BA94992442E04D
:10131000A42E9CCF8F3F51F480914A26813009F052
:1013200044C00E94CBC910924A263FC090E08B0D6A
:10133000911D8130910589F48091E9329091EA32D2
:101340006AEF70E040E65AEE22EC00E00E947688F8
:101350009093EA328093E93262CF8230910589F42A
:101360008091EB329091EC3260E070E044E650E026
:1013700023EC00E00E9476889093EC328093EB326D
:101380004ECF039709F04BCF8091ED329091EE3222
:1013900061E070E044E150E024EC00E00E947688D7
:1013A0009093EE328093ED323ACFCDB7DEB7EEE0D8
:1013B0000C94A5DAA0E0B0E0E0EEF9E80C9487DA4E
:1013C0001092F52B10924A260E9483B7AA24772404
:1013D000BB24B394B6E34B2E512CA2E16A2E01C07C
:1013E000B12E0E9483B786EB90E00E94903EAC0144
:1013F00080E060E022E00E94ACBB81E090E00E94CF
:10140000903EAC0180E067E020E00E94ACBBAA20E7
:1014100039F081E061E04EEA5DE420E00E947EBBAD
:101420000A2D10E0049D7001059DF00C149DF00C38
:101430001124C0E0D0E048016E01C00ED11E89E049
:10144000C816D10484F440917632CE018F5F682FA4
:10145000469DA00111244E0D5F1D4E53544B83E059
:1014600020E00E947EBBC53059F498E0C916D10433
:101470003CF481E066E04CEA5DE420E00E947EBB43
:10148000219686E390E0E80EF91EC630D105A1F65C
:10149000772039F4AA2079F481E065E04B2D20E033
:1014A0000EC093E08916910434F082E066E04B2D83
:1014B00021E000E005C082E065E04B2D21E001E085
:1014C0000E94553B182F8E3F31F4A39477247394D8
:1014D000F5E0BF2E9CCF8D3F29F4AA947724E2E05B
:1014E000BE2E95CF8F3F51F480914A26813009F06E
:1014F000A1C00E94CBC910924A269CC0C82FD0E040
:10150000CA0DD11DC130D10551F48091DF3261E0A7
:1015100043E028EB0E949D7F8093DF3233C0C230CE
:10152000D10571F48091DE3290E060E070E041E03E
:1015300050E027EB05E00E9476888093DE3233C0CE
:10154000C330D10571F48091E03290E060E070E04A
:1015500041E050E029EB05E00E9476888093E0327C
:1015600033C0C430D10571F48091E13290E060E085
:1015700070E047EF50E02AEB01E00E94768880930C
:10158000E13233C0C530D10571F48091E23290E090
:1015900060E070E041E050E02BEB05E00E947688CF
:1015A0008093E23236C0C630D10571F48091E332C7
:1015B00090E060E070E041E050E02CEB05E00E943C
:1015C00076888093E3320CCFC730D10571F48091D7
:1015D000743290E060E270E047EF50E02BE701E00A
:1015E0000E94768880937432FBCEC830D10589F48E
:1015F0008091E4329091E53260E070E040E355E79D
:101600002DEB00E00E9476889093E5328093E432DF
:10161000E7CE299709F0E4CE8091E73290E060E0D0
:1016200070E041E050E02FEB05E00E947688809367
:10163000E732D6CECDB7DEB7E0E10C94A3DAA0E076
:10164000B0E0E5E2FBE80C9488DA1092F52B1092FA
:101650004A260E9483B799248824BB24B394AA24E1
:1016600096E3692E712C82E1582E01C0BF2C0E9496
:1016700083B785E990E00E94903EAC0180E060E095
:1016800022E00E94ACBB81E090E00E94903EAC0161
:1016900080E067E020E00E94ACBB992039F081E057
:1016A00061E049EC5EE420E00E947EBBC92CDD24B1
:1016B000C69C8001C79C100DD69C100D1124C0E063
:1016C000D0E07E01EC0CFD1C86E0E816F10484F409
:1016D00040917632CE018F5F682F459DA001112485
:1016E000400F511F465C564B83E020E00E947EBBBA
:1016F000C53059F495E0E916F1043CF481E066E068
:1017000047EC5EE420E00E947EBB21960A5C1F4FFE
:10171000C630D105B1F6882069F4992029F481E01A
:1017200066E04B2D20E00AC082E065E04B2D21E011
:1017300001E005C082E066E04B2D21E000E00E9460
:10174000553BF82E8EEFF81631F493948824839449
:1017500005E0B02EA2CF9DEFF91629F49A948824C3
:1017600012E0B12E9ACF8FEFF81689F480914A26B5
:10177000813009F0BAC20E94CBC9AA2009F4B5C2CF
:101780000E94D2300E9484D30E94E430AEC2CF2D9A
:10179000D0E0C90DD11DC130D105E1F4809198266A
:1017A0008823B1F40E9483B780E060E047EB5EE4F9
:1017B00020E00E947EBB0E94D2300E949BD00E94FB
:1017C0008DD10E94E4300E944682AA24A39449C08D
:1017D0000E944682C230D105B1F40E9483B780E0F6
:1017E00060E047EA5EE420E00E947EBB0E94D230C7
:1017F0000E949BD00E948DD10E94E4300E944682BC
:10180000AA24A39472C0C330D10589F48091CF3249
:1018100090E060E070E041E050E02BED02E00E94DB
:1018200076888093CF3280914A268130A9F0C430E7
:10183000D105B9F48091CE3290E060E070E041E0F3
:1018400050E027E905E00E9476888093CE328091AF
:101850004A26813009F00ACF0E94CBC910924A264D
:1018600005CFC530D10509F040C00E9483B786E995
:1018700090E00E94903EAC0180E060E022E00E9497
:10188000ACBB8DE190E00E94903EAC0182E167E04C
:1018900020E00E94ACBB80E061E04FE95EE420E024
:1018A0000E947EBB80E064E04AE95EE420E00E94A2
:1018B0007EBB80E062E04CEA52E320E00E94ACBBD9
:1018C000C0E0D0E0FE01E054FD4C8C2F65E040818B
:1018D00020E00E94B5BB2196CC30D10599F780E17C
:1018E0000E9405738823D9F3C1CE269709F0BECE96
:1018F00080EF0E9405730E9483B78DE190E00E9403
:10190000903EAC0182E167E020E00E94ACBB80E049
:1019100060E04CEA52E322E00E94ACBB0E94D2306D
:1019200080918732813011F40E949BD080E061E089
:101930004BE85EE420E00E947EBB80EC92E30E94D4
:10194000E4D2182F80E062E04CE75EE420E00E94E1
:101950007EBB8EE062E0412F50E022E030E000E00C
:10196000EE240E945BC1113051F480E061E04DE64D
:101970005EE420E00E947EBB1093422111C080E013
:1019800062E04FE55EE420E00E947EBB8EE062E014
:10199000412F50E022E030E000E0EE240E945BC1E5
:1019A00080914221813009F080C10E9483B780E09C
:1019B00060E04CEA52E322E00E94ACBB80E061E0D0
:1019C00049E55EE420E00E947EBB8BE061E042E5F9
:1019D0005EE420E00E947EBB80E062E04CE45EE4D6
:1019E00020E00E947EBB8BE062E045E45EE420E004
:1019F0000E947EBB80E063E04FE25EE422E00E9452
:101A00007EBB80E066E049E25EE420E00E947EBBAF
:101A10008DE190E00E94903EAC0182E167E020E021
:101A20000E94ACBB1092962611E010934D260E94A6
:101A300018CC882319F41092422113C10E94916D91
:101A400040916E2A85E061E050E022E030E000E065
:101A5000EE240E945BC14091992681E161E050E053
:101A600024E030E00E945BC140916D2A85E062E095
:101A700050E022E030E00E945BC140919B2A5091EF
:101A80009C2A4115510541F480E162E043E25EE4A5
:101A900020E00E947EBB08C080E162E024E030E0EC
:101AA00000E0EE240E942CC06091692A70916A2A9D
:101AB00080916B2A90916C2A20E836E948E950E041
:101AC0000E946ADA81E064E0A90122E030E000E0EF
:101AD000EE240E945BC183E064E041E25EE420E02A
:101AE0000E947EBB6091692A70916A2A80916B2A5C
:101AF00090916C2A28EE33E040E050E00E946ADAD0
:101B0000CA01B90120E137E240E050E00E946ADA00
:101B10009B01AC0184E064E0A90124E030E001E035
:101B20000E945BC16091692A70916A2A80916B2A38
:101B300090916C2A2AE030E040E050E00E946ADA9E
:101B4000CA01B90124E630E040E050E00E946ADAC0
:101B50009B01AC0188E064E0A90122E030E00E9432
:101B60005BC16091912A7091922A8091932A909101
:101B7000942A20E836E948E950E00E946ADA8CE0CD
:101B800064E0A90122E030E000E00E945BC18EE049
:101B900064E04FE15EE420E00E947EBB6091912A08
:101BA0007091922A8091932A9091942A28EE33E0A2
:101BB00040E050E00E946ADACA01B90120E137E250
:101BC00040E050E00E946ADA9B01AC018FE064E0E3
:101BD000A90124E030E001E00E945BC16091912AFC
:101BE0007091922A8091932A9091942A2AE030E071
:101BF00040E050E00E946ADACA01B90124E630E010
:101C000040E050E00E946ADA9B01AC0183E164E0AD
